:020000040800F2
:100000000050002015440108B14401083D300108AA
:10001000B1440108B1440108B144010800000000E6
:10002000000000000000000000000000B1440108D2
:10003000B144010800000000B1440108350A01087C
:10004000B1440108B1440108B1440108B1440108B8
:10005000B1440108B1440108E9D50008F3D500080E
:10006000F1D50008EFD50008EDD50008DD530008F4
:10007000CD530008BD530008AD5300089D53000840
:100080008953000877530008B1440108B1440108BE
:10009000B1440108B1440108B1440108EBD500089E
:1000A000B144010869070108B14401085907010872
:1000B0004D0701083D0701082D070108C756000834
:1000C000CD560008BD560008C3560008B1440108CB
:1000D000B1440108E1FA0008D5FA0008C9FA00089D
:1000E000E7D50008B1440108B14401080000000050
:1000F0000000000000000000000000000000000000
:0C01000000000000000000005FF808F1A3
:100110002DE9F04F914BADB01D780093002D00F00C
:10012000A7808F4B1868002801F012870DF062FA43
:10013000DFF85C92DFF85C82D9F800000BF036FA49
:10014000002801F00587D9F800000BF02CFA0928E7
:10015000844C01D03F2855D14FF0000A57465546F0
:1001600026680AEB080B36B132465AF808107E486A
:1001700018F0D1FE20B90DB15F4601E05D465F4643
:100180000AF1080ABAF5907FEBD1F5B1D5F800A0D5
:10019000D7F800B0DFF8D0C123681AF803001BF8C5
:1001A0000310814211D15A1CDFF8BCE149B92D2B53
:1001B00007D86C48026020200EF803000EF80210E9
:1001C00003E00CF803002260E6E723680BB1BD42B0
:1001D0000FD0664806F088F9BD4207D855F8080BDD
:1001E00006F082F909200EF054FDF5E709F0BCFE97
:1001F00000265D4D23689E429ED2A85D0EF049FD0B
:100200000136F7E723686BB9042804D1564806F095
:1002100089FB01F09DBE0C2841F09686544806F0FB
:1002200063F922E00C28F9D00A2841F041864E4EAD
:10023000504806F059F92321304618F05EFE354645
:1002400008B1801B206023680022002B41F0348617
:10025000002A41F04C8630220021434818F016FE57
:10026000009B1B78002B01F0738609F07DFE63E78D
:10027000414B03F13007414BEA18EB58002B01F0DA
:100280005A803F4C3F4922603F4A26468946924663
:100290000B60059300238DF819303C4814238DF82A
:1002A000183004AB04920360D9F80000DFF8D48062
:1002B0000BF07CF9002801F02A80D8F800000BF040
:1002C00072F93368834693F8481019B9242863D12A
:1002D00001221DE0012903D14D2808BF022204E0BC
:1002E000022907D13C2808BF032218BF002283F847
:1002F000482085E003290ED140284FF0000102D9A3
:1003000083F84810D0E758711971D9719871042297
:1003100083F84820C8E7042907D1997983F8490070
:1003200080EA01029A710522F2E7052968D158791D
:1003300019798842987908D98BEA00009871481C8D
:1003400018710B4483F808B0AEE7584503D1062274
:1003500083F848205AE00022DAE700BF04140020A6
:100360002436002000140020D013002010B2010811
:1003700015B20108F3BB010854910108EC400020BC
:100380001836002020360020B9B500081C360020A1
:10039000CC1300202C970108BE490B7803F004030E
:1003A00003F0FF0E002B7FF47FAF23281DD1009AAE
:1003B0000123D8F800001370B74B01911860B74BB8
:1003C0001860B74B586010201872B648C3F800A0E8
:1003D000036083F809E0B44806F086F809F0C4FD2C
:1003E00001990B7843F002030B70B04B1B681B782C
:1003F0005B4505D1AE4BAF4A1A60AF4BAF4ADA60EE
:10040000336893F84820062A7FF44EAF93F849806A
:10041000B8F1520F00F0818600F2D880B8F1340FA5
:1004200000F04A8467D8B8F1240F00F0D0842DD8AA
:10043000B8F1040F00F0348215D8B8F1020F00F0C3
:10044000148200F22182B8F1010F40F0A587032049
:100450000EF00AFC00200EF0C8FB40460EF0C5FB73
:10046000152000F030BFB8F10A0F00F05782B8F144
:10047000220F00F00084B8F1050F40F08D871A209C
:100480000EF0F2FB0026DFF84C821AE2B8F12C0FD6
:1004900000F0F2841BD8B8F1280F00F0D484B8F132
:1004A0002A0F00F0E384B8F1260F40F07587844EE0
:1004B00006200EF0D9FBB6F8C8010EF0D8FBB6F84E
:1004C000CC010EF0D4FBB6F8D00100F0F9BEB8F1C3
:1004D000300F00F08785B8F1320F00F02B85B8F1AE
:1004E0002E0F40F05987764E40200EF0BDFB06F1EE
:1004F000400800F067BDB8F1450F00F0138636D80C
:10050000B8F13B0F00F0B08319D8B8F1380F00F004
:100510008784B8F13A0F00F02483B8F1360F40F029
:100520003B87684B664E187806F12808C0EBC00080
:10053000C0B20EF099FBDFF8A09100F03FBDB8F11A
:10054000400F00F0FE84B8F1420F00F00A85B8F1C8
:100550003D0F40F021875A4E02200EF085FB96F8A1
:100560008F020EF042FB96F88E0200F0ACBEB8F19E
:100570004B0F00F0AC8410D8B8F1470F00F087851E
:10058000C0F07185B8F1490F40F0068702200EF0E7
:100590006BFB4D4B988A00F093BEB8F14F0F00F003
:1005A000AF85B8F1500F00F09985B8F14D0F40F0CC
:1005B000F386464EDFF8248130784FF0000900EBD7
:1005C0004000C0B20EF050FB00F09CBCB8F1700FC0
:1005D00000F0228300F28680B8F1660F00F0DA8125
:1005E0002CD8B8F15E0F00F036860DD8B8F15A0F4E
:1005F00000F0E585B8F15C0F00F00086B8F1540F0B
:1006000040F0CA8600F089BDB8F1640F00F0768131
:1006100000F29681B8F1600F40F0BE86284E0320AC
:100620000EF022FB96F8D5010EF0DFFA96F8EE01F7
:100630000EF0DBFA96F8ED0100F045BEB8F16C0F54
:1006400000F07F8216D8B8F1680F00F06182C0F028
:10065000CD81B8F1690F40F09F86DFF870800026E9
:1006600098F80000DFF87890400000F0FE000EF0EF
:10067000FBFA5BE2B8F16E0F00F0778200F29A822B
:1006800006200EF0F1FA00200EF0FAFA104B18884E
:1006900000F016BEF8350020CC13002018180020FA
:1006A000E00900202436002040B20108AC400020C0
:1006B000F04F0020EFBEADDE00ED00E00400FA05D3
:1006C000303B0020602700200C2D0020B04100208E
:1006D000CC95010882B20108B0400020883D00207E
:1006E00058170020B8F17D0F00F03F855BD8B8F1B6
:1006F000750F00F0AD823ED8B8F1730F00F0408363
:1007000000F2AE80B8F1720F40F04686D94E162046
:100710000EF0AAFAB6F848020EF0A9FAB6F8CC0024
:100720000EF0A5FAB6F8CE000EF0A1FAB6F8D00099
:100730000EF09DFAB6F89C020EF099FA00200EF029
:1007400054FA00200EF051FA00200EF04EFA96F8FE
:1007500023020EF04AFA96F844020EF046FA002000
:100760000EF043FAB6F9F0310A2093FBF0F080B2B4
:100770000EF07DFA58E3B8F1780F00F04681B8F139
:100780007C0F00F0E384B8F1770F40F00586DFF8C6
:100790000C83002698F800000EF066FADFF800A33C
:1007A000DFF80093E2E2B8F1A00F00F002833FD837
:1007B000B8F17F0F00F02384C0F0F284B8F1960FF7
:1007C00040F0EA850F200EF04FFAAB4B18880EF080
:1007D0004EFAAA4B188880B20EF049FAA84B1B6853
:1007E000C3F3C000C3F38002800040EA4200C3F3B9
:1007F00040021043C3F3401240EAC20003F010036A
:1008000018430EF034FA0EF023F90EF039FA994B32
:1008100093F8AC040EF0E9F99A4B18886428A8BF45
:1008200064200EF024FA02200EF0DFF9964B20E24D
:10083000B8F1F10F00F04681B8F1FE0F00F0AB8285
:10084000B8F1F00F40F0A8858A4E04200EF00CFAA3
:10085000B6F8F4010EF00BFAB6F8F20100F030BD74
:100860004FF000094FF0010B52E204200EF0FCF9AA
:10087000DFF83482002618F8060001360EF0B5F9CC
:10088000042EF8D100F03DBD03200EF0EDF9032059
:100890000EF0ABF900200EF0A8F9012000F013BD16
:1008A00006200EF0E1F9DFF80482002618F80600B1
:1008B00001360EF09AF9042EF8D1744B187800F036
:1008C000FFBC18F8060001360EF08FF90B2EF8D198
:1008D000DFF8DC81002618F8060001360EF085F9F5
:1008E000082EF8D1DFF8CC81002618F80600013672
:1008F0000EF07BF9072EF8D100F003BD07200EF0B3
:10090000B3F9E7200EF071F95A4B58790EF06DF9F2
:1009100000200EF06AF9042000F015BC5C4812F0CB
:10092000C3FBC6B230460EF09FF9DFF88C81464417
:10093000B04500F0E68418F8010F0EF056F9F7E71D
:100940000B200EF091F94C4B18880EF090F94B4BA0
:10095000188880B20EF08BF9494B1B68C3F3C000B6
:10096000C3F38002800040EA4200C3F34002104318
:10097000C3F3401240EAC20003F0100318430EF024
:1009800076F90EF065F80EF07BF93A4B93F8AC046B
:1009900000F099BC12200EF067F93E4BDFF81C9175
:1009A0001B890026B3F5007F94BF4FF001084FF07C
:1009B000040859F82600013690FBF8F080B20EF0DA
:1009C00056F9032EF5D1344E30880EF050F9B08828
:1009D0000EF04DF930890EF04AF900200EF047F97B
:1009E00000200EF044F9002000F06ABC10200EF048
:1009F0003BF9DFF8CC80002618F8060001360EF02F
:100A0000F4F8102EF8D100F07CBC1A4E70200EF0D5
:100A10002BF9B0464FF0000A4FF00E09B6F854011A
:100A20000EF025F9B6F856010EF021F9B6F8580186
:100A30000EF01DF996F85A010EF0D7F896F85B0102
:100A40000EF0D3F896F85C010EF0CFF896F85D0141
:100A50000EF0CBF809FB0A830AF1010AD3F85E0114
:100A60000EF00EF9BAF1080F06F10E06D6D100F01D
:100A700048BC00BF303B0020CC3700202C3B00207E
:100A8000502D002028140020CF370020242D0020D6
:100A900096400020002D0020C01F0020F9350020C6
:100AA000FA3500205491010878B201087DB201089E
:100AB0008EB2010897B20108954000200C13002067
:100AC000FC09002070200EF0CFF8C44E06F170082B
:100AD00096F8E4000EF089F896F8E5000EF085F837
:100AE00096F8E6000EF081F896F8E7000EF07DF833
:100AF00096F8E8000EF079F896F8E9000EF075F82F
:100B0000073696F8E3000EF070F84645E0D1F8E3BA
:100B100010200EF0A9F8DFF80083002618F8060070
:100B200001360EF062F8102EF8D1EAE398F80030A2
:100B30009E4280F0E68339F816000EF098F80136F0
:100B4000F4E7A74E06200EF08FF830880EF08FF8ED
:100B500070880EF08CF8B6F904300A2093FBF0F0A0
:100B600023E004200EF080F8ECE207200EF07CF881
:100B70009C4B1888FF28A8BFFF20C0B20EF035F8A4
:100B8000994B186880F3100080B20EF070F8974B04
:100B900018880EF06CF8914B93F82322944B186848
:100BA0002AB10A23584380F3100080B288E300F38F
:100BB0000F00FAE78F4E0C200EF056F83368B0465F
:100BC00018780EF012F833684FF0000998780EF09C
:100BD0000CF8D8F80030874E4B44587909F10109D8
:100BE0000EF003F8B9F1030FF3D13368187A0DF062
:100BF000FCFF3368D8780DF0F8FF336818790DF0F2
:100C0000F4FF336858890EF032F83368587A0DF0E3
:100C1000ECFF3368587856E31E200EF025F8DFF815
:100C2000DC810026D8F80030334458780DF0DDFF21
:100C3000D8F800303344D87A0DF0D7FFD8F8003018
:100C40003344587D01360DF0D0FF0A2EEAD158E327
:100C50002F200EF009F8684E16F8010F002800F05A
:100C600050830DF0C2FFF7E701200DF0FDFF634B4D
:100C70001B68187827E350200DF0F6FF574E4FF011
:100C80000C0906F150085E4A96F8AD34043609FBAB
:100C9000032393F838000DF0A8FF96F8AA040DF08E
:100CA000A4FF96F8AB040DF0A0FF96F8AC040DF08D
:100CB0009CFF4645E7D124E35A200DF0D5FF474E6F
:100CC00006F15A0896F802050DF08FFF96F8FD041C
:100CD0000DF08BFF96F8FE040DF087FF96F8FF04E9
:100CE0000DF083FF96F800050DF07FFF063696F8AD
:100CF000FB040DF07AFFB045E4D102E3BBF1000F35
:100D000000F0FF825FFA89F00DF0AEFF4FF0000BAC
:100D100000263C4B1B789E42F0DA3B4B0021F05CF6
:100D20004FF00C0E0EFB01F313F807C0844503D0FF
:100D300001311F29F6D10CE0314A1344D3F834A015
:100D4000504612F0B1F90146BBF1000F00F0F982F4
:100D500089440136DDE700FB02F313F807E08E4516
:100D600000F0FC8201321F2AF5D1013698F80030DC
:100D70009E4280F0C68216F80A1000220C20EAE794
:100D800008200DF071FF0126F0B201360DF02DFFA5
:100D9000092EF9D1B5E208200DF066FFDFF87C805E
:100DA000002638F8160001360DF061FF042EF8D148
:100DB000A7E20C200DF058FF144B18680DF060FFEF
:100DC000134B18680DF05CFF124B1868BBE1042050
:100DD0000DF04AFF014B9868B5E100BF303B0020A1
:100DE000B81F002014170020C8160020D44300208C
:100DF00020130020C835002053910108081400205A
:100E000054910108F9350020FA350020E8F7FF1F5A
:100E1000ECF7FF1FF0F7FF1F84390020EC160020CD
:100E200004200DF021FFDA4E96F816020DF0DDFEDB
:100E300096F81A020DF0D9FE96F819020DF0D5FEBB
:100E400096F81B023FE2D24E07200DF00DFFB6F8D8
:100E50001E020DF00CFFB6F820020DF008FF96F808
:100E600022020DF0C2FEB6F8240229E201200DF0A4
:100E7000FBFEC74B587926E2C54E10200DF0F4FE5C
:100E800096F840020DF0B1FEB6F84C020DF0EFFE00
:100E9000B6F848020DF0EBFEB6F84A020DF0E7FE98
:100EA00096F842020DF0A1FEB6F854020DF0DFFEF6
:100EB000B6F856020DF0DBFE96F84E020DF095FEE8
:100EC00096F84F020DF091FEB6F85202F8E1B04EDE
:100ED00008200DF0C9FE96F89A020DF086FE96F8ED
:100EE0009B020DF082FEB6F89C020DF0C0FE96F853
:100EF0009E020DF07AFEB6F8A0020DF0B8FE96F84C
:100F0000A202E0E1337808F10208994580F0F98106
:100F100018F8020C0DF069FE18F8010C09F101092E
:100F200000EB800000EB800000F2EE2080B20DF0BC
:100F30009EFEE7E701200DF097FE954B93F84402E3
:100F4000C1E108200DF090FEDFF84482002606EB98
:100F5000080393F8380201360DF047FE082EF6D14B
:100F6000CFE18B4E10200DF07FFE70790DF03DFE2D
:100F7000B0680DF085FE96F840020DF036FEB6F82A
:100F8000C8010DF074FEB6F8CC010DF070FEB6F895
:100F9000D0010DF06CFEB6F81E020DF068FEB6F83A
:100FA00020028DE113F90920824200F0DD810C332B
:100FB0003C2BF7D10836B04500F0A38196F9A60284
:100FC0000023EFE7B6F864030DF051FE96F86603D0
:100FD0000DF00BFE043696F863030DF006FEB045E7
:100FE000F0D18EE180200DF03FFE6A4E06F18008C0
:100FF00056F8040F0DF044FEB045F9D181E18D2083
:101000000DF032FE00264FF0060A0AFB06F94FF0FB
:10101000000B5FFA86F840460DF0E7FD5FFA8BF0B3
:101020000DF0E3FD5A4B0BEB0901194491F8A403B1
:101030000BF1010B0DF0D9FDBBF1060FEBD1013621
:10104000062EE2D1002606200DF0CFFDF0B20DF005
:10105000CCFD4F4B334493F8C80301360DF0C5FD6A
:101060000B2EF0D14DE10D200DF0FEFD08F056F8ED
:10107000494E40F00200C0B20DF0B7FD30880DF0CF
:10108000FFFDF0680DF0FCFD08F028F85BE00DF0C6
:10109000A3FD064684200DF0E7FD30460DF0F0FD7F
:1010A0003D4B0DF13008DA6806F1800393428CBFA6
:1010B000C6EB02094FF0800908F00AF94A463046AB
:1010C000414608F043F9814600264E4580F21981D9
:1010D00018F806000DF089FD0136F6E72C4E0420C5
:1010E0000DF0C2FD01200DF080FD96F859050DF0C0
:1010F0007CFD96F857050DF078FD96F85805E2E06E
:101100000B200DF0B1FD00200DF06FFD00200DF063
:101110006CFD00200DF069FD11E001200DF0A4FD33
:101120000020D0E013200DF09FFDDFF87080002636
:1011300018F8060001360DF058FD0B2EF8D10020EE
:101140000DF09EFD00200DF09BFDDAE0104E062014
:101150000DF08AFDB6F8D6000DF089FDB6F8D8007E
:101160000DF085FDB6F8DA00AAE0094E05200DF075
:101170007BFD96F826020DF038FD96F827020DF05B
:1011800034FD96F828020DF030FDB6F8DC0097E04B
:10119000303B0020103E00208400002082B2010875
:1011A000CD4E03200DF060FD96F8C5010DF01DFD3C
:1011B00096F8C6010DF019FD96F8C70183E0C64EFA
:1011C00006200DF051FDB6F8D83123B108200DF0FE
:1011D0000CFD012005E096F8DA010DF006FD96F809
:1011E000EA010DF002FD96F8E3000DF0FEFC96F822
:1011F000E2000DF0FAFCB6F8DE0061E0B64EDFF872
:10120000DC8211200DF030FD96F8DC010DF0EDFCD4
:10121000D8F80030188C0DF02AFDD8F80030588C22
:101220000DF025FDB6F8DE010DF021FDB6F8E00168
:101230000DF01DFDD8F80030988C0DF018FDD8F891
:101240000030D88C0DF013FDB6F8E2010DF00FFD63
:10125000B6F8E40134E0A14E11200DF005FD33682D
:10126000588D0DF004FD3368988D0DF000FD336846
:10127000D88D0DF0FCFC336893F828000DF0B5FC18
:10128000336893F833000DF0B0FC336893F8360000
:101290000DF0ABFC336893F837000DF0A6FC00208E
:1012A0000DF0A3FC00200DF0A0FC336893F835008E
:1012B0000DF09BFC3368588F0DF0D9FC3368188F04
:1012C0000DF0D5FC1DE00DF090FC1AE040F23084EA
:1012D000B8F1D00F00F04A84B8F1D20F40F0168177
:1012E0000DF066FC020600F14E847D4B1B785B0717
:1012F00004D4022828BF00200CF086FA00200DF04C
:10130000B3FC0DF081FC2368002283F84820754B64
:10131000754C18680CF06EF994F82C305BB1734B77
:1013200058590AF099FE0FF020FB002384F82C3066
:101330006F4A704BDA604C35982D00F00986FEF745
:101340009ABFD046CAEB08008842BFF602AD18F833
:10135000010B01910DF049FC0199F3E74B4493F81F
:1013600038000DF042FC00E5C0B20DF03EFCB6F8CE
:10137000A8020DF07CFC96F8AA020DF036FC96F857
:10138000AB020DF032FC96F8AD020DF02EFC96F893
:10139000AC020DF02AFC0DE6B8F15B0F15D10DF093
:1013A00007FC4D4E86F8DA010DF002FC86F8EA01E2
:1013B0000DF0FEFB86F8E3000DF0FAFB86F8E20084
:1013C0000DF000FCA6F8DE0098E700F26282B8F1AA
:1013D000370F32D15B794FF00708B3FBF8F8C8EB51
:1013E000C8029B1A13F0FF0F02D00BF03FFB85E7FA
:1013F0005FFA88F8B8F1000F80D00DF0D9FB4FFAF2
:1014000080F948460AF0BAFE06460028EDD080F87A
:1014100000900DF0D7FB70800DF0CAFB30710DF01D
:10142000C7FB70710DF0C4FBF0710DF0C1FB08F14A
:10143000FF385FFA88F8B071DCE700F22881B8F174
:101440002B0F04D10DF0B4FB234B587156E700F27B
:101450008680B8F1250F08D11F4E0023B3600DF030
:10146000BBFBB3681843B06048E752D8B8F10B0F24
:1014700019D111220021204817F008FDDFF85890FB
:101480004FF0000833685B79102B28BF1023984574
:10149000BFF434AF0DF08CFB08EB090383F866054D
:1014A00008F10108EEE7B8F1230F2FD10DF080FB12
:1014B0001328064699D80DF07BFB00220C2101FB76
:1014C00002F307EB030E9EF808E0864500F0CB849C
:1014D00001321F2AF3D188E7303B00200814002096
:1014E000F83500201C360020E0090020EC400020E8
:1014F0000400FA0500ED00E096400020B8F1FA0F74
:1015000004D1CE4B1B785A0740F137830BF0AEFA6B
:10151000F7E6B8F1270F0DD10DF054FBC84EC6F811
:10152000C8010DF04FFBC6F8CC010DF04BFBC6F81F
:10153000D001E3E6B8F1290FE8D10DF043FBC04E2E
:10154000A6F81E020DF03EFBA6F820020DF030FBBF
:1015500086F822020DF036FBA6F82402CEE6B8F19A
:10156000310F14D10DF024FB1F2806463FF63DAF86
:1015700023685B79052B7FF438AF0DF02DFBB04B62
:1015800003EB8603C3F8E40210F016FFB6E64BD86F
:10159000B8F12D0F32D10DF00BFBA94E86F84002A9
:1015A0000DF010FBA6F84C020DF00CFBA6F848025B
:1015B0000DF008FBA6F84A020DF0FAFA236886F847
:1015C00042025B79082B07D90DF0FCFAA6F8540209
:1015D0000DF0F8FAA6F8560223685B790C2B7FF61B
:1015E0008DAE0DF0E5FA86F84E020DF0E1FA86F8C0
:1015F0004F020DF0E7FAA6F852027FE6B8F12F0F7E
:1016000084D18F4E06F140080DF0DCFAA6F8640391
:101610000DF0CEFA86F866030DF0CAFA043686F8A5
:1016200063034645F0D169E6B8F1330F05D10DF0FB
:10163000BFFA834B83F8440260E6B8F1350F7FF4BC
:1016400065AF0DF0B5FA0E2880463FF6CEAE0DF030
:10165000AFFA03283FF6C9AE794B062606FB0836DB
:1016600086F802050DF0A4FA86F8FD040DF0A0FA44
:1016700086F8FE040DF09CFA86F8FF040DF098FA47
:1016800086F800050DF094FA86F8010536E6B8F103
:10169000440F04D16B4B012283F82C202EE672D824
:1016A000B8F13E0F09D10DF083FA654E86F88F022E
:1016B0000DF07EFA86F88E0220E62CD8B8F1390FAC
:1016C00011D10DF075FA5E4E86F816020DF070FA23
:1016D00086F81A020DF06CFA86F819020DF068FA15
:1016E00086F81B020AE6B8F13C0F7FF40FAF564EA6
:1016F000D6F800800DF05CFA0128A8BF012088F818
:10170000000033681B78012B18BF504A504B08BFAC
:10171000504A1A60F2E5B8F1410F0CD1DFF8208190
:1017200000260DF045FA06EB08030136082E83F873
:101730003802F6D1E2E5B8F1430F7FF4E7AE0DF0E1
:1017400037FA3F4E0023B36070710DF045FAB3686D
:101750001843B0600DF02CFA86F840020DF032FA12
:10176000C6F8C8010DF02EFAC6F8CC010DF02AFA21
:10177000C6F8D0010DF026FAA6F81E020DF022FAE6
:10178000A6F82002BAE5B8F14C0F19D10DF010FA05
:101790002B4E86F89A020DF00BFA86F89B020DF09C
:1017A00011FAA6F89C020DF003FA86F89E020DF0DD
:1017B00009FAA6F8A0020DF0FBF986F8A2029DE551
:1017C00013D8B8F1480F09D107F0EAFD224A0023E7
:1017D0001370224A1370224A13608FE5B8F14A0F42
:1017E0007FF494AE0DF0EEF988E5B8F14E0F39D1E3
:1017F0000DF0DEF9112806463FF6F7AD0DF0D8F9E9
:10180000DFF83C8006F5967608F816000DF0DAF958
:1018100040F2ED239842424605DD40F6CA03984265
:10182000A8BF184601E040F2EE2002EB4603A0F20A
:10183000EE20192290FBF2F058705FE5F835002099
:10184000303B0020E00900200814002033B60008D7
:10185000A402002031B90008C4130020C5130020E1
:10186000C8130020B8F1510F7FF450AEDD4B1B7848
:10187000012B3FF643AD0DF09BF9DB4E86F8590581
:101880000DF096F986F857050DF092F986F858058F
:1018900034E5B8F1D30FA5D000F27E81B8F1CC0FBA
:1018A00052D15B79092B7FF6A0ADD04ED6F80080DF
:1018B0000DF07EF988F80000D6F800800DF078F978
:1018C00088F802000DF074F933686428A8BF64201A
:1018D00058710DF06DF933686428A8BF64209871C1
:1018E0000DF066F93368FF28A8BFFF20D8710DF00E
:1018F0005FF9D6F80080642828BF642088F80800C3
:101900000DF056F988F80300D6F800800DF050F974
:1019100088F80400D6F800800DF054F92368A8F880
:101920000A005B790A2B05D9D6F800800DF040F942
:1019300088F8090023685B790B2B7FF6DFAC3668EB
:101940000DF036F97070D9E400F2B880B8F1610F8B
:101950000DD10DF02DF9A44E86F8D5010DF028F922
:1019600086F8EE010DF024F986F8ED01C6E47FD883
:10197000B8F15D0F38D10DF01BF9DFF874829A4E83
:10198000D8F8009086F8DC010DF01CF9A9F82000C9
:10199000D8F800900DF016F92368A9F822005B79B9
:1019A000052B13D90DF00EF9A6F8DE010DF00AF99A
:1019B000D8F80090A6F8E0010DF004F9A9F8240089
:1019C000D8F800800DF0FEF8A8F8260023685B79AF
:1019D0000D2B7FF693AC0DF0F5F8A6F8E2010DF0B3
:1019E000F1F8A6F8E40189E4B8F15F0F7FF48EAD59
:1019F0007F4ED6F800800DF0E5F8A8F82A00D6F85A
:101A000000800DF0DFF8A8F82C00D6F800800DF06B
:101A1000D9F8A8F82E00D6F800800DF0C9F888F89B
:101A20002800D6F800800DF0C3F888F83300D6F807
:101A300000800DF0BDF888F83600D6F800800DF073
:101A4000B7F888F837000DF0B3F80DF0B1F8D6F814
:101A500000800DF0ADF888F83500D6F800800DF064
:101A6000B1F8A8F83A0036680DF0ACF8308745E4D4
:101A7000B8F1C80F3FF442ACB8F1CA0F7FF446ADDD
:101A80005B4E4FF00008D6F800900DF091F8C1447D
:101A900089F80100D6F800900DF08AF8C14489F861
:101AA0000B00D6F800900DF083F8C14408F101084E
:101AB000B8F10A0F89F81500E5D11FE4B8F1CF0F8E
:101AC0007FF404AC0DF07EF86FF4AF6E00EB0E0304
:101AD0009BB2454EC62B98BFA6F848020DF072F88F
:101AE000A6F8CC000DF06EF8A6F8CE000DF06AF85E
:101AF000A6F8D0000DF066F8A6F89C020DF058F894
:101B00000DF056F80DF054F80DF052F886F8230257
:101B10000DF04EF886F844020DF04AF80DF052F838
:101B200000EB80004000A6F8F0010DF041F8CBE595
:101B3000B8F1CD0F0AD12F4B1B7858073FF5DEAB1C
:101B40002D4B4FF4C8721A80FFF7D8BBB8F1CE0FF7
:101B50007FF4DCAC274B1B7859073FF5CFAB274A06
:101B6000137843F004031370FFF7C8BB214B1B78B5
:101B70005E073FF5C3AB08F0F5FF0BF09DFD08F0E5
:101B80000BFCFFF7BBBB00F07F00032828BF002041
:101B90000BF072FDFFF7B2BBB8F1DC0F0ED10DF008
:101BA00007F8114E86F8C5010DF002F886F8C60157
:101BB0000CF0FEFF86F8C701FFF7A0BB00F284809F
:101BC000B8F1D90F1CD10CF0FDFF074EA6F8D600D6
:101BD0000CF0F8FFA6F8D8000CF0F4FFA6F8DA0035
:101BE000FFF78CBB7A270020303B0020C83500204F
:101BF00008140020F8350020400E0020A11300201A
:101C000042D8B8F1D40F2FD15B790F2B7FF4EDAB15
:101C10000CF0CEFF072880463FF6E7AB0CF0D2FF72
:101C2000CD4B0E2606FB0836A6F854010CF0CAFF71
:101C3000A6F856010CF0C6FFA6F858010CF0B8FF44
:101C400086F85A010CF0B4FF86F85B010CF0B0FF87
:101C500086F85C010CF0ACFF86F85D010CF0BCFF6F
:101C6000C6F85E01FFF74ABBB8F1D60F7FF44EAC61
:101C7000DFF81C8300260CF0A5FF28F816000136BB
:101C8000082EF8D1FFF73ABBB8F1DA0F12D10CF0F9
:101C90008FFFB14E86F826020CF08AFF86F82702E5
:101CA0000CF086FF86F828020CF08CFFA6F8DC000A
:101CB000FFF724BBB8F1DB0F7FF428ACA74B186803
:101CC00008F01EFDFFF71ABBB8F1F20F29D10CF096
:101CD0006FFF0F2806463FF688AB0CF069FF9E4B5E
:101CE000C6EBC6061E4486F8E4000CF061FF86F8D9
:101CF000E5000CF05DFF86F8E6000CF059FF86F871
:101D0000E7000CF055FF86F8E8000CF051FF86F86C
:101D1000E9000CF04DFF86F8EA000EF00BFCFFF72F
:101D2000EDBA38D8B8F1DD0F26D10CF041FF80466E
:101D30000CF03EFF06460CF03BFF0F283FF6E6ABEB
:101D4000B8F1050F0BD8052E3FF6E0AB824B06210C
:101D500001FB0832931983F8A403FFF7CFBAB8F157
:101D6000060F7FF4D3AB0A2E3FF6D0AB7A4B334449
:101D700083F8C803FFF7C2BAB8F1EF0F7FF4C6AB20
:101D80000CF020FF744EA6F8F4010CF01BFFA6F82F
:101D9000F201FFF7B3BAB8F1F50F7FF4AFABDFF89C
:101DA000F4A10120D0460CF05FFF00266C4B3146B9
:101DB00030226C481E708AF80060DFF8DCB117F042
:101DC00065F8DFF8A0918DF80F60674E9DF80F3031
:101DD00096F832209A4232D99DF80F3006EBC303B1
:101DE00093F83530DB0723D59DF80F3006EBC3039E
:101DF00093F834303BF91330002B19DD9DF80F3088
:101E000006EBC3039B6B18790BF0BAF998F8003016
:101E10004A2149F823000BF0D9F998F8003059F815
:101E200023000BF0B6FB98F80030013388F800303F
:101E30009DF80F300133DBB28DF80F30C6E79AF80A
:101E400000000CF0D2FE0CF0DFFE484B18680BF0DF
:101E5000D1FB236818680AF0FFF8236818680BF0B4
:101E6000C3FEFFF74BBA424ADFF8EC80134493F805
:101E7000303006F5957608EB860673710CF098FE07
:101E8000B0710CF095FEF0710CF092FE334B3949B5
:101E90001A6808F1CC030B60374B307200201A60CF
:101EA0000EF027FF354B80F001001870FFF726BABF
:101EB0000D2828D1FEF7BBB9591E685C202819D11E
:101EC00001220B46FEF7C1B90835B5F5907F16D053
:101ED00055F808102A4805EB080604F059FD0028BB
:101EE000F2D0284B9E420AD27368984700232360A1
:101EF000FEF7B1B902B123600025F554E8E72248A6
:101F000004F0F2FAF2E77F2809D11D4A013B0021D3
:101F10001E482360D15404F0E7FAFEF70DB92F2BC9
:101F20003EF60AA9A0F12002D2B25E2A3EF604A92A
:101F300013B920283EF400A95A1C2260104AD0543C
:101F40000CF0A7FEFEF7F8B87F28EBD1FEF7F4B847
:101F50002DB0BDE8F08F00BF303B002008140020FA
:101F60005D030020DC170020E00900201C36002063
:101F7000549101084C18002050180020A0020020A5
:101F8000D01300204C98010820B201083CB201088F
:101F9000AC130020DB35002084390020764B2DE97E
:101FA000F04F1B68754D9A6A754BA3B01A802B7859
:101FB000012B04D1734B1A80734A12885A80734CD8
:101FC0002378002B00F0D1860EF0A8FC704B049013
:101FD0009B680BB16F4898476F4B704E1B78C3B12D
:101FE0006F4BB3F90620B6F84A329A4211DC737986
:101FF000012B01D0192B02D196F893224AB90E2B4E
:1020000007D0082B05D0674B00229A80664B002230
:102010009A6096F81472002F30D0644B1B889B078F
:102020002CD0634B6349D3F82080404611F09CFFCD
:10203000F8B9404614F0F6FC5F4B196811F0ECFD5E
:1020400014F076FCB0F5617FA8BF4FF4617011F019
:102050008FFD5A4911F094FE10F08CFD80463846F1
:1020600011F086FD414611F0D7FD14F061FC00B27D
:1020700000E000204B4AD3881844D08096F84E32B6
:102080004F4A23B949490988002900F0A1801278F4
:10209000444F002A50D0022B09D0032B19D196F8B7
:1020A0004F32C3EB431203EB8203DB000FE0454BDF
:1020B000D3F8F820B2F57A7F05DB44F6206393422B
:1020C000A8BF134601E04FF47A7303F57A739BB20D
:1020D00000E063883C4A10682A78B3FBF0F0461CA5
:1020E00036B2092AA68005D1264A3988D3801180C4
:1020F00079885180B4F906A0DFF8A8B00023DFF892
:102100008CE03BF913800EF1080939F913100EF138
:10211000100C0AFB01F191FBF6F13CF813202CF8AE
:102120001380C2EB08020A4429F813200133042B60
:10213000E5D1AEF8060002E0E388013BE380B4F9A4
:102140000600124A00284FF0000312DDB2F90460C5
:1021500010321E4932F813E031F91310414391FB5C
:10216000F6F1C1EB0E0127F813100133042BF0D167
:1021700033E0D38031E000BF48170020EA1600208A
:10218000CC370020EC16002028140020800A002004
:102190000C2D002018130020A0020020303B00204E
:1021A00058170020B01F0020A41F0020F035002089
:1021B000D03A00208FC2753C8C180020EFB6B04496
:1021C000460E002098000020D01F0020880A002022
:1021D0001378E180002B00F0AA80A74B93F85002FF
:1021E00020B1A64B1B689F0001F11684A44B1F6809
:1021F0002B7807F104090593A24B00251B681B7877
:1022000006936B00022D07939F4B15BF38787878A3
:1022100097F8028097F8098033F9154011F0A8FC6F
:102220009A4911F0ADFD4FF08041064611F0B0FE25
:1022300060B14FF08041304611F0E4FB944911F059
:10224000EBFC0146304611F0DFFB0646204611F05C
:102250008FFC904911F094FD0021044611F098FE86
:10226000002841F0388404F1004B8B4A4FEA850A7C
:1022700042F825B0B8F1000F23D0404611F078FCA9
:10228000824911F07DFD59468046584611F0C4FC44
:102290000146584611F0C0FC214611F0BDFC4146F4
:1022A00011F0BAFC414607904FF07E5011F0AAFBA6
:1022B000214611F0B1FC079B0146184611F0A4FB22
:1022C00004467649304611F0A7FC214611F0A4FCE3
:1022D00019F8018F0646B8F1000F41F0FF83059B06
:1022E0000C2B05D1304611F073FE6D4B6A009852ED
:1022F000069B6C4C002B41F024846B49304611F056
:102300008BFC6A49064611F025FE002841F0168430
:102310006749304611F03CFE00B1654E0135032D92
:1023200044F80A607FF46DAF624B00221A70624B72
:102330001878002840F00C85604E33681C0340F18B
:1023400007855F4C2378033B052B1CD84A4B5D4D1A
:1023500093F8593533B1012B08D106F0CFFEC0F107
:102360007F0003E0286A03689B6898476B6A95F8CA
:1023700028201344B3F5807FA8BF4FF480738342B5
:10238000D4BF6B6268622378023B092B00F2908411
:10239000DFE813F00A00140046008E048E045F008C
:1023A000A200400461047104464B00225A62DA62C2
:1023B000454A12681A63032300F079BC424B414D31
:1023C0001A682B6B6433934280F07284402010F0C3
:1023D00057F8002840F06C842F46DFF8F0904FF05B
:1023E0004008EB6A19F8030060B110F023F97B6A2A
:1023F000B8F1010803F1FF337B62FB6A03F10103CB
:10240000FB62EED1EA6A31492E4B8A5C002A40F029
:102410004F84DA624FF0FF321A63042300F047BCA6
:102420002B4A5021A2F10C03019325230292009321
:102430004920A2F10A03163A0DF0E8FD002840F009
:102440003784204B4FF0FF32D8621A63072300F025
:102450002EBC052300931F4B002102910191A3F193
:10246000080253200DF0D2FD002840F02184154BC6
:10247000D862082300F01BBC303B0020F43500205C
:10248000C835002008140020B01F00200000C842FA
:10249000D7A368410000FA43F42600200000484317
:1024A000EC160020A41F00203333834000F0FFC54A
:1024B00000F0FF45460E00200414002054170020B1
:1024C0007A270020800A002084170020F892010853
:1024D0006E9301081C95010840200FF0D1FF0028E1
:1024E00040F0E683A34DEB6A492B01F23C83DFE821
:1024F00013F04A004D00520056005900600065007C
:102500006A006E0072007E0089008C0097009B00BC
:10251000A000A500B600C700D800E900FA000B0132
:102520001C012D0189019301A101AF01BD01CB0166
:10253000D901E701F50103020D021B0225022F025A
:10254000390243024D02570261026B0275027F029B
:10255000890293029D02A702B102BB02C502CA0210
:10256000CF02D402D902DE02E502EE02F902FE0237
:1025700003035B03600365036A036F03740379035A
:102580007E03830388037C497C483DE37C4B7D4A82
:102590007D497E4833E07E4A7E497F4894E27F4908
:1025A0007F4831E37F4B804893F8582593F85715BF
:1025B0008AE27C4B7D48B3F8CC1025E3794B7C480C
:1025C000B3F8CE1020E37B4B7B4819691CE37B4BAF
:1025D0007B48198918E36B6BD90404D5714B794892
:1025E00093F8161210E3634B0B22DA620EE36D4987
:1025F000754891F8193291F81B2291F81A1210F0CF
:10260000F4F803E3298F7148FEE233681A0540F1BC
:10261000FD82644B6E48B3F91E22B3F8201253E2D8
:10262000644B6C485969EFE25E4B6B4893F8DA11E2
:10263000EAE25C4B694893F8EA11E5E259486C22FA
:1026400090F8AC3402FB03F1431893F818240C23E0
:1026500003FB0213034493F81A146148D4E251486F
:102660006C2290F8AC3402FB03F1431893F8182461
:102670000C2303FB0213034493F81C145948C3E2D0
:1026800048486C2290F8AC3402FB03F1431893F8ED
:1026900018240C2303FB0213034493F81B14524821
:1026A000B2E240486C2290F8AC3402FB03F14318CC
:1026B00093F818240C2303FB0213034493F8231408
:1026C0004A48A1E237486C2290F8AC3402FB03F18F
:1026D000431893F818240C2303FB0213034493F8C4
:1026E0001D14434890E22F486C2290F8AC3402FB52
:1026F00003F1431893F818240C2303FB021303443B
:1027000093F81E143B487FE226486C2290F8AC34C4
:1027100002FB03F1431893F818240C2303FB021364
:10272000034493F8221434486EE21E486C2290F859
:10273000AC3402FB03F1431893F818240C2303FB79
:1027400002130344B3F824142C485DE215486C23AB
:1027500090F8AC144B43C21892F818240C2101FBDA
:102760000233C11891F8213491F82024244891F8BB
:102770001F1444E7800A0020ADB30108B9B3010873
:10278000CAB3010897B20108CFB30108D5B3010855
:102790008EB2010882B20108FDB301089640002004
:1027A00011B40108303B00201FB4010830B4010807
:1027B0003FB401080C2D00204EB40108002D00206C
:1027C0005EB4010868B4010875B401088EB401084C
:1027D00099B40108ACB40108B8B40108CBB401083D
:1027E000E0B40108EAB40108F4B4010801B5010835
:1027F0000EB5010818B5010823B5010830B5010868
:1028000042B50108BF4B6C2193F8AC24BE4801FBD4
:10281000023393F8D413F7E1BA4A6C2192F8AC343E
:10282000BA4801FB032191F8E93391F8DF2391F8CD
:10283000D513E4E6B34A6C2192F8AC34B44801FBFA
:10284000032191F8EA3391F8E02391F8D613D6E604
:10285000AC4A6C2192F8AC34AE4801FB032191F8EC
:10286000EB3391F8E12391F8D713C8E6A54A6C2120
:1028700092F8AC34A84801FB032191F8EC3391F8AD
:10288000E22391F8D813BAE69E4A6C2192F8AC3450
:10289000A24801FB032191F8ED3391F8E32391F86D
:1028A000D913ACE6974A6C2192F8AC349C4801FBF2
:1028B000032191F8EE3391F8E42391F8DA139EE6C0
:1028C000904A6C2192F8AC34964801FB032191F8B0
:1028D000EF3391F8E52391F8DB1390E6894A6C21F8
:1028E00092F8AC34904801FB032191F8F03391F851
:1028F000E62391F8DC1382E6824B6C2193F8AC243A
:102900008A4801FB023393F8DD137DE17D4A6C2197
:1029100092F8AC34864801FB032191F8F23391F828
:10292000E82391F8DE136AE6764B6C2193F8AC2429
:10293000804801FB023393F8F31365E1714B6C217E
:1029400093F8AC247C4801FB0233B3F8F4135BE149
:102950006C4B6C2193F8AC24784801FB0233B3F83C
:10296000F61351E1674B6C2193F8AC24744801FBDA
:102970000233B3F8F81347E1624B6C2193F8AC24AF
:10298000704801FB0233B3F8FA133DE15D4B6C2153
:1029900093F8AC246C4801FB023393F8FC1333E149
:1029A000584B6C2193F8AC24684801FB0233B3F810
:1029B000FE1329E1534B6C2193F8AC24644801FBCE
:1029C0000233B3F800141FE14E4B6C2193F8AC2492
:1029D000604801FB0233B3F8021415E1494B6C2146
:1029E00093F8AC245C4801FB023393F806140BE126
:1029F000444B6C2193F8AC24584801FB023393F804
:102A0000071401E13F4B6C2193F8AC24544801FBBF
:102A1000023393F80814F7E03A4B6C2193F8AC2496
:102A2000504801FB023393F80914EDE0354B6C215B
:102A300093F8AC244C4801FB023393F80A14E3E00A
:102A4000304B6C2193F8AC24484801FB023393F8D7
:102A50000B14D9E02B4B6C2193F8AC24444801FBB8
:102A60000233B3F80C14CFE0264B6C2193F8AC245E
:102A7000404801FB0233B3F80E14C5E0214B3E4839
:102A800093F82612C0E01F4B3C4893F82712BBE096
:102A90001C4B3B48B3F8D811B6E01A4B394893F8B1
:102AA000DB11B1E0174B384893F8DC11ACE0154B63
:102AB0003648B3F8E221B3F8DE1105E0114B344893
:102AC000B3F8E421B3F8E0110FF08FFE9EE00D4B58
:102AD0003049D3F8F80111F09FF811F079FA014666
:102AE0002D4891E0074B2D4893F8D5118CE0054B0C
:102AF0002B4893F8EE1187E0024B2A4893F8ED112A
:102B000082E000BF303B002051B5010862B50108EA
:102B100073B5010885B5010895B50108A5B501088B
:102B2000B5B50108C6B50108D7B50108E9B5010872
:102B3000D9B50108F3B5010808B6010818B60108AF
:102B400026B6010838B601084EB601085DB6010880
:102B500079B601088FB601089EB60108B5B601081E
:102B6000CEB60108E2B60108F7B601080DB70108B4
:102B700024B7010839B701084FB701084BB701085E
:102B80005BB7010867B7010879B701088CB701087E
:102B9000A0B701080000C842B8B70108C6B70108CD
:102BA000D6B70108E7B70108984B994893F88D12FA
:102BB0002AE0964B974893F84E1225E0934B96489F
:102BC00093F84F1220E0914B9448B3F852121BE057
:102BD0008E4B934893F8401216E08C4B914893F833
:102BE000E31011E0894B904893F8E2100CE0874B1A
:102BF0008E48B3F8DE1007E0844B8D4893F8EB1154
:102C000002E0824B8B4899680FF0EFFDEB6A0133CD
:102C1000EB624DE0884B1B689B0119D5874DAB8F4C
:102C2000B3B9874BD5F8408045201F680FF002FDEF
:102C30000E200FF0FFFC40460FF0B7FD38460FF0B6
:102C4000B4FD4FF480536B870A2323700CF04EFFC2
:102C50000DF0BAF92CE0794B93F84420002AF5D016
:102C6000754A12689701F1D493F84530002BEDD1E5
:102C700009232370ECE7734B704D1A682B6BC83334
:102C8000934204D2614B93F859757FB904E00FF079
:102C90003DFC0028F6D10BE0286A09F005FA95F80A
:102CA00046302F62022B01D10EF078F801232370F9
:102CB0000FF016FC50B101232370604B93F84520B0
:102CC000002A45D0002283F8452041E04F4B93F87D
:102CD0005A25002A3CD032680026D50432464CBF23
:102CE000B3F8DA10B3F8D010574D35F912000132AD
:102CF000884218BF46F001060C2AF6D1514A4F4DC2
:102D0000126826B102F59C520832AA6402E0A96C4E
:102D1000914213D92278012A1AD195F84520BAB9DF
:102D200093F859352BB105F0E7FF012385F84530BD
:102D30000EE080200EF02AF850B9F4E72378012B3A
:102D400006D095F845301BB105F0A8FF85F8456021
:102D50003E4B1B78072B05D10DF0E0FD049BC01AFC
:102D60003B4B5880354B00221A703A4C13A86368CD
:102D70009847A146002800F06A81374DBDF94C30D4
:102D8000364F2B60BDF94E3029466B60BDF950308F
:102D90002846AB60324B1A7805F03AFC3B88002B92
:102DA00000F0D1802F4B304E1B6806F10C041B78CD
:102DB0004FF0000804933B88D9F8142005934FF492
:102DC0007A73B3FBF2F3C3EB431203EB8203DB0032
:102DD000059A9BB29A4202BF00233360236155F8E3
:102DE000280033684FEA880B0344336010F0C0FEBC
:102DF000226902F1010ABAF1010FC4F810A035D11D
:102E0000002360602060A36053E000BF303B0020DF
:102E1000F7B7010810B8010824B8010841B8010843
:102E20005EB8010873B8010888B801089DB80108A8
:102E3000AFB80108BDB80108F4350020800A0020B1
:102E4000380D002084170020AC130020EA16002063
:102E5000EC1600200C2D0020C01F00209016002032
:102E60004C2D002054180020CC0A00202268089025
:102E70001146079210F0C6FD0690504610F078FEFD
:102E80000146069810F07CFF079A114610F0BCFD31
:102E9000089B014682466060184610F0B3FD069913
:102EA00010F0BAFEA16810F0AFFDC4F800A0E06019
:102EB000A0609A4A002345F80B304BF80230059B7E
:102EC000012B2ED12069012807DD013810F050FEBA
:102ED0000146E06810F054FF00E0002013F0E8FF26
:102EE000049B82464BB1184610F042FE514611F049
:102EF00031F810B105F079FB25E0D9F814204FF432
:102F00007A73B3FBF2F3C3EB431203EB8203DB00F0
:102F100032689BB202EB530292FBF3F37F4A42F812
:102F20000B3008F10108B8F1030F06F1040604F1B3
:102F300014047FF440AF3888012801D109F046FA23
:102F40003B88013B3B807548002355F8232050F80F
:102F50002310734C521A45F823200133032BF4D16C
:102F6000704B1A781F46002A64D0DFF8FC816E4E41
:102F7000C246DFF8F891043C002598F80030032B96
:102F800004BF636829F81530684B1B78012B0AD100
:102F9000606810F0EDFD664B01461C2000FB05301B
:102FA0000FF0ACFE1CE083B9606810F0E1FD97F80B
:102FB00000B001465F4B60484FF00C0E1B685A464C
:102FC0000EFB05000FF086FF0AE0606810F0D0FDF0
:102FD0005A4B01464FF4F87000FB05300FF038FEF5
:102FE00070609AF80030082B04D1706813F0A0FCD0
:102FF00029F81500524B1B883BB1524B1C207168BD
:1030000000FB05300FF07AFE70604F4B1B883BB120
:103010004E4B1C20716800FB05300FF06FFE706096
:1030200056F8040F13F084FC0135032D44F8040F07
:10303000A3D10CE0206810F09BFD454D286060682E
:1030400010F096FD6860A06810F092FDA860414AFB
:1030500092F8C430144623B1013B82F8C43000F02A
:103060008DBD3D4B93F8DC211E4622B193F8EA3129
:10307000013BDBB200E0012384F8C4300DF04EFCCC
:10308000364B374DD3F80080364BB6F82A12A3F1F1
:10309000460207462868C047334B1A781E46072A5F
:1030A00004D10DF03BFC314BC01B98800DF036FC79
:1030B00096F800B00490BBF1010F0AD12C49D4F866
:1030C000C8302A4A0968C31A93805B1AD380C4F8AF
:1030D000C800284B2A681B68E3B192F83340D4B18A
:1030E000254A126894074DD5244A1278012A49D9F5
:1030F000DB7823495A430988D31A994215B203DB76
:1031000091420B46A8BF13462D031BB295FBF3F566
:1031100001243AE01C46254637E000BF140B00208E
:10312000C01F0020552D0020CC260020582D002047
:103130005C2D0020B02D0020200B0020B42D00209D
:10314000562D00208C33002084330020E4330020EF
:10315000D0260020800A0020303B0020A40200205E
:1031600008140020683D0020EA160020EC1600201C
:10317000D01F0020C4160020541700206403002034
:103180001417002001244FF48055AA4BDB780D93CF
:103190002CB1BDF954306B431B13ADF854304FF0D4
:1031A00000094E464F46A44BDFF8BCA293F80080BE
:1031B000A24BB3F902200892B3F90020B3F904300E
:1031C00009929F4A059312689E4B0692474545D245
:1031D00008980A9310F0CCFCDAF8081010F01CFDE7
:1031E0000790099810F0C4FCDAF8041010F014FDF0
:1031F000079A0146104610F007FC069B079093F9CA
:103200000000059B4042584310F0B2FCDAF80C1065
:1032100010F002FD079A0146104610F0F5FB10F081
:10322000D7FE15AA00B20A9B0CB16843001322F81E
:10323000170015AA32F91720B24203DC9145A8BF46
:10324000914600E01646BBF1050F03D1042F98BF4D
:1032500023F8172001370AF1100AB7E77A4BC9EBB8
:103260000606196836B211F480530793774A40D0A6
:10327000774B78481B78B2F9062013F0040F08BF8B
:103280000368754F02BF1C8A734BA3F88C41036817
:1032900072481B8A0068724CC588C5EB030E7245E4
:1032A00008DCB0F900302068A7F88C21B0F90040A4
:1032B00015440AE02B449A4209DB2368B0F9024026
:1032C000B3F90230A7F88C21551B2DB219E0B7F9DC
:1032D0008C319E45B3BF2368B0F900302268B0F945
:1032E0000240A7BFB2F900401D46B3F9023025469F
:1032F00007E05B4BB2F906501B68B3F90040B3F925
:1033000002309BB2A4B2C4EB030A0FFA8AFA564504
:10331000514A18DD4FEA0A3999FBF6F60020C2F847
:103320009061804508D915AB33F9107077433F138E
:1033300023F810700130F4E702239AFBF3F31C44E6
:1033400024B20A9408E04FF0020996FBF9F69B1BA1
:1033500034441BB224B20A93B2F98C31404A0C9324
:1033600017683B4A3B4B16783E4A1B68B2F9062069
:1033700006933A4B0B924FEA480206F004060E926F
:103380001B6801F01002DFF8E490F6B24FF0000B7A
:103390000F920E9A93456BD015AA3BF8022028464F
:1033A0001092119310F0E4FB2F4B53F83B1010F0E8
:1033B00033FC10F00DFEA0422146109A119B03DB56
:1033C0000A998142A8BF01460A440D9912B229F810
:1033D000022F09B1B9880EE0079959B10699D8882A
:1033E000098A091A0C98884202DC3988188803E097
:1033F000598800E0398878888A4203DB9042014688
:10340000A8BF11460F9AA9F800107AB176B1079AB1
:1034100062B9109308F0B4FF109B38B9069A0B9963
:10342000528A9142BCBFBA88A9F800200BF1020B66
:10343000AFE700BF88170020CF1F002034260020F0
:1034400068180020EC16002054170020B01F002040
:10345000F83500206C180020800A0020403A002037
:10346000443A0020581700204C0B002082390020DD
:10347000398949B39F4B4FF47A721B68B2FBF3F35F
:10348000B1FBF3F3012B05D942F210729342A8BFAE
:10349000134600E002231BB29A4515DD964C3A888C
:1034A00034F9185095484FEA480147189542B7F942
:1034B000947103DBFA18AA42A8BF2A4612B201444B
:1034C00024F81820A1F8942116B98B4B8C4A06E0F9
:1034D0008A4B93F8AC21192A00F2468107E0B045E7
:1034E000F6D932F8161023F816100136F7E7012343
:1034F00003FA02F2834B1340002B00F03581824B1C
:103500001B88D80508D5814B1A88ADF86C205A88DD
:103510009B88ADF86E2014E0BDF82430ADF86C3017
:10352000BDF82030ADF86E30BDF81430ADF8703015
:10353000079B43B1069B0B9A1B8A9A4203DA059BB1
:103540005B42ADF8703072484FF47A72B0F90230D5
:103550004FF4616103F5E163534393FBF1F3A3F58A
:10356000FA73ADF88430B0F9003003F5E1635A43E3
:1035700092FBF1F2604BA2F5FA721B88ADF886203F
:10358000A3F2DC53ADF87230624B634A1B681188BA
:103590001B8AC91AADF874105188C91AADF8761093
:1035A0009188C91AADF87810D188C91AADF87A1087
:1035B0001189C91AADF87C105189C91AADF87E106D
:1035C0009189D289C91AD31AADF882300023ADF897
:1035D00080101946514A22F813100133082BFAD1F2
:1035E0004F4B50491B68504D0593504BDFF82CA1B1
:1035F0001B684FF0640E06934D4B4FF001091B788A
:10360000C3EBC303CB180993099B8B4200F0928054
:103610000B782BB11533059A09FA03F3134064D0E4
:10362000069B11F806CC0E2202FB0C38B8F90230CA
:10363000B8F9002011F9010C9A1A11F9023C92B262
:10364000534393FBFEF34FEA520B11F8057CCBEB8F
:103650000303089011F8030C1BB207937E0028B9EE
:1036600022A8064436F81C0C288019E022AB1E4420
:10367000B5F9004036F91C6CB44208DA20448442A3
:1036800003DC86423446A8BF04462C8008E007DDF0
:10369000201AB04203DB8442A8BF044626462E808F
:1036A000D8F80A0009FA07F73842B5F9006011F9AD
:1036B000040C079B00FB06F090FBFEF00CBF0124FE
:1036C0004FF0FF34984209DB089B5A4392FBFEF20D
:1036D000CBEB02031BB28342A8BF03463AF81CB0EF
:1036E00004FB03B32AF81C3000E02B8002350731BD
:1036F0008AE700BFD01F002084390020800A002004
:10370000AC13002032413003F0350020B01F002000
:10371000B81F00206C18002058170020FC0900205A
:10372000F43500204F3A00202E0C0020C03A002033
:10373000483A0020A94BAA4ED3F8008000254FF04C
:103740000E09642709FB058393F9064036F9023F09
:10375000E8B25C4394FBF7F434800CF013FF0135BE
:103760002044082D3080EDD19E4EDFF87082336802
:1037700013F0200F30D000200CF004FF9A4C0546C7
:10378000208001200CF0FEFE984B60801B6819061B
:1037900022D5974B974A1B681B78012B22D1D8F86A
:1037A00000E0B2F902109EF9063032275B424B432B
:1037B00093FBF7F3B2F9002099B29EF9143053430A
:1037C0006FF0310293FBF2F293FBF7F30A44AD1A68
:1037D0000B44258018446080D8F80030804A03F1FB
:1037E00070041AE0D8F80070B2F9023097F90610A8
:1037F0004FF0320E4B4393FBFEF3E918218097F90B
:103800001430B2F9001001FB03F292FBFEF21044F7
:10381000E1E70E339C4211800CD032F9020FB3F96C
:103820000010B3F902508842F3DB85422946A8BF55
:103830000146EEE7704F714D3B6893F90430ABB928
:1038400095F8AC8108F1FF33182B00F29280DFE885
:1038500003F05090906B9090906490909090907640
:1038600090909090906B839090765000A9460023A2
:10387000DFF874B1A5F8CE31B5F9CE41072CDFDC05
:1038800099F8D021DFF88CA172B93A68508810F00D
:103890006BF95B4A01461C20126800FB04A00FF084
:1038A000E5FA012289F8D0213BF9140010F060F903
:1038B00001461C2000FB04A00FF020FA13F038F89A
:1038C000D8F800100E2202FB041200B22BF81400EC
:1038D000B2F90010B2F90220884203DB8242A8BF8D
:1038E00002461146404B23F814100134A5F8CE418E
:1038F000C2E73B685B781BB13B4B0020598908E06D
:10390000404B1B7803F0040303F0FF01002BF3D1BD
:10391000084609F019FC01242CE0334C0020E18812
:1039200009F012FC218905E02F4C0020218909F0C3
:103930000BFC6189012009F007FC02241AE02A4FE0
:103940000224A01E37F81410C0B2013409F0FCFBA9
:10395000082CF6D106240DE0234F0324E01E37F88F
:103960001410C0B2013409F0EFFB072CF6D1042487
:1039700000E0002433689A0602D4B8F1050F0BD199
:10398000194F2046398809F0DFFB601C7988C0B2E6
:1039900009F0DAFB0234E4B23368DB0205D495F8AF
:1039A000B43273B10CF044FD0BE0174F0026A019A0
:1039B00037F8021FC0B209F0C7FB0D2EEFD0013659
:1039C000F5E7124B1B78072B05D10CF0A7FF049BE2
:1039D000C01A0F4BD88001232B70CFE0C03A0020D3
:1039E000FA09002054170020FC090020F4350020BB
:1039F00064180020B81F002068180020800A0020EA
:103A0000D01F0020F83500205E170020EA160020A5
:103A1000EC160020540C00205A4B1B885E063EF525
:103A2000E5AB237E584E8342DFF8808111D030769B
:103A300010F09EF8554910F0EFF8554907460FF081
:103A4000E3FF0FF097F8C8F8000038460FF092F83F
:103A5000F061504EB6F9000010F08AF80746B6F94A
:103A6000040010F085F8D8F80080814641463846B9
:103A700010F0D2F8E46982462146484610F0CCF8AE
:103A8000014650460FF0BEFF10F0A2FADFF820A169
:103A9000B0F5FA7FA8BF4FF4FA705045B8BF504652
:103AA00049463080404610F0B7F8214680463846F7
:103AB00010F0B2F8014640460FF0A6FF10F088FA69
:103AC000B0F5FA7FA8BF4FF4FA705045B8BF504622
:103AD000B080FEF78BBBA346FEF7C7BB0021204694
:103AE00010F056FA08B904F10044404610F040F8CE
:103AF000294910F045F9214610F08EF801464FF0A3
:103B00007E500FF07FFF2549044610F023FA40B99C
:103B10004FF07E51204610F03BFA18B14FF07E5422
:103B200000E01E4C21464FF07E5010F029F901466E
:103B3000304610F071F80646FEF7D1BB184EFEF77E
:103B4000EDBB1849304610F005FA48B91649304621
:103B500010F01EFA00283EF4E1AB134EFEF7DEBB78
:103B6000104EFEF7DBBB0EF0D1FC00283FF4A0A8FE
:103B70004FF480536B870A23FFF799B823B0BDE851
:103B8000F08F00BFF0350020800A002035FA8E3C0F
:103B9000DB0FC93FB01F00200000C8420AD7233CFA
:103BA00000F0FFC500C0F9C400C0F94400000020C7
:103BB0000CFEFFFF9A4B2DE9F04F196887B001F515
:103BC0009C4220325A60974A9A46157815B9964F0A
:103BD000964E15E0964B1B68994240F2F780013DE6
:103BE0001570F3E0072C96BF3B682146195D91489C
:103BF00033689847032C09D90AEB44042081013526
:103C000004F0BEFEECB28442ECD31FE03A6804F14B
:103C1000100302EB83039988DA880028ECD04FF474
:103C20007A73401A5843531A90FBF3F040F6C903D5
:103C300000F57A70984205DC40F2EE239842B8BF56
:103C4000184601E040F6CA0080B2D5E742F2010B07
:103C5000794B7A4F1B6803EA0B0B3B680093BBF16F
:103C6000000F06D09AF82D308AF82C30744B5A7811
:103C70001A709AF82C501DB1714B1D7885F0010512
:103C8000704E0F238AF82E30002406F1460904F006
:103C900077FE844260DA4FEA44081DB16A4B33F87C
:103CA000140000E02846604BA1001A68938B834201
:103CB000664B02D8D28B82421BD259F80110009871
:103CC000574A814202D933F8080017E0E0B2029364
:103CD000019204F06DFE032C029B0FDC019A01217E
:103CE00001FA04FE92F82E1021EA0E0182F82E103D
:103CF00004E0009A02F5967249F80120BBF1000F2A
:103D000025D09AF8C0100322B1FBF2F202EB420276
:103D10008A1AD2B208EB040E72440AEB42021086F1
:103D20009AF8C1202AB9022911D93D4A012182F805
:103D3000C11036F8020C3288718802440A4412B26B
:103D4000032092FBF0F0424980B221F8082023F8CA
:103D50000800013406369AE79AF82E300F2B0CBF74
:103D6000012300238AF8DA303A4B0DD13A4A12681F
:103D7000520109D43A68D9689A60521AC82A20D9DF
:103D8000012283F821201CE02D4A0121517011707D
:103D90003A689968DA605B68521A9A4284BF2D4B80
:103DA00000222A4D88BF83F82120002404F0E8FD7A
:103DB000844206DAE0B204F0FBFD25F81400013479
:103DC000F4E79AF8C03001338AF8C0301A4B1A6809
:103DD000994612F4805F05D01F4B1B68DF0701D4A2
:103DE0000FF00EF9104B0E4A1D68DAF80040287BE0
:103DF000B0B3164AAB7B013832F910001BB1C0F5E5
:103E00003B60083000B2A0F57A70B0F57A7FA8BFA9
:103E10004FF47A7020EAE0700FF0AAFE0F4955E0E7
:103E2000380D00208017002050170020900300203C
:103E30007C170020B0410020541700208417002078
:103E4000040000206A0D0020400D002058170020BB
:103E5000FA0D002088170020F435002000007A4475
:103E6000D9F800301E043AD5D2F8DC30E31A002B22
:103E700035DB04F59C432033C2F8DC30AD4BD979F7
:103E8000AD4B33F811108BB2697B93FBF1F192F8D3
:103E9000E030013303F00F0382F8E030134483F87D
:103EA000E1100346E132815C01300B4410281BB263
:103EB000F9D193FBF0F000B2002803DB6428A8BF1F
:103EC000642000E000200FF053FE9C490FF058FFE3
:103ED0009B490FF0A1FE10F0A1F89A4B1880D9F879
:103EE0000030D80540F1F580974BDFF860B29C4276
:103EF00005D99BF8022012B901228BF802209BF809
:103F00000220002A00F0E580904A914B914992F8F6
:103F1000214008681A78012C02F0040600F0806342
:103F2000F6B20093019107D012F0080F0CBF4FF0CA
:103F300000084FF0020801E04FF00008864D874F5F
:103F40009BF82020052A00F2BE80DFE802F003463D
:103F5000597988A7A6B3BAF8F210DAF8F40008F095
:103F6000CFF9012807D139682A68C988642000FB85
:103F70000122CBF81020009B53B13A6812793AB174
:103F80000CF0B4FB03228BF820204FF47A7234E05B
:103F9000012C00F098802968DBF810006B4A8842F9
:103FA0000AD202920CF0A2FB029A032182F820109E
:103FB00040F6B831D161C3E7012182F82010BFE794
:103FC000009B4FF4806013B109F03EFB01E009F063
:103FD0002BFB0022CBF8102075E0012C52D03A6860
:103FE000127A012A02D00CF081FBA9E70CF07EFBCB
:103FF00003228BF8202040F6B832CBF81C209FE734
:10400000012C04BF05228BF8202066B1DAF8F420D9
:104010004FF00308B2F91010514A1180518091807D
:1040200039684988D1802A68DBF81410914201D39D
:10403000002E45D147F23052CBF81C20032222E05B
:10404000434B1A7842F002021A700EF0D9FF2A6828
:10405000DBF81C100A44CBF81820042213E0012CD2
:1040600014D12A68DBF8181091422CD23D4B1A78F3
:104070001AB9019B1A68D10725D4354B1A7822F05A
:1040800002021A7005228BF8202059E7324ADBF829
:104090001C1012680A44CBF8182014E039682A680A
:1040A000C988642000FB01224FF48060CBF8102007
:1040B00000228BF820208BF8032009F0B5FA3FE7A7
:1040C000012C3FF43DAFB8F1000F02D0404608F09C
:1040D0007DF9254DB5F8DC1005F50E7008F010F9E6
:1040E000044608F04DF9AB46204D70B1184B1B78D3
:1040F0005A070AD51E4BB3F90620BBF852329A4232
:104100003EDB01238AF8F8303FE000238AF8F830DC
:10411000002C3AD1174B00221A605A609A60164B55
:1041200016491B68002093F83430086048608860A6
:104130005BBB2BE0CC160020E01600200000C8423C
:1041400000C07F44D4430020404B4C00881700201F
:10415000F8350020F435002084170020F43A0020C0
:1041600058170020A0020020303B002048260020E5
:10417000B01F0020DC26002008140020D41F0020DF
:104180001CB99AF8F830002BC4D001232B70A44B33
:104190001B785B0737D5D9F80030DF0633D5A14A45
:1041A0001278D6062FD4DD042DD408F0E9F850BBE0
:1041B0009D4B1B7883B19BF88F329CB96BB19B4BA5
:1041C0001A68DAF8FC309B1A002B06DA0EF018FF9A
:1041D000974B83F8004116E06CB9102008F0F6F810
:1041E00001230EE03BB1914A4FF47A71126801FB52
:1041F0000323CAF8FC309AF8003123B108F0CEF856
:1042000000238AF80031002213469BF88E12BBF877
:104210004A52BBF84C62874F37F912009B08A842FC
:10422000C4BF63F07F03DBB20132B042B8BF43F0DA
:104230004003042AF0D19AF801217D489A4205D121
:1042400090F80221F92A04D8013200E0002280F817
:104250000221754E8AF801313378754A764D23BBB9
:104260002868C00709D582F80331F4B96C4B1B7874
:10427000DA071AD50EF060FE17E0694B1B785B0772
:1042800013D592F82C3083B16C4BDB786BB992F874
:1042900003310133DBB2032B82F8033105D911B1AD
:1042A0000EF0AEFE01E0002CFAD09AF80231604C1C
:1042B000142B56D1337893B194F801315F2B0ED182
:1042C000574B1B7803F0040303F0FF0713B10EF004
:1042D00097FE04E00B2008F079F884F80271504B47
:1042E0001B7803F0040303F0FF02D3BB9AF80141EB
:1042F0004F4B572C02D104F078F932E0D9F8001076
:104300004F0717D55A2C15D193F8041129B183F80A
:104310000421012283F8052123E093F8062182F08D
:10432000010283F806210AB10C2000E00D2008F0FC
:104330004DF816E05D2C00F0EE835B2C00F0ED8371
:104340005E2C01D10320E9E3562C01D109F06EFA6D
:104350003378002B00F0E7836F2C40F0E4830EF0FD
:10436000EBFDD9F80030580738D59AF80631304AB5
:104370009BB12B4B1B7859070FD52E4BB3F9061069
:10438000BBF84A32994208DD2B6813F0010302BFE3
:104390003221A2F80A1182F806312B68DA030DD512
:1043A0009AF80C21224B2AB993F8042112B932222F
:1043B000A3F80A2101238AF80C310FE09AF804319E
:1043C0001B4A5BB1164B1B7803F0040303F0FF019B
:1043D00023B9012382F8041182F80531184C002317
:1043E0002B6004F150060127214614F8010C07F058
:1043F00061FF30B114F8023C07FA03F22B68134353
:104400002B600434B442EFD10E4B1D78F5B10A4C49
:104410000D4D236813F0020F40F0CC81C3E100BFC3
:10442000F8350020A1130020A002002084170020EE
:10443000380D002058170020F43500208817002080
:10444000DF3F002004140020F0350020B44CB54EAE
:1044500004F15A074FF00C08214614F8010C07F03C
:1044600029FFE0B12179A37808FB01FEAE4A013BA8
:1044700003EB430306EB0E001344426894F803C0B9
:1044800093420CD04360012303FA01F19AF80D31F5
:1044900006F80EC023EA010185608AF80D11063482
:1044A000A742D9D1A14BA24F1C68A24BA24D1B68B9
:1044B00001939AF82C300293002300933A68002A63
:1044C00000F069811678002E00F065817B68019903
:1044D000CB1A002B0CDB01F5FA7300997B600123EA
:1044E00003FA01F19AF80D3123EA01038AF80D313C
:1044F000029B002B00F04F8117F8043C51780433E5
:10450000DBB2002940F0FD808C4931F91310BBF873
:10451000483203F1C800814202DD92F8028015E0C2
:10452000C83B994203DA9178C1F100080EE0009A85
:10453000012303FA02F29AF80D3123EA02038AF802
:104540000D31019B03F5FA737B6024E1009B9AF81F
:104550000D211A41D30700F11E81B8F1000FCCBF25
:104560000220012007F072FF721E132A00F20A8156
:10457000DFE812F014001E00280038005000570039
:1045800071008B00A400AF00BC0008013800460099
:10459000570071008B00660080009900217801208F
:1045A0004144FA29A8BFFA2121EAE17121709AE079
:1045B000A178022041446429A8BF642121EAE17165
:1045C000A17090E026795E4B4644642EA8BF642615
:1045D00026EAE67619682046267107F015FE314670
:1045E000032080E0A1790D2041446429A8BF642103
:1045F00021EAE171A17107F0A3FE0D2E00F0C28047
:1046000061790E2041446429A8BF642121EAE17147
:10461000617168E0E1790520414481F30801E171AD
:1046200061E02A680F2091784144C829A8BFC821B9
:1046300021EAE171917007F083FE0F2E00F0A28055
:104640002A68122051784144C829A8BFC82121EA0C
:10465000E171517047E02A681020117B4144C8295C
:10466000A8BFC82121EAE171117307F069FE102E7D
:1046700000F088802A681320D17A4144C829A8BF55
:10468000C82121EAE171D1722DE02A681120917DC3
:104690004144C829A8BFC82121EAE171917507F0FA
:1046A0004FFE112E6ED02A681420517D4144C82936
:1046B000A8BFC82121EAE171517514E02A680920D8
:1046C000D1784144C829A8BFC82121EAE171D1703D
:1046D00009E02A680A20517B4144C829A8BFC821A3
:1046E00021EAE171517307F02BFE4BE02A680B20A1
:1046F000D17D4144C829A8BFC82121EAE171D17503
:10470000F1E701293ED10D4931F91300B0F5617F80
:1047100018DB40F633038342A8BF034614E000BF12
:104720002E4000201C1800203C950108C8350020B0
:10473000201800208417002050180020581700204F
:104740004C1800204FF461730C2E1BD190784FF45D
:10475000966292FBF0F0A3F5617393FBF0F3824A4B
:10476000DBB212789A420DD01846039308F084FF0A
:10477000039B3046194607F0E3FD039B581CC0B26B
:1047800007F064FE009A012303FA02F29AF80D3151
:1047900013438AF80D31009B0C370133042B00932F
:1047A0007FF48CAE33E6D9F80030DE050FD56F4BC1
:1047B000DB7863B16E4B1B68980708D52B8813F024
:1047C000010609D1012008F03FFF334605E0012032
:1047D00008F02AFF012300E00023226851070AD5D0
:1047E0004BB1012008F020FF2B889A0706D4022045
:1047F00008F02AFF02E0022008F016FF298811F0D5
:1048000003011ABF01210846012008F0D1FE2368E8
:104810004FF480701B0502D508F016FF01E008F088
:1048200003FF9BF80530082B01D00E2B02D140204E
:1048300008F0FAFED9F800305F0519D59BF8D032A0
:1048400023B94C4B1B7813F0040F02E0236813F4D8
:10485000002F09D03C200CF099FA48B10AF088F9F1
:104860003C200CF05DFAF8E709F0EBFF0CF096FA4B
:1048700001238AF80E31404BB3F906203F4B1B68E9
:1048800059898A420CDB187AB2F5FA6FBFBF531A06
:104890004343C1F5FA6093FBF0F0C0F1640300E01C
:1048A000642300939BF9D431BBF848525B429BB21E
:1048B0009BF826E29BF827C2184640F2E63B304EB2
:1048C0000021304B9DF800404FEA4108CC542A4B60
:1048D00033F911707B1B03F2F3145C45284C0FD89D
:1048E000002BB8BF5B4202290ED0734502DDCEEB30
:1048F000030300E00023AF4226F808300DDB11E08F
:1049000002294FF4FA73F2D19C45B4BFCCEB0303F8
:1049100000234343AF42B38007DA36F808305B42E6
:1049200026F8083001310329CBD1D9F8006016F4FC
:1049300080560DD0B2F57A7F05DBB2F5FA6FA8BFCD
:104940004FF4FA6201E04FF47A72A2F57A7226E02F
:104950000D4BB3F84A128A4218DBB2F5FA6FA8BFC2
:104960004FF4FA6213E000BFCF3700208817002011
:10497000502D0020F835002058170020C8350020A1
:10498000B01F0020CC1F0020303B00200A46521AE6
:104990004FF47A735343C1F5FA62B3FBF2F2642326
:1049A00092FBF3F07F4F00F1010E37F9101037F949
:1049B0001E706FF0630E0EFB00227F1A7A4392FB8B
:1049C000F3F30B449BB2E380B6B1774A1268D6008A
:1049D00012D5764AD2787AB9A3F57A731BB24FF41E
:1049E0007A721B0393FBF2F3C5F5FA6212B25343DA
:1049F00005EB23356E4BDD806E4B1B885D0642D583
:104A00006D4B0A20B3F9043093FBF0F0BAF8103183
:104A1000C01A00B20FF0ACF868490FF0FDF8684911
:104A200005460EF0F1FF0EF0A5F8074628460EF0F9
:104A3000A1F80546B4F902000FF09AF80646B4F959
:104A400000000FF095F8394680460FF0E5F8314642
:104A5000814628460FF0E0F8014648460EF0D2FFA6
:104A60000FF0B6FA3946208030460FF0D5F84146AF
:104A7000064628460FF0D0F8014630460EF0C4FF37
:104A80000FF0A6FA60804F4B1A78540706D5012123
:104A9000002007B0BDE8F04F08F08ABD424B4A49FC
:104AA0001B6813F0010F474B02D091F8120110B1AF
:104AB00042F001021A70454AB1F808111278100745
:104AC0005EBF1A7822F001021A70414A19B14149B9
:104AD0000968890706D44049098819B93F48008800
:104AE000642806D9022111701A7822F001021A7086
:104AF00005E01B78DB0756BF0223117013700BF023
:104B00000DFF374B1B68C01A002848DB07B0BDE813
:104B1000F04F03F0D5BF012000E002200138C0B201
:104B200008F072FE1DE4972C04D14FF4C873AAF864
:104B3000083116E4A72C05D1244A137843F0040366
:104B400013700EE40023BB2C059301D1022303E074
:104B5000B72C04D14FF6FE73ADF816300AE0BE2C28
:104B600001D1022304E0BD2C7FF4FBAB4FF6FE73B2
:104B7000ADF81430BBF8F221BDF814301344ABF893
:104B8000F231BBF8F421BDF816301344ABF8F43120
:104B900008F04CFE00238AF80231FFF7E2BB07B0B1
:104BA000BDE8F08F62270020F43500208817002030
:104BB000B01F0020F0350020B81F002035FA8E3CD1
:104BC000DB0FC93FF8350020380D0020A11300206D
:104BD000AC170020502D0020901600202814002033
:104BE000B0170020426A806A131A58425841704731
:104BF0004171704743799B070AD5436A8269D15452
:104C0000436A01690133B3FBF1F201FB12334362E2
:104C10007047427902F0020202F0FF0342B10369D9
:104C2000426A806A013BDBB2101A23EA0000704737
:104C300018467047437913F001031FBFC369026A26
:104C40009A1AC3681ABF03F1FF3302EA0300184639
:104C50007047437910B513F0010301460DD0FFF7FB
:104C6000E9FF58B10B6A4A69CC68D05C0133B3FBE9
:104C7000F4F204FB12330B6210BD184610BD90F81D
:104C8000433230B583B990F8423290F84112012492
:104C90008B4209D2B0F8482204FA03F52A430133C3
:104CA000A0F84822DBB2F3E730BD0C2343439B4A14
:104CB000F0B5D3589A499D8A9A4AADB2ECB214F035
:104CC000010F4FEA001031D01C8824F40064240442
:104CD000240C1C801C88A4B244F480641C80002432
:104CE00014700C18A579ADB1557815B9E478FF2C7E
:104CF00010D1012454700C182479022C01BF1C8897
:104D0000A4B244F400641C800C18A47844F001049C
:104D10001C82EDE00D18AC7804F0FE041C82EC78E7
:104D2000FF2C00F0E580FF241470E1E0A6073BD5DE
:104D3000BFF35F8F0C182579EDB2012D13D1A47943
:104D40008CB154787CB11C8824F480642404240C35
:104D50001C80BFF35F8F1C8B1C889570A4B244F439
:104D600000741C801BE01C8BBFF35F8F0C1825792F
:104D7000022D0AD1A47944B1547834B11C8824F4AA
:104D800080642404240C1C80ACE00C182579032DCD
:104D900005D1A4791CB15478002C40F0A3809C88E4
:104DA000A4B244F48064A2E067075CD501240D1826
:104DB0009470AC79002C3CD05478002C39D02C79EC
:104DC00092F90060022C1C881FD924F4806424040A
:104DD000240C1C80B3F810E0EF685FFA8EFE07F831
:104DE00006E0F4B21E88B6B246F400761E80EE6885
:104DF000A51C15701D8A013464B2EDB235559C882E
:104E0000A4B244F480649C8029E0A4B244F4007409
:104E10001C80B3F810E0EF685FFA8EFE07F806E03A
:104E2000F4B2EF681D8A661C76B2EDB2BD5503344C
:104E30000BE0547814B90C18647944B11C88A4B2FE
:104E400044F400741C8014780134147007E01C884A
:104E50000125A4B244F480741C80324C65701C8817
:104E6000E605FCD444E004F0400404F0FF0604B37B
:104E700092F900C01C8A01EB000EDEF80C70E4B25F
:104E80005FFA8CF607F80C40751C6DB29EF8047042
:104E9000EC1CA742157005D19C8824F4806424047E
:104EA000240C9C800C182479A54221D1023616705E
:104EB0001EE02D061CD592F900506C1C0AD00F186C
:104EC000BE686C1C755D64B21D823D791470A5428C
:104ED0000ED107E00C18E57816701D82A5790DB982
:104EE00024792CB99C8824F480642404240C9C80AC
:104EF0000C18247992F90060621C9642094D0CD17D
:104F000000226A70AA782AB19A8822F440721204A8
:104F1000120C9A80084400234370F0BDB4B101081C
:104F2000FC3A00204C0E00201FB50123ADF80830DC
:104F3000ADF80410002301A9ADF80A30ADF80C302B
:104F4000ADF8062003F014FA05B05DF804FB38B59F
:104F5000A0F515746379DB0744D5A57994F8403240
:104F600005F00105F3B1A16B0868838DC3F34E030F
:104F7000838494F8443223B1B4F84A320133A4F85C
:104F80004A326A004979FFF7CFFF012384F84332A0
:104F9000002384F8413284F8423284F84032A4F885
:104FA000483238BD94F843322046012B04BF94F8B0
:104FB000413284F84232FFF762FE94F84322A36B39
:104FC0002AB9012284F8432205FA02F205E0002200
:104FD000954284F8432208BF022259791868BDE837
:104FE0003840A1E738BD8379406BDB0744BFB1FA95
:104FF00081F1490909B108F0CCBA08F0C5BA10B579
:10500000A0F5147494F84422BAB9A36A616A99426B
:1050100028D0591CA069A162C35C2069DBB25B0087
:1050200043F400738142A4F846324FF00A0384F837
:10503000453228BFA262012312E094F945327BB1C8
:10504000B4F8461220464B08A4F8463201F001019C
:10505000FFF7C9FF94F84532013B84F8453201E07F
:1050600084F8443294F84032002B4ED194F8413207
:105070000133DBB2092B84F8413203D12046BDE86D
:105080001040FCE50A2B40D194F843322BB9B4F818
:10509000483243F00103A4F848326379D9071CD59C
:1050A000B4F84802820501D4C30705D4B4F84C32E1
:1050B0000133A4F84C3210E0E36AC0F347000BB1AF
:1050C00098470AE0E3696269D054E369E168013313
:1050D000B3FBF1F201FB1233E361012284F84022B9
:1050E00094F843220023012A84F841320DD1A27999
:1050F00084F84332A36B12F0010F0CBF022200228E
:1051000059791868BDE810400EE710BD026D70B502
:1051100015880446ADB2A90613D5036B8BB9C36AD3
:105120001BB1908880B298470BE0E1699288406992
:105130004E1CD2B2E6614254E169E268914228BF56
:10514000E3612B0613D5636AA26A9A42236D0AD0E3
:10515000511CA069A162825C9A802369994206D39E
:105160000023A36270BDDA6822F08002DA6070BDAD
:105170002DE9F04F99464FF416734343554D85B0D2
:105180002F1D0646924607EB030810B92B44524ADE
:1051900003E0012805D1514A2B44DA630C32C3F8ED
:1051A00040214FF4167373434D4AEC18626003229A
:1051B0006272FA1803F5A0733C323B44D4F840B154
:1051C0002163A2614FF480710022E361012384F81E
:1051D00044322161626222626161E262A26284F809
:1051E000482284F84522A4F84E22A4F85022C4F89C
:1051F0000CA084F80A9084F852629BF80400039390
:1052000007F0BEFFA0639BF8040007F0B9FF06F1AA
:10521000010B05225FFA8BFB8271C27180F808B026
:105220001221029207F0D2FFE16B0879019107F099
:10523000A7FF01996063087907F0A2FF029A80F83E
:1052400008B082710622C2714A2107F0BFFF039B9A
:1052500040461946FFF7C7FE32200BF09DFB214B5D
:10526000D4F840411B681A46B2FBFAF1B1F5803F11
:1052700003D3012AF8D95208F6E71B4A2046B3FBAC
:10528000F2F289B2D2B20BF01FFB4FF416735E43F9
:10529000164B354406F5147637440022C5F85432CF
:1052A000394620460BF062FAEC6B19F0010F0CBF87
:1052B0000222002261792068FFF736FE0C4B20465F
:1052C000C5F858320022391D0BF050FA404605B09F
:1052D000BDE8F08F4C0E00202C900108449001088E
:1052E000789501086803002040420F00FF4F000836
:1052F0004F4F000883790A46C16A90F84E0237E79B
:105300002DE9F043B1F800E000234FF00F0C012627
:105310004EFA03F2D20729D58D78DF0815F0100F69
:1053200018BF91F8039003F0070805F00F024FEA49
:10533000880850F8274018BF42EA09020CFA08F919
:1053400024EA090402FA08F22243282D40F8272013
:1053500005D1C26806FA03F422EA040205E0482DEA
:1053600004D1C26806FA03F42243C2600133102B51
:10537000CED1BDE8F0830348D0F898300BB190301F
:1053800018477047A80200200348D0F880300BB1BE
:1053900078301847704700BFA80200200248836E8B
:1053A0000BB1603018477047A80200200248036D17
:1053B0000BB1483018477047A80200200248836BA1
:1053C0000BB1303018477047A80200200248036A2A
:1053D0000BB1183018477047A802002002488368B4
:1053E00003B11847704700BFA80200202DE9F0471D
:1053F0000C244443824E86B006EB0409804699F89B
:10540000040007F0BDFE054699F8050007F0B8FE58
:10541000074608F101030921DBB20D22E971AA71E7
:105420002B7282710A22C271037299F806000BF086
:105430001FFB34592846A3884FF0080923F4407312
:105440001B041B0CA38008F0A4F8384608F0A1F850
:105450001621284607F0BAFE1621384607F0B6FE98
:105460004FF0640A284608F0ABF840B9BAF1000FD3
:1054700005D00A200BF06EFA0AF1FF3AF2E728464F
:1054800008F082F80A200BF065FA284608F081F847
:105490000A200BF05FFAB9F10109E3D1384608F0B0
:1054A00073F80A200BF056FA284608F06DF80A2027
:1054B0000BF050FA284608F06CF80A200BF04AFA74
:1054C000384608F066F828461F2107F07FFE384668
:1054D0001F2107F07BFE4B4B4B499C4203F5DE330B
:1054E0001A6901A80BBF42F4001242F480021A614B
:1054F0001A610BBF1A691A6922F4001222F48002A1
:105500001A61A38823F440731B041B0CA3800C2393
:1055100003FB08663D4BF779002F0CBF1F460F4673
:1055200023889BB243F001032380A58807F024FC65
:10553000039A374825F03F05B2FBF0F02D042D0CFF
:105540000543ADB2A580218807EB470321F0010197
:105550000904090C21804FF49671B2FBF3F301FBAF
:1055600000F24FF47A7192FBF1F29BB2002B08BF6C
:105570000123013292B243F400432284A38323889F
:1055800000259BB243F001032380238801A823F464
:10559000816323F002031B041B0C43F4806323800C
:1055A0004FF480432381238823F080031B041B0CCA
:1055B0002380737A01248DF804308DF805508DF81E
:1055C00006508DF807400BF071FA337A9DF80720EA
:1055D0008DF804308DF805508DF806501AB101A8E9
:1055E0000BF064FA08E05A090A4903F01F0304FAB1
:1055F00003F3203241F8223006B0BDE8F08700BF47
:10560000B4B101080054004000350C00801A0600B7
:1056100040420F0000E100E00C23434337B5254A28
:105620000546D458A38A9BB20193019B13F4706F73
:105630001FBF214A03010121D154019B13F4E06FE4
:105640002BD0238BA38823F480631B041B0CA38023
:10565000019B9A0521D423889B051ED42388D80555
:1056600010D52388D905FCD423889BB243F400735A
:10567000238023889A05FCD46B1C0ED02846FFF7A4
:10568000B5FE0AE023889BB243F400732380A3880D
:1056900023F440731B041B0CA380A38A23F47063C0
:1056A0001B041B0CA382044B03EB051500236B703A
:1056B00003B030BDB4B10108FC3A00200120FFF76F
:1056C000F4BA0120A8E70020FFF7EFBA0020A3E713
:1056D0002DE9F04F87B009F0B4F8884B1D78002D04
:1056E00040F0CE85864E3368590540F1C985854C1A
:1056F000854F2378002B00F07E813A686368D31AC7
:105700007C2B40F27881814BDFF820B2B3F8DC804B
:10571000237A62600133237205F12400DFF8E491FB
:10572000C0B209F071F809F10C0353F825000EF02E
:105730001FFA8246BBF808000EF01AFA01465046DE
:105740000EF01EFB72490EF067FA0EF041FC0135B7
:1057500000B209F047F8032DDED1302009F054F8EB
:10576000002009F03FF809F047F899F8085015F0C3
:10577000030524D141F28833D9F804209A420BD989
:10578000102009F041F8284609F02CF8212009F0F2
:105790003BF8284609F026F8142009F035F85D4B4F
:1057A000B3F904000A2390FBF3F009F01BF81C2066
:1057B00009F02AF8002009F015F809F01DF8237AFD
:1057C0005A0740F0F080022009F01EF84D4B4FF0D0
:1057D0000509B3F918000A2390FBF3F009F002F869
:1057E0004D4B0320B3F9065009F00EF895FBF9F57F
:1057F0004A4BADB21B785B070BD54146484806F0D3
:105800007FFD20B9336813F0100F18BF002528B2B0
:1058100005E0444B1B68D889B0FBF9F000B208F0F2
:10582000E1FF33689D0740F18C80DFF80491DFF8D9
:10583000F88099F80010B8F80020642303FB0212E6
:105840004B00B2FBF3F3658B06202D01ADB245EAA8
:105850000325ADB2C3F303231D4308F0D5FF28B2DF
:1058600008F0C0FF638B99F8001001339BB293FBE3
:10587000F1F201FB1233E2696383937B012B05D1C3
:10588000392008F0C1FFB8F9000021E0B8F8005055
:105890006E236B43152593FBF5F5D37BADB20BB1AE
:1058A00095FBF1F53A204FF0640908F0ADFFB5FB28
:1058B000F9F809FB18550FFA88F008F093FF3B2020
:1058C00008F0A2FFA8B2451D0A2095FBF0F000B237
:1058D00008F088FF282008F097FF236A0A2093FB2E
:1058E000F0F000B208F07EFF042008F08DFF0D4BB1
:1058F0001B68DB89F3B102F045FF1FE004140020B0
:10590000541700200013002084170020303B002093
:1059100000007A44B81F0020B01F0020F835002096
:10592000683D0020C416002014170020002D002020
:1059300064030020BE4B186880F3100000B208F02A
:1059400051FF05A9BB4808F023FF132008F05CFFB6
:10595000BDF9140008F046FF1B2008F055FFBDF903
:10596000160008F03FFF232008F04EFF4E2008F0FD
:1059700039FF05A9AF4808F00BFF122008F044FFDB
:10598000BDF9140008F02EFF1A2008F03DFFBDF904
:10599000160008F027FF222008F036FF452008F007
:1059A00021FF08F029FF237A282B24D1A24B0022C3
:1059B00017201A723D6808F027FF4EF66020B5FBED
:1059C000F0F04FF03C08B0FBF8F308FB13000002C6
:1059D00000B208F007FF182008F016FF4FF47A70A5
:1059E000B5FBF0F5B5FBF8F008FB105000B208F07D
:1059F000F9FE08F001FF94F824308F4D002B00F0E1
:105A0000B7800AF08BFFAB6A8C4AC31A9342804678
:105A10003CD9002385F82E3085F83030884B1B8820
:105A2000DAB21B0A85F84A2085F84B3085F8402009
:105A300085F84130AA6D3B689A1AEB6D197C4FF4DA
:105A40007A734B439A420DD37E4B1B68AB657E4BFA
:105A50001B78013B012B9FBF102385F82E300223BA
:105A600085F83030724B226A1B680A2192FBF1F2F2
:105A700093FBF1F384F8482084F84C3012121B1287
:105A800084F8492084F84D30C4F8288094F860A048
:105A9000694DBAF1000F0FD1A86E05F087FDC0B2B5
:105AA000012809D90228DFF8A49100F0A38308F0A7
:105AB00061FE012389F80030E56E5F4B002D57D061
:105AC00093F860203AB140F6B7315A6FC2EB080242
:105AD0008A4215D84CE0012283F860209A6F127830
:105AE000022A05D8986E0221043008F02DFE03E04A
:105AF0000221986E05F051FD002384F87C3035E0DA
:105B000093F870209AB9DA6683F860209A6F127859
:105B1000022A05D8986E0121043008F015FE03E032
:105B20000121986E05F039FD08F024FE1EE0013ACF
:105B3000D2B283F8702093F87C1093F87D0032B9CC
:105B40004A1C013083F87C2083F87D000BE02A4654
:105B500012F801EB01300EEB0105714683F87C5021
:105B6000DA6683F87D00986E05F023FDC4F8748032
:105B70003B6894F87E8001932F4BB8F1000F00F042
:105B80006281D3F88020002A00F05D8193F88420A0
:105B9000013A012A00F257819A464FF0020B012583
:105BA000254AD4F88000029205F000FD029AD8B18F
:105BB000DAF8800005F0F7FC9AF8851081467E2916
:105BC0003A680ED11B288AF884B00AD1DAF880002E
:105BD000029205F0EBFC20B9029A8AF88C50CAF8C0
:105BE000882084F88590DBE7D2F888103B685B1A40
:105BF00041F658318B4203D9032382F8843022E1E5
:105C00000546DFF84CA094F88CE094F88D30002223
:105C1000BEF1000F00F0148139680198091A0129BA
:105C200018D90AB184F88D30002384F88C300AE149
:105C3000C816002080969800001300203F0D030036
:105C40001417002084170020CE3700200800002001
:105C5000A09501083AF8130010B903464FF4036009
:105C60000133B0F5826FDBB2424600F0C28056D8F5
:105C7000B0F5007F00F0868008D8B0F5807F00F096
:105C80009C80B0F5887F00F09880C1E7B0F5047F74
:105C900062D0B0F5806FBBD184F88D3094F8943029
:105CA000914A0133DBB2032B88BF012382F8943081
:105CB00042F2107394F8941059438C4B1B78D80718
:105CC00048BF01319A0748BF02315807884B48BF87
:105CD00004311B88DA0748BF0A31980748BF1431DE
:105CE0001A0648BF2831D80548BF28315A0748BF8F
:105CF0006431180748BFC8319A0548BF01F5C8711B
:105D0000980648BF01F57A71DA0648BF01F5FA61D5
:105D1000580648BF01F57A614FF480608AE0B0F51B
:105D2000E26F5FD00AD8B0F5C06F3DD0B0F5E06F3C
:105D30007FF46EAF84F88D30E16856E0B0F5046F03
:105D400044D0B0F5116F67D0B0F5E46F7FF460AF69
:105D500084F88D30616948E084F88D3033689807A5
:105D60007FF551AF604BD3F89030DA7B614B1B88E5
:105D70001AB1614A117893FBF1F30A2159434FF4A8
:105D800004702AE084F88D303368DFF85CB11905BF
:105D90007FF539AFDBF820100A2391FBF3F108F00F
:105DA0009FFC8BF88C502EE784F88D3033681A05F1
:105DB0007FF529AF514B19683CE084F88D30504B8A
:105DC0001B685B077FF51FAF002133E084F88D303F
:105DD0004C4B0A21B3F90430594308F081FC84F894
:105DE0008C5010E7216984F88D302C2391FBF3F15E
:105DF000F3E784F88D30424B1B6813F0200B7FF4DF
:105E000002AF33681A067FF5FEAE594608F068FC0B
:105E1000354B83F88CB0F6E684F88D3033689B07F9
:105E20007FF5F1AE334B344A19880A234B4311787E
:105E300093FBF1F108F054FC2B4B83F88C50E2E615
:105E40000AB184F88D3094F89530274D002B00F07E
:105E5000AF80D5F89830002B00F0AA803E68D5F8C6
:105E60009C30F31A632B40F2A380DFF89880412026
:105E700008F01DFCB8F902000A2790FBF7F080B289
:105E800008F00CFCB8F9000090FBF7F080B208F0C5
:105E900005FCB8F9040090FBF7F080B208F0FEFBB7
:105EA00008F0E2FB95F8A05015F001055BD1104B0E
:105EB0001B88D90529D4DA060DD49F060DD45806BF
:105EC0000DD419070DD4DA071ED413F0020F14BF36
:105ED0000325012519E00D2517E0092515E0042506
:105EE00013E0082511E000BF00130020F835002062
:105EF000F03500201417002064030020C81600208D
:105F0000502D0020B81F00200225BE4B1F78BE4B2D
:105F1000C7F38007DB7813B147F00207FFB25320C5
:105F200008F0C5FBB94B188800EB800000EB80003F
:105F3000800080B208F0B2FB002008F0AFFBB44B49
:105F40001888FE23584340F2FF3390FBF3F0C0B2B1
:105F500008F094FB002008F091FB47EA850008F068
:105F60008DFB08F081FB94F8A030A3B94F2008F016
:105F70009EFB0AF0C3FF0AF0C1FF0AF0BFFF012039
:105F800008F07CFBA34B93F8A10000F0010008F09F
:105F900075FB08F069FB94F8A0300A210133DBB2ED
:105FA000B3FBF1F201FB1233C4F89C6084F8A0301B
:105FB000994D95F80080AA46B8F1020F40F0028191
:105FC0000AF0ACFC954B1F6840F6B833C71B9F42E4
:105FD00007D900232B70B4F8A2300133A4F8A23003
:105FE0004EE18F4E33793A2B40F00081B178304644
:105FF00002F04EFD002840F0F980844B894D1B884B
:10600000D4F8A4B0EB61236AE863EB62864BEF66D9
:106010001B685846EB64B4F8A230DFF8F891EB65E2
:1060200005F003F80746002840F0CC80414658466A
:1060300005F0B3FA042385F87430F378019399F8E6
:10604000A830642B47D199F8A930072B08BF89F8ED
:10605000A97094F8A98005EB0816716808460391A9
:106060000DF022F8B3685FFA80F9184602930DF03C
:106070001BF85FFA80FB6D4E09EB0B020832F271E0
:1060800028F00F02B27208F00F0272730BEBC90214
:10609000B27303994A4606F10F0010F065FA029BAD
:1060A00006EB090019465A460F3010F05DFA16F853
:1060B000079F08F101084946304602F0CDFC06F87A
:1060C000090001980AF0FAFE002384F8A83084F849
:1060D000A980564E5FE095F8756000223307534B58
:1060E00008BF013603F10D019B468E4608BFF6B28C
:1060F000072EDFF83CC128BF01269A72330105EB59
:10610000030898F81020481C43EA0209624481F809
:106110000090D8F80C8092F82210012900F10102B9
:1061200007D9013902F8018C10464FEA1828C9B284
:10613000F3E72B445B7C013628F06008F6B248EAAE
:106140000308082E114680F800800CD0354B3848E3
:1061500003EB06131B7C034493F82200CEEB0203EF
:106160000344132BCADDCEEB020808F106085FFAE0
:1061700088F8DFF8C09048F040038BF807304146BC
:10618000484602F069FC09F80800019885F8756036
:106190000AF094FE9DE7B37807F10108FFB2BB4215
:1061A00006D9F15DD4F8A40005F003FA4746F2E7FA
:1061B00094F8A8300322013385F8742084F8A830BD
:1061C0008AF80020174D95F87430032B58D1D4F875
:1061D000A40005F0E5F9002852D00E4B0121D3F8B8
:1061E000A40005F0DAF9022385F8743000238AF858
:1061F000003045E099F80030F3B1C5F8648089F8C3
:1062000000A059E4F835002088170020141700205A
:10621000D443002000130020271600206016002021
:106220005416002008000020C816002084410020D9
:10623000A09501088B4100206B6EC3EB0803B3F5FA
:106240007A6FFFF439AC0123A86E89F8003005F0AD
:10625000AAF98146A86E05F0A6F919F07F0F7FF420
:106260002BAC8E287FF428AC95F86030002B7FF49F
:1062700023AC05F12C03EB662D2385F870301BE46D
:1062800007B0BDE8F08F00BF08B5037833B9084BFD
:1062900008481978BDE8084008F002BD10F034F94C
:1062A000022804D8C0B207F0E7F90348EDE708BDBB
:1062B000CF370020D2B901083FB2010810B50C4C0D
:1062C00003783BB90A4B0B4893F8AC14BDE8104077
:1062D00008F0E6BC10F018F9012807D884F8AC04DF
:1062E00007F0EAF904F058F80348E9E710BD00BFE9
:1062F000303B0020D6B901083FB2010870B50378E1
:10630000F3B9254B1C680134132C05D823490C2202
:1063100002FB0412956825BB2546204A0C21013555
:10632000132D01DD002500E003D801FB0520866860
:106330004EBBA542F3D11A48BDE8704008F0B0BC8E
:1063400010F0E2F81328044605D8144A0C2303FB86
:1063500000239D682DB92146BDE87040114808F022
:106360009FBC0D4B1C6006F019F82A4621460E48CA
:1063700008F096FC25460C235D43084B585DBDE8AC
:10638000704006F023B81D6006F008F83246294632
:10639000054808F085FCEEE780000020D095010854
:1063A000E3B90108F9B9010811BA010873B5037816
:1063B00013B903F089FB37E0002401AA1B4910F050
:1063C0003CF92646254680B12CB1012C06D110F0AF
:1063D0009BF8064602E010F097F8054601AA13491B
:1063E0000020013410F029F9EDE70B2D03D9014607
:1063F0000B220F480BE0022C0FD1A6F57A73B3F5F0
:106400007A7F07D90B484FF4FA624FF47A7103F0A0
:1064100002FB09E0084B23F81560074B294633F9C6
:106420001520064808F03CFC02B070BD70C10108A0
:1064300028BA010844C90108AC1300202EBA01088B
:10644000064B93F8662503F26653002A044A06BFFA
:10645000012113460021034A08F0D4BF303B00203D
:106460003DBA01083FBA010838B505460CF01CFEDC
:10647000044690B1112200210A4812F007FD22467D
:106480000949284612F070FD38B1102C22462946E1
:1064900028BF1022034812F07CFDBDE838400120DF
:1064A000CEE700BF964000203DBA010808B50B4872
:1064B00008F0F6FB02F074FF094B00221A765A76B8
:1064C000DA6102F02BFE18B964200AF065FAF8E7E9
:1064D0000448BDE8084008F0E3BB00BF49BA010822
:1064E000AC13002056BA010838B5054D441E14F807
:1064F000011F19B1286807F089F8F8E738BD00BF17
:10650000243600202DE9F04105461D4FDFF8748048
:1065100028460CF0C9FD064658B91A4B1A485A7954
:106520001A4BBDE8F04103EB8203D3F8EC1008F0FE
:10653000B7BB02461649284612F0EDFC08B100240C
:106540000CE01448FFF7D0FF134C54F8041F19B1A6
:10655000124808F0A5FBF8E7114803E057F82410AB
:1065600019B91048BDE8F041BEE73246284612F09E
:10657000D2FC01340028F1D188F805400A4DC7E764
:10658000C0960108303B00205EBA0108D095010892
:106590006ABA01086FBA0108BC96010882BA0108FC
:1065A000F3BB010886BA01083FB2010838B5064DB1
:1065B000002455F83400FFF797FF01340348FFF734
:1065C00093FF242CF5D138BD2C970108F3BB0108AB
:1065D000F0B585B005460CF067FD082827D16E1E82
:1065E000EF1D16F8014F0FF0A3FF2044437803F08E
:1065F0000303022B08BF203CB7423470F1D12C4674
:1066000005F1080714F8016B1648314612F075FCC5
:1066100020B13146204612F070FC10B103F054FA5C
:106620001DE0A742EED11049284602F08FF90F482D
:10663000FFF75AFF0E4C0B4800231A1992F8382224
:1066400004A90A44195C0133082B02F80C1CF4D18C
:10665000002301A907488DF80C3008F021FB05B094
:10666000F0BD00BF85A00108683D002095BA010873
:10667000303B002023BA01082DE9F74F82460CF089
:1066800013FD464D0446D5F85C75B8B9444808F08A
:1066900007FB444E012505FA04F33B4206D00C23C8
:1066A00003FB04634048996808F0FAFA0134122C9D
:1066B000F1D1CFB93D48FFF717FF15E002463C493D
:1066C000504612F028FCDFF8DC90064670B93948D5
:1066D000FFF70AFF344609EB0403996832480C348B
:1066E00008F0DEFAF02CF6D133481FE09AF80030BB
:1066F0004FF000082D2B03BF0AF1010A04F1FF340B
:106700004FF0010B4FF0000B0C2303FB089296682F
:10671000504622463146019312F0FDFB019B48B1E1
:1067200008F10108B8F1140FEFD1244803B0BDE817
:10673000F04FD9E6BBF1000F14D0B8F1120F01D120
:106740001F4B04E0B8F1130F04D1D5F86035C5F83C
:106750005C3505E0012202FA08F31F43C5F85C75B9
:10676000184812E0B8F1120F02D1C5F85CB50BE081
:10677000B8F1130F1DBF012303FA08F39F43C5F8B7
:10678000607518BFC5F85C750F48FFF7ADFE314660
:106790000E4803B0BDE8F04F08F082BA303B00204D
:1067A0009BBA0108D0950108ACBA0108A5BA010846
:1067B0006ABA0108B1BA0108F3BB010886BA010838
:1067C000FFFF0300BCBA0108C5BA010822BA0108DC
:1067D0002DE9F84F81460CF067FC324E0446D6F89E
:1067E000088098B93048FFF77FFE304D012655F8F4
:1067F000241049B106FA04F313EA080F02D02C481A
:1068000008F04EFA0134F2E72A4824E002462A4909
:10681000484612F080FB58B92848FFF765FE284C1F
:1068200054F8041F0029EFD0214808F039FAF7E79F
:1068300099F80030DFF874B02D2B03BF09F101097E
:1068400004F1FF344FF0010A4FF0000A00255BF815
:1068500025701FB91B48BDE8F84F45E6224639466A
:10686000484612F058FBD0B90120A840020601D5D5
:106870001548F0E78305FBD4BAF1000F03D006F00A
:10688000F3FE124803E040EA0800B0601048FFF74A
:106890002BFE3946BDE8F84F0E4808F001BA013525
:1068A000D5E700BF303B0020CDBA01084C98010865
:1068B00082BA0108F3BB01086ABA0108D7BA010815
:1068C0004898010886BA0108E3BA0108BCBA010871
:1068D000C5BA010822BA010810B504460A48FFF7F4
:1068E00003FE0A4B186806F085FE094B186A05F08E
:1068F000B3FB0AF03AF8074B074A14B107480849B6
:106900000860DA6010BD00BFF1BA0108243600202B
:10691000AC13002000ED00E00400FA05EFBEADDE90
:10692000F04F002038B50A4D0A48FFF7DDFD286812
:1069300006F060FE084B002483F824405C6583F871
:10694000584009F0D9FD2046FFF7C6FF2C6038BD3E
:1069500024360020FDBA0108AC13002008B5054814
:10696000FFF7C2FD04F0FEF806F0A6FEBDE8084001
:106970000020B1E729BB010808B50448FFF7B4FDC2
:1069800006F09AFEBDE808400020A5E73FBB0108DD
:1069900070B5044608460D460CF086FB29460246B3
:1069A000204612F0B8FA08B1002070BD0FF0C0FD0B
:1069B000064628460CF078FB235C33445B785B0783
:1069C000F2D10130204470BD2DE9F04F0E4691B058
:1069D00061490446FFF7DCFF0546B0B95F49204630
:1069E000FFF7D6FF054690B95D492046FFF7D0FF77
:1069F000054670B920465B49FFF7CAFF00280546E7
:106A000012BF08242546012404E0012402E00224E8
:106A100000E004240EB144F01004534803F0F0FEEB
:106A200052492846FFF7B4FF08B144F0200414F09F
:106A3000090F00F01E824E48FFF756FD002008F0B7
:106A40008DF904F01803182B02D14A48FFF74CFDCA
:106A50004948FFF749FD494D2046DFF80C81FFF713
:106A6000EFFC4748FFF740FD98F805306E79454F39
:106A7000C3EB060CDCF1000646EB0C0607EB8303C8
:106A80003146D3F8EC30404A204608F09BFC6B7945
:106A9000314607EB8303D3F8EC303B4A204608F03D
:106AA000B1FC0021E8680DF04BFA4FF00106CDF87B
:106AB0001080039700B90646344AF1B2204608F028
:106AC000A1FC2949204601F02FF83148FFF70CFDC1
:106AD0002549204600F076FC2E48FFF705FD95F984
:106AE000E6102D4AB1FA81F12046490908F08AFCE6
:106AF0001D49204600F046FA2848FFF7F5FC049BA4
:106B0000D5F80890D3F808A0DFF89880002658F848
:106B1000267017B969EA0A0B67E04FF0010B0BFA10
:106B200006FB6AEA090313EA0B0F14BF01210021D7
:106B30003B461B4A204608F045FC69EA0A0313EA73
:106B40000B0F174A3B4614BF01210021204608F0D5
:106B500059FC0136DBE700BF5FBB0108C2BE01087C
:106B600066BB01086CBB01088827002070BB0108C8
:106B70007DBB01088BBB0108C3BB0108303B002073
:106B8000CEBB0108D0950108DABB0108E5BB0108BE
:106B9000F6BB010802BC010812BC010821BC0108B7
:106BA0002FBC01084C9801084FF0010808FA07F8BB
:106BB0001AEA080F09D01BEA080F3346B74A14BF78
:106BC00001210021204608F0FDFB19EA080F0BD037
:106BD0006AEA090313EA080FB04A334614BF0121D9
:106BE0000021204608F00EFC0137AD4B53F827601A
:106BF000002ED9D1AB48FFF777FC049BD5F85C7524
:106C0000D3F85C35DFF8F4B27B40DB43DFF8F0A269
:106C100007934FF00109079A09FA06F31A4218BFC1
:106C2000C846039A08BF4FF000083B4006934FF058
:106C30000C0303FB06239B6814BF5A465246414689
:106C40002046059308F0BEFB069A059B002A14BF58
:106C500052465A46414620464E4408F0D3FB122E77
:106C6000D7D14F469048914EFFF73EFC0023EA18DB
:106C700092F83822995D10A8104400F8201C04985E
:106C80000DF1400E184490F8380286440EF8101C9E
:106C90002FB1C0EB020EDEF1000747EB0E07013308
:106CA000082B07F00107E2D10CAB814A39460026D8
:106CB00020468DF8286008F085FB08AB7C4A3946F1
:106CC000204608F09FFB7B48FFF70EFC7A492046E0
:106CD00002F080FD7948FFF707FC7749204600F075
:106CE00095FD7748FFF700FC7349204600F0F6FC5D
:106CF0007448FFF7F9FB7049204600F04DFC7248DC
:106D0000FFF7F2FB6C49204602F0E8FD6F48FFF701
:106D1000EBFB6949204602F0E5FC6D48FFF7E4FB18
:106D20006549204600F06AFE6A48FFF7DDFBDFF8A0
:106D3000C881DFF884A198F858129AF8583299421D
:106D400007D19AF8597298F85922D01B4742474107
:106D500000E00027022928D19AF859224FF019099A
:106D600009FB02F202F2EE220192039A3946134421
:106D700093F8DC32584A00932046334608F022FB51
:106D800098F85932039A09FB03F909F2EE230193AB
:106D900098F858323946134493F8DC324E4A00933F
:106DA0002046334608F02EFB17E0039A3946134479
:106DB00093F8DC32494A00932046334608F002FB40
:106DC00098F85832039A3946134493F8DC32434A10
:106DD00000932046334608F015FB0136122E08F1C9
:106DE00002080AF1020AA6D13D48FFF77DFB2146C1
:106DF000002005F097FE14F0080F3A4E2ED095F8BB
:106E0000AC740025E8B2214605F0D6FEF36D2146AC
:106E1000002093F8448005F0EFFE2146012005F0A4
:106E2000EBFE2146022005F0E7FE404606F024FC7A
:106E30002D48FFF759FB01352C48FFF725FA022DA5
:106E4000E0D1384606F0E0FC2948FFF74DFB274823
:106E5000FFF734FA2748FFF747FB0AE0214695F889
:106E6000AC0405F0A9FEF36D214693F8440005F04B
:106E7000C3FEA20705D5204B214693F8AC0405F0CC
:106E80009BFE630706D5174B2146DB6D93F8440044
:106E900005F0B2FE11B0BDE8F08F00BF3DBC0108A7
:106EA0004C9801084ABC010857BC010885A001089C
:106EB00061BC01086ABC01088827002077BC010872
:106EC00081BC01088DBC01089EBC0108A8BC01085A
:106ED000B7BC0108C5BC0108D2BC0108E4BC01086C
:106EE000F3BC0108AC13002000BD01083FB201084B
:106EF0002DBD010856BD0108303B002046BB0108EE
:106F000052BB010801215FE500215DE5027983683C
:106F100002F03002102A06D10A4A6C2192F8AC2401
:106F200001FB02330CE0202A0AD1064A92F8AC1485
:106F3000054A10780C2242436C2000FB01221344C6
:106F400018467047303B0020CF3700202DE9FF4125
:106F50000A480488856846888788D0F80C8002F043
:106F6000BDF88DE88001029033462A462146044848
:106F700007F096FE04B0BDE8F08100BF8400002059
:106F8000BBC001082DE9F04F82460D468FB0544E2C
:106F90000D91002796F8E43096F9E6800A9396F86A
:106FA000E53096F9E9B0099396F8E73095F8E520D1
:106FB000089396F9E83095F9E6100B9396F8EA30C5
:106FC00095F8E7000C9395F9E8E095F8E43095F929
:106FD000E9C095F8EA90B8F1000F07D1DFF8008119
:106FE0004048FFF781FA0024C34642E00A9C9C42D5
:106FF00012D1099C94420FD188450DD1089C84423E
:107000000AD10B9C744507D1E34505D10C9C4C4536
:1070100014BF0024012400E00024CDF814C0CDF8F2
:1070200010E003900291019200932F4A3B462146C3
:10703000CDF81890504608F0C5F90C9BCDF814B067
:1070400006930B9BCDF808800493089B264A039374
:10705000099B214601930A9B504600933B4601370A
:1070600008F0D0F9102F06F1070605F1070591D1B8
:10707000B4E70E2666430BEB0603002508930D9B31
:1070800001273344D3F85E2108EB0603D3F85E31C1
:10709000AF40534037EA030314BF4FF001094FF0EC
:1070A00000093A4206D000952346104A4946504608
:1070B00008F088F9089BD3F85E313B4206D0009572
:1070C00023460A4A4946504608F09CF901350E2DE0
:1070D000D5D10134082CCCD10FB0BDE8F08F00BF62
:1070E000303B0020F3BB010818C1010837C101087B
:1070F0002DE9F0410546A14C88B028460BF0D4FF9D
:10710000C1B221B9012008B0BDE8F0413AE705223B
:107110009B49284611F0FFFE064690B901467022B1
:10712000984811F0B3FE3046324697490E2404FBCE
:10713000001301300828A3F85E21A3F86021F6D1DE
:1071400018E104229149284611F0E5FE0646002880
:1071500049D1284602F024FC0746002800F00A81A5
:107160000BF0A2FF35465FFA80F854F825602EB97F
:10717000874808B0BDE8F04107F092BD424631466D
:10718000384611F0C8FE01350028EED17E4B1F466F
:1071900003F1700283F8EA0083F8E60083F8E50063
:1071A00083F8E40007339A42F4D17A4B002213F8B3
:1071B00035C003EBC505624510DA6868C2EBC2034F
:1071C00007EB030E034418680132CEF8E4009888F8
:1071D000AEF8E8009B798EF8EA30ECE731466E486D
:1071E00007F05EFDBFE007226C49284611F093FED0
:1071F0000646002872D12021284611F07EFE07465F
:107200000BF052FFC5B275BB654807F049FD2C462F
:1072100021466448013407F043FD0E2CF8D1624842
:1072200007F03EFD584F00242146604807F038FD26
:107230000E2606FB0476DFF888810025D6F85E214D
:107240000123AB401A425A495A4818BF41460135FA
:1072500007F026FD0E2DF1D15348013407F020FD33
:10726000082CE1D186E0544938460FF089F93546BB
:1072700000287AD0022D09D00FF046F94E494DF87A
:10728000250000200FF07CF90135F1E7009B072B6A
:1072900020D8019A0D2A1DD8017872290DD06E29A7
:1072A00018D139490E2000FB0313012101FA02F223
:1072B000D3F85E1121EA020209E033490E2000FBF7
:1072C00003130121D3F85E0101FA02F20243C3F86D
:1072D0005E2101E002F0F8FB304D0EE7284636490A
:1072E0000FF04EF9002558B1082D3ED00FF00CF9E3
:1072F00031494DF8250000200FF042F90135F2E741
:10730000082D32D1009B0F2B2FD8DDF804E0BEF101
:10731000070F2AD8029F0D2F27D8039E06F164027B
:10732000C82A22D8049DFF2D1FD8059964291CD88E
:10733000069A642A19D8914217DA0798032814D8B4
:10734000DFF844C0C3EBC303634483F8E4E083F88D
:10735000E57083F8E66083F8E75083F8E81083F877
:10736000E92083F8EA00154DC7E608B0BDE8F04112
:1073700002F0AABB08B0BDE8F08100BFC0960108CA
:107380004FC60108143C0020303B002056C10108C4
:1073900086BA01080C9901085BC101084EC10108B9
:1073A000AFBA010867C10108F3BB010890CF01081B
:1073B0000FCC01086CC1010870C101083FB201087F
:1073C00016C601082DE9F04180460D46314C88B0C3
:1073D0000027B4F95421B5F954319A4295F95D2149
:1073E0001DD1B4F95601B5F95611884217D1B4F937
:1073F0005801B5F95811884211D194F85B0195F8FC
:107400005C1188420BD194F95A0195F95A118842BE
:1074100005D194F95D11881A4142414100E00021F3
:107420000E46069295F95A214046059295F85C2140
:107430000E34049295F85B210E350392B5F94A217A
:107440000292B5F94821009301923B46124A07F097
:10745000B9FF94F94F31104A069394F94C313146F3
:10746000059394F84E314046049394F84D310393BC
:10747000B4F94A310293B4F948310193B4F9463171
:1074800000933B46013707F0BDFF082FA1D108B09C
:10749000BDE8F081303B002072C10108F0B50178F1
:1074A00085B0054609B1002417E0012005B0BDE80C
:1074B000F04087E72D2B14D1072C19DC28460FF05C
:1074C00023F804AB661C03EB440424F8100C15F8F5
:1074D000013F303B092BFAD934462B78002BE9D1F8
:1074E00004E0A3F13002092A07D8E5E7082C09D007
:1074F00005B0BDE8F04002F0E7BA202BF8D1013525
:107500002646E9E7BDF9002093B2072BF0D840F2F8
:10751000DC54BDF90200A0F2EE239BB2A342E7D8EF
:10752000BDF90410A1F2EE239BB2A342E0D8BDF94D
:107530000640A042DCDCA142DADB8842D8DCBDF99F
:107540000C6006F164039BB2C82BD1D8BDF90E5074
:10755000112DCDDCBDF908E01FFA8EF3B42BC7D88E
:10756000BDF90A70BBB2B42BC2D80A4B4FF00E0C57
:107570000CFB0233A3F85401A3F85611A3F85841A9
:1075800083F85BE183F85C7183F85A6183F85D519D
:1075900005B0F0BD303B00202DE9F74F07460E4601
:1075A000DFF8A4A000254FF0060808FB05F800242A
:1075B00004EB080303EB0A02334492F8A49393F814
:1075C000A433204AC3EB0901D1F1000B4BEB010BB3
:1075D000019300942B465946384607F0F3FE8DE898
:1075E00010022B46174A59463846013407F00AFF65
:1075F000062CDFF85490DBD10135062DD3D106F2ED
:10760000C735002409EB040393F8C88315F8013F3C
:107610003846C3EB080256425641019300940623B4
:10762000084A314607F0CEFE8DE810010623054AD0
:1076300031463846013407F0E5FE0B2CE2D103B0A9
:10764000BDE8F08F92C10108303B002030B50178D1
:1076500085B021B9012005B0BDE830409CE71C4948
:107660000EF08EFF002460B1032C0FD00EF04CFF03
:1076700001AB43F82400164900200EF081FF0134CD
:10768000F1E7032C02D1039B0F2B04D905B0BDE811
:10769000304002F019BA0199029AC8B2052809D8F7
:1076A000052AF3D80B4C062505FB0040104480F852
:1076B000A43307E00628E9D10A2AE7D80548104490
:1076C00080F8C833044805B0BDE8304007F0E8BA98
:1076D00070C10108303B002092C101082DE9FF472D
:1076E0001F4C804689460F46A2460026B7F8641311
:1076F000B4F864338B420BD106F1D8039B000AEB3C
:1077000003024B44DD88D288531B5D425D4100E09B
:10771000002597F86733134A029397F8663340467B
:107720008DE80A003346294607F04CFE94F867338B
:107730000C4A029394F8663329460193B4F86433F3
:10774000404600933346013607F05CFE102E04F1EC
:10775000040407F10407C9D104B0BDE8F08700BFF5
:10776000303B0020A8C101082DE9F0410178054611
:1077700019B9BDE8F0410120B0E70EF0C5FE0F28B1
:1077800004462CDC284602F00BF90646DFF8788028
:107790001B4F0025D83430460EF0B6FE38F81530B1
:1077A000984223DC012D07EB840303D0022D03D084
:1077B000988002E0987100E0D87130462C2111F0D9
:1077C0009CFB064610B10136012302E0AA1E53427B
:1077D0005341013553B1032DDDD1BDE8F0810F22B6
:1077E00000210848BDE8F04102F015B9044B03EB55
:1077F000840400236360BDE8F04102F065B900BF76
:10780000303B002028BA0108E49901082DE9F0472F
:1078100006468EB0DFF85CA001F53879002409AF88
:1078200059F8045F5AF8043F029503935B1B5D42CD
:10783000394603A80DF110085D4109F0EFFA414601
:1078400002A809F0EBFA2346094A2946CDF8008040
:10785000304607F0B7FD23460097054A29463046D3
:10786000013407F0CFFD202CDAD10EB0BDE8F0874F
:10787000BCC10108103E00202DE9F04F017887B00F
:10788000054619B90120FFF7C1FFA8E00EF03CFE44
:107890001F28044600F39E80284602F081F804F178
:1078A000B80300240746A046A246A146A3462546A3
:1078B00026460093009A4B4B03EB820254600193DF
:1078C000494BE2B2E05C0023BE4617F8011B49B108
:1078D000884207D00A2B05D00DF10C0E03F80E10CC
:1078E0000133F1E706AF3B4488424FF0000703F84D
:1078F0000C7C02D002F0E8F871E0013A0EF10107C9
:10790000032A0FD8DFE802F0130902450DF10B003E
:10791000DFF8E4C04FF0010E2DE00DF10B014FF048
:10792000010C15E003A80EF0EFFD064639E003A8B0
:107930000EF0EAFD054634E00133062B08D02B4853
:1079400013F800E09645F7D10CFA03F349EA03096E
:1079500011F8012F2AB30023F1E7254AD25C8A42AD
:107960000ED1002212F80CA08A450ED10EFA02F2B6
:1079700048EA02089A4610F8011F91B10023ECE78B
:107980000133072BE9D15346EBE70132062AE9D14F
:10799000F0E703A80EF0B8FD0F28D4BF83464FF0E0
:1079A000000B0134052C8BD19DE80C0005F00F0570
:1079B00045EA8B4545EA895949EA0A2A36014AEAE5
:1079C0000838F6B203EB820348EA06065E600AF066
:1079D000F3FC04E01F220021064802F01CF807B067
:1079E000BDE8F08F303B0020EA990108A0B1010802
:1079F000A6B1010828BA0108ADB101082DE9F3418B
:107A000080460F46174D0026B5F87C22B7F87C3229
:107A10009A42B7F87E2205D1B5F87E42A11A4C42AF
:107A20004C4100E00024019200930F4A3346214666
:107A3000404607F0C7FCB5F87E320B4A0193B5F813
:107A40007C322146009340463346013607F0DAFC8B
:107A5000042E05F1040507F10407D5D102B0BDE8F5
:107A6000F08100BF303B0020C8C10108F8B50178A3
:107A7000054619B9BDE8F8400120BFE7274911F0D4
:107A80000DFAA8B9264B4FF47A714FF4FA62A3F8B5
:107A90007C12A3F87E22A3F88012A3F88222A3F816
:107AA0008412A3F88622A3F88812A3F88A22F8BDCC
:107AB00028460EF029FD0328044627D8284601F061
:107AC0006FFF074620B10EF01FFD0125064600E0BE
:107AD0000546384601F064FF18B9BDE8F84001F0EA
:107AE000F3BF0EF011FD012DF7D140F2DC53A6F2E9
:107AF000EE229A42F1D8A0F2EE229A42EDD8084B3B
:107B00009E3403EB84039E80D880F8BD03220021BD
:107B10000448BDE8F84001F07EBF00BF4FC6010831
:107B2000303B00203BC401082DE9F04F0D4693B0D7
:107B30003C4E09900027D6F80C80002140460CF0FE
:107B4000FFF9044600286AD13369D5F80CB00593D3
:107B5000736959460693B36940460793AB69D5F8F4
:107B600010A0D5F8149008930CF0EAF988B15146AA
:107B700005980CF0E5F960B1494606980CF0E0F97B
:107B800038B1089907980CF0DBF9003018BF0120D4
:107B900000E0204600F0010410A9584603F094F8D4
:107BA0000EA98346504603F08FF80CA9824648463A
:107BB00003F08AF80AA98146089803F085F83B4645
:107BC000194A0390CDF80890CDF804A02146CDF8CD
:107BD00000B0099807F0F6FB10A9404603F074F8CE
:107BE0000EA98046059803F06FF80CA98146069807
:107BF00003F06AF80AA98246079803F065F83B4645
:107C000003908DE80007084A21460998013707F0DC
:107C1000F9FB0C2F06F1100605F110058BD113B0FE
:107C2000BDE8F08F303B0020DBC101082DE9F843AF
:107C3000054600262B7823B900210120BDE8F84332
:107C400072E705224E49284611F065F940B94D49C1
:107C5000002243181030C028DA60FAD1BDE8F8835A
:107C600004224949284611F056F904462846002CBA
:107C700040D101F095FE074600287ED00BF014FAA3
:107C8000DFF81C815FFA80F958F8245025B93F4885
:107C9000BDE8F843FEF728BC4A462946384611F0AD
:107CA0003AF901340028EFD1364A83181030C02841
:107CB000DE60DFF8D0E0F8D1354B03EBC404D4F834
:107CC000E8C0BCF1000F03D0002794F8E48005E081
:107CD0002946304806F0E4FF2F4DABE74745F7DA79
:107CE0003B010EEB03040C3463440FCB013784E8F3
:107CF0000F00F3E70EF008FC0B28064636D828469E
:107D000001F04EFE054638B102F04CFF1D4B012438
:107D100003EB0613D86000E00446284601F040FE5D
:107D2000054630B102F03EFF164B013403EB06135B
:107D30001861284601F034FE054630B102F032FFEA
:107D4000104B013403EB06135861284601F028FE5E
:107D500018B9BDE8F84301F0B7BE02F023FF094BA4
:107D6000032C03EB0616B061F3D165E70B2200216B
:107D70000A48BDE8F84301F04EBEBDE8F88300BFF5
:107D80004FC60108303B002056C1010886BA0108E1
:107D90000C9901085BC101083FB2010828BA01082B
:107DA000C0960108064B186840B19A6864214A439E
:107DB000B2FBF0F29A8000221A609A60704700BF0E
:107DC0002414002003788B4283BF034B03EB410153
:107DD00088890020704700BF24140020F0B50025DA
:107DE0002B46274E4219324492F82420244C83EA31
:107DF0000223082113F4004F4FEA430218BF82F414
:107E0000815201F1FF3118BF82F0010211F0FF0130
:107E100093B2EFD10135192DE4D100F1190200F12F
:107E20001A062244264492F8247096F82420144D11
:107E300002EB072292B29A4221D10B4695F8456097
:107E400001300C354FF4AF67DAB2964214D900EB2B
:107E50004202D1B262180131214492F824E091F833
:107E6000242002EB0E2292B27A43121302F54872DA
:107E700025F813200133E7E7012384F84630F0BDED
:107E80002414002007299DBF034B03EB8101B1F8A7
:107E900048000020704700BF24140020034B03EB70
:107EA0004101B1F86800C008704700BF24140020E9
:107EB00003788B420CD9074B89001A78064B19447A
:107EC000D1F8880002B1400800F5777080B27047A1
:107ED00000207047B44100202414002008B5084B4E
:107EE00003EB8101D1F8B8000BF03EFE05490BF021
:107EF00093FE05490BF088FD0CF090F880B208BDA8
:107F0000241400200000203F00005C440020704743
:107F1000024B03EB4101B1F800017047241400202B
:107F2000024B03EB4101B1F800017047241400201B
:107F300003788B4283BF034B03EB4101B1F8180177
:107F40000020704724140020024B03EB8101B1F89C
:107F5000380170472414002070B5054608F0DEFC97
:107F6000314CD4F87031C4F87001C31AB3F5FA5F1C
:107F700082BF002384F8743184F8753194F8743129
:107F80002BB9A12D02BF284A012182F8751194F85E
:107F90007511254A31B1D118EDB2013381F8245061
:107FA00082F8743194F8745194F87631AB4239D137
:107FB0001D4B93F87731052B02D0062B03D02CE014
:107FC0000020FFF70BFF94F825301E2B25D1002150
:107FD0000B46013DCAB2AA4217DA224492F8242085
:107FE00018461346082283EA00065B0816F0010FC4
:107FF000DBB202F1FF3218BF83F08C0312F0FF02F4
:10800000C0F34700EFD10131E4E7254495F824207F
:10801000934202D10320FFF7E1FE002384F875317B
:1080200084F8743170BD00BF2414002010B50446DC
:1080300008F074FC41F288310D4BD3F87821C3F875
:108040007801821A8A4284BF002283F87C2193F847
:108050007C210749142A134418BF013283F87D415B
:1080600012BF81F87C21012381F8923110BD00BF3D
:108070002414002038B5044608F050FC274A27494C
:10808000D2F89431C2F89401C31AB3F57A6F84BF61
:10809000002382F8983192F8983133B9A82C3BD15B
:1080A00081F89931A1F89A3106E0022B02D181F8CA
:1080B0009C4101E0242B02D8D11881F89D4192F80F
:1080C0009C1101330231DBB249008B42134D82F81F
:1080D000983118DAB5F89A31E0B283EA0020082323
:1080E00010F4004F4FEA400018BF80F4815003F1B4
:1080F000FF3318BF80F0010013F0FF0380B2EFD10F
:10810000A2F89A0138BD01318B4201BF002385F8E6
:108110009831012385F8993138BD00BF241400201F
:1081200010B5044608F0FAFB41F288310F4BD3F842
:10813000C421C3F8C401821A8A4284BF002283F892
:10814000C82193F8C831094A0F2B0DD8591CC9B260
:1081500013441029E4B283F8C94114BF002301235A
:1081600082F8C81182F8D93110BD00BF2414002054
:1081700010B5044608F0D2FB40F6AC51114BD3F8D1
:10818000DC21821A8A42C4BF002283F8E02193F8DE
:10819000E0212AB90F2C13D10A49C1F8DC0101E012
:1081A000182A0DD8511CC9B21929064883F8E011C4
:1081B000134483F8E14114BF0023012380F8FA310E
:1081C00010BD00BF2414002038B5054608F0A6FBFA
:1081D000364CD4F8FC31C4F8FC01C31AB3F57A7FED
:1081E00009DD0023282284F8003284F8012284F873
:1081F000023284F8033294F800322C4A83B93D2DC0
:1082000007D03E2D50D1012182F8021202F50271F1
:1082100004E0012182F8031202F50C71C2F8041285
:10822000D4F80412214ACD540133DBB2062B84F872
:1082300000321CD192F80232012B02D18B78282B0C
:1082400007D994F80332012B06D18B78092B03D878
:10825000164A82F8013238BD0023282284F8003201
:1082600084F8012284F8023284F8033238BD92F88F
:108270000112994218D192F802320C4D012B04BF21
:10828000022382F8023294F80332012B06D1022332
:1082900085F8033208F042FBC5F83C02002384F85D
:1082A0000032282384F8013238BD00BF2414002096
:1082B00038B5044608F032FB2249D1F84032C1F803
:1082C0004002C31AB3F5FA7F84BF002381F8443219
:1082D00091F844221B4B1ABB93F84502F0B9552C78
:1082E0000CD101201F2583F8460283F8454283F80C
:1082F0004752A3F8482283F84A0211E0202C1FD1EC
:10830000022083F84A024FF6FF7083F8462283F872
:10831000454283F84742A3F8480201E084420FD166
:108320008B1883F84B4291F847320648013B9A423A
:1083300003D1012380F86B3238BD013280F844222A
:1083400038BD00BF24140020084BDA68D10709D4D7
:10835000DA68520708D4DB6813F0100F14BF03204B
:10836000042070470120704702207047002002401F
:108370000A88F0B54B888E88B1F808E0CC88002ACE
:108380003AD1028C43F0010322F001021204120CD4
:108390000284058B078CADB225F0F30545EA0E117A
:1083A00089B246EA01027B49BFB2884212D001F588
:1083B000006188420ED0B0F1804F0BD0A1F598310A
:1083C000884207D001F58061884203D001F58061C1
:1083D000884202D127F0020701E027F00A071F4375
:1083E00002830784038B23F00C031B041B0C038301
:1083F000038B9BB21C4344E0042A44D1028C22F03C
:1084000010021204120C0284018B058C21F44072BC
:108410001205120D42EA0E325E4992B242EA06227B
:108420008842ADB292B212D001F5006188420ED0FE
:10843000B0F1804F0BD0A1F59831884207D001F5FB
:108440008061884203D001F58061884207D125F020
:10845000200141EA03139BB243F0100304E025F02E
:10846000A00143F010030B4302830384038B23F426
:1084700040631B041B0C0383038B9BB243EA04245D
:10848000A4B20483F0BD082A028C3ED122F480728B
:108490001204120C0284828B3E4D92B222F0F3073A
:1084A000018C47EA0E1292B2A84289B242EA060251
:1084B00012D005F50065A8420ED0B0F1804F0BD068
:1084C000A5F59835A84207D005F58065A84203D0E8
:1084D00005F58065A84207D121F4007141EA032324
:1084E0009BB243F4807304E021F4206143F4807371
:1084F0000B4382830384838B23F00C031B041B0C2C
:108500008383838B9BB21C4341E022F4805212048C
:10851000120C0284858B018C25F440752D052D0DE0
:1085200045EA062545EA0E321A4D89B2A84292B2B2
:1085300012D005F50065A8420ED0B0F1804F0BD0E7
:10854000A5F59835A84207D005F58065A84203D067
:1085500005F58065A84207D121F4005141EA0333B3
:108560009BB243F4805305E047F6FF5543F4805334
:108570000D402B4382830384838B23F440631B04CD
:108580001B0C8383838B9BB243EA0424A4B28483B1
:10859000F0BD00BF002C01400F4B1A6842F00102F1
:1085A0001A6059680D4A0A405A601A6822F08472AB
:1085B00022F480321A601A6822F480221A605A6803
:1085C00022F4FE025A604FF41F029A60044B4FF0EF
:1085D00000629A60704700BF001002400000FFF880
:1085E00000ED00E080F308887047074B5A694FF4AC
:1085F0007A73B3FBF2F3C3EB431203EB8203034A38
:10860000DB00A2F86C3270470C2D002024140020EF
:108610002DE9F8431346594C0D4607C884E8070076
:108620009A1EA4F51C74062A05D8DFE802F00A1089
:108630001822292F3500D4F870322B60D4F8743208
:1086400013E0D4F874322B60D4F8703205E0D4F81B
:1086500070325B422B60D4F874325B4205E0D4F890
:1086600074325B422B60D4F870326B60D4F878328D
:108670001DE0D4F870325B422B60D4F8743212E003
:10868000D4F874322B60D4F870320CE0D4F8703225
:108690002B60D4F8743205E0D4F874325B422B605E
:1086A000D4F870325B426B60D4F878325B42AB60D6
:1086B000334B1B78002B5FD128680BF059FA8046AA
:1086C00068680BF055FA0746A8680BF051FAD4F821
:1086D0007C12064640460BF09FFAD4F88812814679
:1086E00038460BF099FA014648460BF08DF9D4F85C
:1086F0009412814630460BF08FFA014648460BF043
:1087000083F90EF015F9D4F88012286040460BF07A
:1087100083FAD4F88C12814638460BF07DFA014674
:1087200048460BF071F9D4F89812814630460BF0A8
:1087300073FA014648460BF067F90EF0F9F8D4F8E1
:108740008412686040460BF067FAD4F890128046B5
:1087500038460BF061FA014640460BF055F9D4F863
:108760009C12074630460BF057FA014638460BF08C
:108770004BF90EF0DDF8A860BDE8F88394160020F0
:108780009400002038B50F4BD3F8A022D3F8A402F0
:10879000D48980F31000201A0BF0EAF90A490BF093
:1087A0003BFA054620460BF0E3F9014628460BF05C
:1087B000E7FA0BF00DFC6428A8BF642020EAE07003
:1087C000C0B238BD241400200000C84244F6FB713A
:1087D000084BD3F8A022137803EB431300FB0313D9
:1087E0005078C0EB0030B3FBF0F39078B3FBF0F0BF
:1087F00080B2704724140020F8B51A4B194F93F833
:10880000AA2293F8C66203EB4202B2F8BC52022ECF
:10881000ADB2A3F8C4521C4608BFA3F8C85293F8DF
:10882000D0324BB94CF250320F4907F535700AF08F
:108830001DFB012387F8D03228460BF095F9094D2E
:10884000014605F535700AF059FA0BF0E7FB80B2E6
:10885000FFF7BCFF022EA4F8F00208BFA5F8CA0279
:10886000F8BD00BF24140020CDCCCC3EF8B51A4D85
:108870000746D5F8F442092C2BDC002305F53E729F
:108880009C4205DD52F823108F4222D00133F7E7D6
:10889000DFF848E00022A2421BDC5EF822109600BE
:1088A0000E48531C71B9A21A8119920000EB830083
:1088B0002E44013410F0CFFAC6F8F872C5F8F4422D
:1088C0000120F8BD91F814C0397D8C45EBD31A46D0
:1088D000E1E70020F8BD00BF241400201C17002091
:1088E0000B2870B506D009282AD8164B342202FB73
:1088F000003002E0144BD3F8240309B1C36823B954
:10890000114B0022D3F8F44203E0BDE87040ADE71C
:108910000A46A24214DA0C4D960005F53E7353F850
:108920002210884202F10101F2D1A21A920003EB57
:1089300081019819013C10F08EFAC5F8F44270BD1F
:1089400070BD00BF98000020241400202DE9F041E4
:1089500005460F46094E441E06F1080814F8011F8B
:1089600051B1064810F0C9FA0028F7D040453EBF83
:10897000801B631B3B54F1E7BDE8F08185A0010833
:10898000094B93F828235AB9D3F82C230749527E70
:1089900009780432D2B28A4228BF0A4683F82823D3
:1089A00093F82803704700BF24140020B041002032
:1089B00070B513494300D1F82C230E46D41894F80F
:1089C000205015B1022D10D00BE0022805D9032844
:1089D00007D1D1F83033DB0401D5108A70BD908BFC
:1089E00070BD3344B3F8340370BD94F8210000EB3C
:1089F000800000EB800000F2EE2080B270BD00BF6E
:108A00002414002008B507F089FF074B022283F8E1
:108A10005C23D3F86023C3F85803C3F86C23012206
:108A200083F8852308BD00BF2414002008B507F093
:108A300075FF084B022283F85C23D3F86C2300F502
:108A4000B71000F5587002F2DC52C3F85803C3F8AF
:108A50006C2308BD2414002030B504460B4D0023C0
:108A6000221AD2B291420ED914F8012B53409A0027
:108A700082EA43025A40DB0803F0180345FA03F385
:108A80005340DBB2ECE7184630BD00BF0007090ECB
:108A900070B5064604460020A31BDBB299420ED9EE
:108AA00014F8013B020A434083EA0313DBB2DD0002
:108AB00042EA032285EA131382EA0300ECE770BD61
:108AC0000E4B10B593F888131C46012909D005D325
:108AD000022909D1002004F045FB05E000210846E9
:108AE00000E0002004F064FD07F018FF00F5F4201A
:108AF00000F59070C4F88C0310BD00BF2414002052
:108B00000168027B30B502230C6803FA02F22242AC
:108B10000BD0064A002414704FF6FE724468256894
:108B20002A402260027B93404B6030BD2D430020E1
:108B300038B50546054C206804F026FD284608F0A7
:108B4000A3F82068BDE8384004F023BDD009002018
:108B5000F8B507460E461546084C206804F014FD8B
:108B600047F0800008F090F832460021284608F0CF
:108B70004FF8206804F00DFD0120F8BD482D0020BD
:108B800070B506460D46074C206804F0FDFC3046E3
:108B900008F07AF8284608F077F8206804F0F9FC25
:108BA000012070BD482D00202D4B2E4A1B681268F5
:108BB00030B51A602C4A2D4C116859605168926882
:108BC0009960DA602A4A116819615168926859619E
:108BD0009A61284A1168D9615168926819625A628B
:108BE000254A11881985518859859188D288998597
:108BF000DA85224A116819865168926859869A86E0
:108C00001F4A1168D9865168926819875A871D4A88
:108C1000118899875188D9879188D288A3F8401004
:108C2000194621F8422F184A10780022824205DAAC
:108C300034F91250013221F8025FF7E7134A128823
:108C4000A3F86C20124A1288A3F86E20114A1288E9
:108C5000A3F87020104A5289A3F8662030BD00BFE7
:108C6000D8370020380D00204C2600208439002001
:108C70005826002064260020B01F0020C01F0020BE
:108C80000C130020EC160020CF1F0020E816002057
:108C9000D8410020D4430020FC090020124A38B5F6
:108CA000137814460B2B17D840F6030501229A407F
:108CB0001540BDB912F4C06F0ED0093B012B0BD883
:108CC000452009F0B7FCFF2009F0B4FC074809F083
:108CD0002FFC284609F0AEFC054B1A68054B5A607C
:108CE0000B23237038BD00BF7A27002028C201085B
:108CF00084170020AC0A00202DE9F04F854E85B086
:108D00003578012D40F00381834C94F8572522B12A
:108D100094F858350BB19A4203D3012384F85735A0
:108D20000FE01846114630B191FBF0F700FB171722
:108D300001463846F7E792FBF1F293FBF1F384F832
:108D4000572584F8583594F85935012B82BF724B5A
:108D5000002283F8592594F8597517B1012F32D0A4
:108D60003BE0802003F048FA8046002835D080217F
:108D700003F018FA694B98F806201870684B98F9B8
:108D8000000053F822308021B3F5613F0CBF02226E
:108D900000220192022200923A4603F099F9614BB7
:108DA0004FF4FA721860604B1B6803EB4303B3FB8C
:108DB000F2F31BB1402BA8BF402300E001235B4A24
:108DC000137060B909E05A4BDB6833B109F088FBD6
:108DD00018B9564B40221A7001E000238FE014228C
:108DE0000021544810F052F800208646524A534B56
:108DF00094F85775136003F17401E8339360504B96
:108E000051601A884F4B94F822921A8094F8582592
:108E10004D4B97424D4A186012684D4B03924D4A94
:108E2000196892F80080637994F844222CBF0027D7
:108E300001278242A3F11902C1F3400A01F4006C38
:108E4000C1F3C03118BF012154425441012B08BF66
:108E500001246A1ED2B2531E132B2AD8DFE803F076
:108E60000C0C0C0C0C0C0C0C0A2F2F51182F53113E
:108E70001111262F234647E09045B4BF002301235C
:108E800016E0039B13445B79003318BF01230FE006
:108E9000BCF1000F06D009F1FF3BDBF1000343EB0F
:108EA0000B0300E0634603F001032DE03B462BE09B
:108EB0002BB10123184603FA02F24EEA020E142DDA
:108EC00002D80135EDB2C4E710B11F4BC3F800E082
:108ED000192007F00EFF204B204A18700023136062
:108EE0001F4A13801F4A13801F4A11681F4A1160CE
:108EF0001F4A11681F4A11601F4A13700223337002
:108F000005E0534600E00B46002BD2D1D9E705B06F
:108F1000BDE8F08F7A270020303B0020C60A0020F1
:108F200080B10108A00A0020D01F0020A80A00205C
:108F300084000020B4170020D8370020E437002038
:108F4000E8160020B80A0020B40A00200814002007
:108F500054170020CF1F0020C40A0020C00A0020A0
:108F6000BC0A002048390020E84100204039002098
:108F7000F435002044390020350D00207FB5264C03
:108F8000264E274D2749284A284B20B128480088DB
:108F9000B0F5805F31D230681F4E91F82010127802
:108FA000019028781B7806F114058DF808008DF8DB
:108FB00009108DF80A202946082201A88DF80B30E7
:108FC0000FF03AFF28B301AB03CB70616960532007
:108FD00009F030FB606909F0E8FB207E09F0E5FB51
:108FE000637E01A80193A37E0293E37E039309F0BD
:108FF0004DFB0F4B00221A800BE0306891F82010D7
:109000006061127828781B7820766176A276E37604
:10901000DDE704B070BD00BFB4170020F4350020B8
:10902000A113002088170020640D0020120E0020DC
:10903000BA0A00202DE9F04188460D4B00249D68B6
:1090400093E8C00005440644074444450EDA37F966
:10905000142035F9143036F914001344022293FB1E
:10906000F2F3C01A09F0B0FB0134EEE7BDE8F0817D
:10907000D8370020094A137818441346C0B210F0BC
:10908000800F18BF80381070054A197813789942FC
:1090900001BF00231370014A13707047C5130020ED
:1090A000C413002010B50A4B0A4A1B7842609C1872
:1090B000094A0460127893429BBFD31A0B60C3F134
:1090C0008003002392BF4B600B604A6010BD00BF5D
:1090D000C5130020AA420020C41300201FB502A817
:1090E0006946FFF7DFFF044B00981B6803440198B3
:1090F000184405B05DF804FBC8130020054A064B70
:1091000010781B7883422EBF181AC0F18000C01857
:10911000704700BFC5130020C4130020104B37B5A3
:1091200018781C46A8B10F4D05238DF8003028682B
:1091300000238DF8013004F027FA0222694601A8C5
:1091400007F066FD286804F024FA9DF8050000F099
:10915000010000F00100207080F0010003B030BD7C
:10916000D4090020D0090020064B70B506461C46E5
:109170001D68FFF7D3FF18B923685B1BB342F8D90A
:1091800070BD00BF841700202DE9F04F824689B0E2
:1091900002930023039104920193049A934207DA05
:1091A000039A019952F82320013311440191F4E705
:1091B000029B23B9FFF7B2FF08B9029878E0019D3E
:1091C000002D73D03C4B1B68DCB22A19B2F5807FAE
:1091D0003A4A88BFC4F58074D26898BF2C4693423F
:1091E00005D3374A00231370364A13705EE0D14628
:1091F000264602228DF81C201A0C8DF81D20062010
:109200001A0A8DF81E208DF81F30FFF7ADFF0620DB
:10921000FFF78EFC2C4A012313702C4B0027186893
:1092200004F0B2F9042207A9002007F0F1FCDDF8F0
:109230000C80049B9F422CDA434658F8042B4FEADB
:10924000870B12B3964210D832465AF80B10002002
:10925000059307F0DDFC5AF80B20059B32444AF8D1
:109260000B201A68961B1E6013E0D9F8001000202E
:1092700007F0CEFC58F8043CD9F80020F61A134445
:10928000C9F80030002348F8043C013709F104090B
:10929000CFE70E4B2D1B186804F07BF9064B1B68BB
:1092A0001C44054B1C60029B002B89D1019B581B61
:1092B00009B0BDE8F08F00BFC81300208400002073
:1092C000C4130020C5130020D4090020D0090020B9
:1092D00030B50B4C0B4D22782B7885B09A420CD0D0
:1092E00002A96846FFF7DEFE0123022202A96846B2
:1092F000FFF74AFF00232B70237005B030BD00BF7D
:10930000C5130020C413002030B50E4D0E4C2A7832
:10931000237885B09A4211D002A96846FFF7C2FEB1
:109320000023022202A96846FFF72EFFFFF7A2FEE4
:1093300020782B781B1A5842584100E0012005B0D4
:1093400030BD00BFC5130020C413002073B5032334
:109350008DF80430030C8DF805308DF80700030AF2
:1093600006200E4614468DF80630FFF7FDFE90B13C
:109370000A4D286804F008F904220DEB02010020D0
:1093800007F046FC22460021304607F041FC2868E1
:1093900004F0FFF8204602B070BD00BFD0090020E5
:1093A00008B545F20820FFF7DFFE0620FFF7C0FBF7
:1093B000034B01221A70C720BDE80840FFF7B8BB75
:1093C000D40900202DE9F04F884A85B01378029225
:1093D00003F0FF05002B40F0058129462F46AE46DD
:1093E000AC46AB46824E3C2496F8202096F821905D
:1093F00096F82230B583F58301960FFA85F8B8F117
:10940000200F00F0BF807B4800EB880C9CF8030025
:109410009CF802C0CCF1FF0C1FFA8CFCBCF1000FD1
:1094200000F08280734ECCF1FF0C36F828803C2689
:10943000B8FBF6FA00FB0CFC4FEA2C2CBAF1050F36
:1094400075D8DFE80AF003102233485A5FFA8CF32C
:10945000CCEB000C08FB0CF8B8FBF4F8984402467F
:109460005FFA88F05CE0B8FBF4F204FB128292B27F
:109470005FFA8CF3C2F13C02CCEB000C0CFB02F265
:10948000B2FBF4F21A44D2B24AE0B8FBF4F304FBA4
:1094900013885FFA8CF21FFA88F8CCEB000C08FBFB
:1094A0000CF3B3FBF4F31344DBB239E0B8FBF4F391
:1094B00004FB13881FFA88F85FFA8CF2C8F13C08A5
:1094C000CCEB000C0CFB08FCBCFBF4FC9444034606
:1094D0005FFA8CF024E0B8FBF4F204FB12885FFA28
:1094E0008CF11FFA88F8CCEB000C08FB0CF2B2FBF5
:1094F000F4F20A44D2B2034611E0B8FBF4F304FBE1
:1095000013839BB25FFA8CF1C3F13C03CCEB000CEC
:109510000CFB03F3B3FBF4F302460B44DBB2084647
:1095200001210F468E4603E003460246F8E748460F
:109530004FEA02284FF0170C48EA00480BEB0C06E4
:1095400048EA03080396039ECCEB0609012606FAB7
:109550000CFA1AEA080F284E14BF4FF0110A4FF008
:10956000090A1FFA89F91CF1FF3C06F809A0EAD2A2
:109570000BF1180C01351FFA8CFBADB24FF0010C4A
:1095800081463AE7BCF1000F02D00198A0F81CB068
:10959000BEF1000F02D0019880F8202017B1019A87
:1095A00082F8219011B1019A82F82230BCF1000FAB
:1095B00002D0019A2023D383029A012313700F4B08
:1095C0001B787BB140F22A330D4A0E4953600023C9
:1095D0008B840B889BB243F001030B80136843F02C
:1095E0000103136005B0BDE8F08F00BF2D430020DC
:1095F000B41700202E43002084060020B409002068
:109600006C000240000400402DE9F84307F086F9A1
:109610000546DFF88C8000F1FA0998F80040204FE9
:10962000A40008EB0406706803F0CAFF58B107F005
:1096300075F98145F1D24FF0FF30BDE8F88307F0AE
:109640006DF98145F7D37068DFF8548003F0B8FFF7
:109650000028F4D007F062F9D8F83830401B98425F
:10966000C8F8340018D805F5FA753E19706803F08B
:10967000A7FF20B107F052F98542F7D2DBE73C445F
:10968000606803F09DFF20B907F048F98542F7D2E2
:10969000D1E70020BDE8F8830120BDE8F88300BFD2
:1096A000D817002038B5054600240470FFF7ACFF3A
:1096B000431C13D0012802BF2B78A040184304F1AB
:1096C000010408BF2870082CF0D1054A297892F8C7
:1096D0003C3001204B4082F83C3038BD002038BD82
:1096E000D81700202DE9F04381460D46374C87B04E
:1096F00000274FF0190895F8FD2494F8FD3495F8EB
:10970000010593421DD194F8FE1495F8FE34994258
:1097100017D194F8FF1495F8FF34994211D194F8B9
:10972000001595F8003599420BD194F80135834224
:1097300007D195F8021594F802355B1A5942594140
:1097400000E00021059095F800350E46049395F849
:10975000FF34484608FB03F303F56173039395F860
:10976000FE34019208FB03F303F56173029395F84D
:109770000235174A00933B4605F024FE94F8013564
:10978000134A059394F800353146049394F8FF3456
:10979000484608FB03F303F56173039394F8FE3422
:1097A000063508FB03F303F56173029394F8FD3467
:1097B0000634019394F8FC3400933B46013705F0DE
:1097C00021FE0F2F97D107B0BDE8F083303B00207A
:1097D00033C201082DE9F04780460D463B4CDFF8C7
:1097E000F8A03B4F86B004F1280994F9A622002383
:1097F00013F90A10914203D00C333C2BF8D15AE0F4
:1098000095F9A6329A4295F8AC225CD1B4F8A80238
:10981000B5F8A812884256D194F8AA0295F8AA126F
:10982000884250D194F8AB0295F8AB1288424AD1E5
:1098300094F8AD0295F8AD12884244D194F8AC1278
:10984000881A4142414157F822200E46049295F869
:10985000AD22404657F82220039295F8AB2257F8E4
:109860002220029295F8AA2257F822200192B5F8F8
:10987000A8220092174A05F0A5FD94F8AC2294F9AD
:10988000A63257F822203146049294F8AD22404681
:1098900057F82220039294F8AB2257F82220029224
:1098A00094F8AA2257F822200192B4F8A822009234
:1098B000084A05F0A7FD08344C4505F1080594D188
:1098C00006B0BDE8F0870021BDE700BF303B0020B7
:1098D00080B1010853C20108B04000202DE9F043D7
:1098E00081460E462C4C85B000274FF0190894F89D
:1098F000AD3496F8AD24934296F8B03411D194F873
:10990000AE0496F8AE1488420BD194F8AF0496F8E2
:10991000AF14884205D194F8B054E91A4D424D4134
:1099200000E0002508FB03F303F56173039396F849
:10993000AF34294608FB03F303F56173029396F8ED
:10994000AE3448468DE80C003B46144A05F03AFD1B
:1099500094F8B034114A08FB03F303F561730393E1
:1099600094F8AF34294608FB03F303F561730293BF
:1099700094F8AE344846019394F8AD34043600931D
:109980003B46013705F03EFD142F04F10404AED12F
:1099900005B0BDE8F08300BF303B002072C2010873
:1099A00008B520210FF0A9FA034618461BB102782A
:1099B0000133202AF9D008BD2DE9F84380460C4632
:1099C000154640F634074FF0000919264046FFF7C8
:1099D000E7FF8046B8B10CF097FDB0F5617F03DB7F
:1099E000B842A8BF384601E04FF46170A0F561703D
:1099F00090FBF6F0B9F1000F01D1207000E060702B
:109A00002B7801332B7009F10109B9F1020FDDD177
:109A10004046BDE8F88313460A460146014805F072
:109A20003FB900BF87C2010873B50178044619B970
:109A30000120FFF753FF41E00CF066FD13280546B7
:109A400037DC0023601C8DF80730FFF7A9FF1C4CA2
:109A5000064605F5957558B10CF056FD1D2807D83A
:109A600004EB850358719DF8073001338DF80730FA
:109A70003046FFF795FF064658B10CF045FD0D281E
:109A800007D804EB850398719DF8073001338DF8F2
:109A9000073004EB85040DF10702E11D3046FFF7A6
:109AA0008BFF9DF80730042B08D00023C4F8053045
:109AB00004E0132200210348FFF7ADFF02B070BDA0
:109AC000303B002028BA01080148FCF70DBD00BF5B
:109AD000A6C20108F7B50178054619B90120FFF7BC
:109AE00001FE6FE00CF010FD0E28044665DC00233B
:109AF000681C8DF80730FFF753FF334E054668B1F9
:109B00000CF002FD032809D8062303FB046383F845
:109B100002059DF8073001338DF807302846FFF71E
:109B20003FFF074668B10CF0EFFC0D2809D806236B
:109B300003FB046383F8FD049DF8073001338DF8BF
:109B400007300625654371190DF1070201F2FE4148
:109B50003846FFF731FFFFF723FF074660B10CF0EF
:109B6000D3FC142808D8184B1D449DF8073085F8FD
:109B7000000501338DF807303846FFF711FF68B153
:109B80000CF0C2FC0D2809D8062303FB046383F8FC
:109B900001059DF8073001338DF807309DF8073037
:109BA000062B0FD0062303FB04640023C4F8FD3406
:109BB000A4F80135FFF788FF04E00E2200210348D6
:109BC000FFF729FF03B0F0BD303B002028BA0108A1
:109BD0002DE9F34103781BB902B0BDE8F04173E70A
:109BE00058490CF0CDFC002605463446B0464FF0EF
:109BF000FF376DB3012E07D0022E0AD00EBB2846C8
:109C00000CF082FC07461CE028460CF07DFC8046E8
:109C100017E04D4928460FF0CFF920B94B492846A7
:109C20000FF0CAF908B144F00104494928460FF081
:109C3000C3F920B9474928460FF0BEF908B144F0EE
:109C40000204404900200CF09BFC01360546D0E799
:109C5000414B78B20C2606FB05F2D118D25682424F
:109C600023D00135052DF6D1B8F1000F02D13946C8
:109C70003A480FE0002C08BF03240022E4B201920E
:109C8000009443464FF4807102F022FA054630B941
:109C90003946334802B0BDE8F04101F076B942469A
:109CA0003946304801F071F907E04D68002DDBD0EE
:109CB00039462D4801F069F9C4BB2C4801F065F91B
:109CC0002B4B1C68204602F0C7F9284602F0C4F965
:109CD0000021084603F06CFC0021012003F068FC21
:109CE000204601F063FC70B10121002003F060FC0C
:109CF000204601F058FC0146284601F05AFC00219C
:109D0000084603F055FC284601F050FC0028E7D037
:109D10000121002003F04CFC284601F044FC0146E0
:109D2000204601F046FC00210846D7E769798C42BD
:109D3000C3D022460F4801F028F9E1B2284601F0CD
:109D40002CFCBAE770C10108B4C2010878D201083E
:109D5000B7C2010870D20108B0400020BAC20108A1
:109D6000E7C2010805C301081FC3010866C3010853
:109D7000CC13002036C301082DE9F743017821B93F
:109D8000012003B0BDE8F04324E5002200920192D7
:109D9000451C0CF0B9FB44B2204602F0EFF9064630
:109DA00018B18DF80040012400E004462846FFF772
:109DB000F7FD074628B10CF0A7FB0134ADF802000F
:109DC000E4B2DFF88C900025C8463846FFF7E8FD7E
:109DD000074680B30CF098FB002159F82120CBB244
:109DE000904203D001310829F7D1002358F82320ED
:109DF000904220D1022D0FD0032D12D05A1E012DDA
:109E0000D2B204D0042A13D88DF804300EE0042A0C
:109E10000ED88DF8053009E0052B09D88DF80730EC
:109E200004E09A1E052A03D88DF806300134E4B206
:109E30000135042DC9D1052C03D803B0BDE8F0438A
:109E400042E66B4603CB3060716003B0BDE8F0833F
:109E500080B10108F7B5047805464CB901A9204640
:109E600002F04EFE0134FFF7F5FF122CF6D16DE043
:109E70000CF04AFBC4B2112C63D8681CFFF790FDAC
:109E8000334D074640B9334B04F5967213F8121060
:109E90008A1E514251413CE0017828460FF02DF8CE
:109EA00050B1032C8CBF032300232B4A401BC0B2AC
:109EB00013441E5C032E02D1FFF706FE46E038462F
:109EC000FFF76EFDD8B1022EF6D10CF01DFB40F26B
:109ED000ED2380B2984205DD40F6CA039842A8BF40
:109EE000184601E040F2EE20A0F2EE20192290FB8D
:109EF000F2F0184B03EB440383F8590201E0022E01
:109F0000DAD0B31E5942134A594104F5967302F848
:109F10001360104B04F5967013F81020AA5C59B129
:109F200003EB4003597819234B430C4803F2EE230B
:109F3000214604F0B5FE09E02146094804F0B0FED0
:109F400004E0112200210748FFF765FD03B0F0BDD2
:109F5000AC980108303B00209AA00108D2BC01084F
:109F6000E4BC01083BC4010808B50448FCF7BCFA8E
:109F7000034B1868BDE8084003F03CBBBEC30108B2
:109F800024360020F7B50023454C464E8DF80330AB
:109F90006023A36333780746152B06D0122B04D019
:109FA000012B0CBF02258C2501E044F62065FFF74C
:109FB0002BFB002802DA013DF9D16EE00A25FFF7FC
:109FC00023FB013069D0013D15F0FF05F7D1626B2D
:109FD000930803EB5203A363FFF716FB431C5CD00B
:109FE0000028F9DC00230DF1030084F83C30FFF772
:109FF00059FB002851D09DF803301B2B4DD10DF19A
:10A000000300FFF74FFB002847D0254B9DF80320A6
:10A0100093F83D309A4240D10DF10500FFF742FB25
:10A020009DF80530012B38D801A8FFF73BFB9DF8C0
:10A03000043093B30DF10300FFF734FB68B39DF8D0
:10A0400003300E2B29D10DF10300FFF72BFB20B3BA
:10A050009DF8032033789A421FD10DF10300FFF7DA
:10A0600021FBD0B19DF80330BBB93D46BDF80430AB
:10A07000EA1B92B2023B9A4205DA2846FFF712FB2E
:10A0800058B10135F2E70DF10300FFF70BFB94F82F
:10A090003C00B0FA80F0400900E0002003B0F0BDC1
:10A0A000D81700203C34002010B50A4C94F83E002C
:10A0B00003F056FD237804EB8304606803F069FA2B
:10A0C000202006F047FC60684A21BDE8104003F0FC
:10A0D0007DB800BFD817002010B5104C122123788E
:10A0E00004EB8303586803F071F8FF2003F038FD98
:10A0F000FF2003F035FD7F2003F032FD00231B20FD
:10A1000084F83E3003F02CFD94F83D000130C0B2DD
:10A1100084F83D00BDE8104003F022BDD8170020B0
:10A120000B4B10B501241C70FFF7D6FF002003F085
:10A1300017FD204603F014FD0E2003F011FD20460C
:10A1400003F00EFDFFF7B0FFBDE81040014819E72E
:10A150003C3400203D34002073B5047805462CB112
:10A1600004F10A03ADF80430002604E04FF48573CF
:10A17000ADF804300126FFF7AFFF9DF8050003F0AE
:10A18000EFFC9DF8040003F0EBFC0E2003F0E8FC6C
:10A19000184B187803F0E4FC304603F0E1FC20464D
:10A1A00003F0DEFC002003F0DBFC002003F0D8FC11
:10A1B000002003F0D5FC002003F0D2FC002003F0C7
:10A1C000CFFC002003F0CCFC002003F0C9FC6B683E
:10A1D000013C187803F0C4FC6B6814F0FF0403F131
:10A1E00001036B60F3D1FFF75FFF034802B0BDE8E6
:10A1F0007040C7E63C3400203D34002038B5047878
:10A200000546B4FA84F4FFF767FF002003F0A8FCCA
:10A21000042003F0A5FC0E2003F0A2FC094B640906
:10A22000187803F09DFC204603F09AFC287803F090
:10A2300097FCA02003F094FCFFF736FF6868BDE8A8
:10A2400038409FE63C34002038B50368164A23F0B6
:10A250007F4323F0FF039342044622D0134B06258D
:10A260001D70FFF739FF002003F07AFC052003F092
:10A2700077FC0E2003F074FC284603F071FC0020EC
:10A2800003F06EFC002003F06BFC607803F068FCC8
:10A29000A07803F065FCFFF707FFBDE838400448ED
:10A2A00070E6012038BD00BF00FFFF003C340020F5
:10A2B0003D340020F0B50124B0FBF4F58D4201D30C
:10A2C0004C43F9E70026CCB1B0FBF4F504FB1500D4
:10A2D000B4FBF1F41EB9002D01DC002CF3D1092DE3
:10A2E00003F1010E04DD002A14BF3727572700E0D1
:10A2F00030273D441D7001367346E4E71C70F0BD05
:10A3000003685A1C026019707047F8B504462A2287
:10A3100000210EF0BBFD23460A4904F12800052266
:10A320000426002511F9017F9A719F70DE715D721C
:10A3300003F8082F8342F5D10123A3805223237011
:10A34000F8BD00BF9FA00108014B186801F031B9AA
:10A35000181800200E4B1A78922A16D15A88B2F596
:10A36000AF6F12D11A79BE2A0FD193F8642500205D
:10A37000EF2A0CD1074A13F8011B934280EA01002F
:10A38000F9D1B0FA80F0400970470020704770475B
:10A3900000F8010878FD01082DE9F74FFFF7DAFF13
:10A3A00010B9042006F002FBB64CFEF73FFB4FF459
:10A3B000AF62B54920460CF0D7F894F8AC34B34EF0
:10A3C000012B84BF002384F8AC3494F8AC246C23B4
:10A3D0005A43A31803F575733360A31893F8183420
:10A3E000AB49AC4D0B700C2101FB032346F2090273
:10A3F000234403F21A432B60A3681A401AB9A14AF6
:10A4000043F001039360A368DF0703D54FF40050C6
:10A4100003F02AF9A368580409D5082003F024F9A9
:10A420004FF4005003F020F9012003F01DF9A36858
:10A43000190706D54FF4005003F016F9012003F078
:10A4400013F9A3689A0413D54FF4004003F00CF9F4
:10A450008C4B93F82232012B03D14FF4006003F0B0
:10A4600003F94FF4803003F0FFF8402003F0FCF8CC
:10A47000A3685B0603D54FF4803003F0F5F84FF086
:10A480000009C846844F854B4FF0FF0A1F6004EB5C
:10A490000903B3F8A802410801F07731830803F0FB
:10A4A0003333C1EB000CC3EB0C01C30803F01133D1
:10A4B000CB1A03EB231303F00F3292FBFAF310F0E5
:10A4C000010EC3EB032318BF08F10108A2EB03033D
:10A4D00018BF5FFA88F8012B10DD022B40F0CE8008
:10A4E000BEF1000F02D010F0BC0F07D109F2A62078
:10A4F000204404F099F9002800F0C08009F108090F
:10A50000B9F1280FC3D108F1FF38B8F1010F00F2FB
:10A51000B580DFF8E4812868614D414601F074FEA2
:10A5200030220021281D0EF0B1FC33680020C5F850
:10A530003480AB6306F0DDFB5A4B80F001001870ED
:10A54000B4F8E011B4F8DE01994688429CBF0023BC
:10A55000A8F81231B4F8E221CDF80480B4F8E4810F
:10A5600094F8DCC142459EBF464A0020A2F8E201B1
:10A570004D4AB4F8DE0182F800C04C4AB4F8E2B1AA
:10A5800010804B4A94F8DBE1A2F800B0DFF86CA130
:10A59000484AC5F83CA082F800E008F073FC464A3F
:10A5A00041461060584608F06DFC444B94F89A12EE
:10A5B00018600AF1E4032B64336864221B784A4371
:10A5C000012B14BF3E4B3F4B3F4EC9F804303F4B6D
:10A5D000C8321E603E4B6F655A6000229A60DA6096
:10A5E0001A615A619A61DA6183F8202083F8212088
:10A5F000A6F16E036B64D4F8F831A6F5A372AB64D0
:10A60000344BB4F8E6011A60A6F1D603EB64324B82
:10A61000A6F5E2721A60019A304B1A60A6F108039F
:10A620002B6509F0A5FA2E4909F0AAFB2866B4F8B3
:10A63000E80109F09DFA2A4909F0A2FB94F81032CA
:10A640009E3E85F8593094F89032E86585F864307C
:10A65000244BB4F81202AB66234BEE662B6709F06D
:10A6600087FA0146214809F08BFB214909F0D4FA09
:10A67000686703B0BDE8F04FFEF7C4B91D48FFF7A7
:10A6800044FE46E7303B002000F801080814002093
:10A69000CF370020C8350020683D0020501700202B
:10A6A00018180020A0020020552D0020562D002053
:10A6B00084330020582D002088330020E033002010
:10A6C00033B6000831B90008CA3D0020F43A002032
:10A6D00088170020C03A0020403A0020443A002069
:10A6E00000401C46701800203661023D00006144A5
:10A6F0004C3D0F44D43D0020FC3B00201C3D00207D
:10A70000F0B52D2646730F264671222686710E2639
:10A71000067435262825867619262B22C572C67121
:10A7200045722126372542703A2114221624467498
:10A730008572532605754FF4FA75012342758170B1
:10A7400084753221C275C67600224B26C585462403
:10A750004FF42F7503700677867705860173C470F2
:10A76000017182730276C2734276017281744284EF
:10A77000C37780F8283080F834301E2380F83630D4
:10A78000C8234FF4827780F83730DC23878403872F
:10A79000A0274FF08043C784C36340F2726703462B
:10A7A0008225458520258585642580F840600584BF
:10A7B00080F83320428780F8352080F8412000F16E
:10A7C00024064FF00A0E83F8465083F8475083F86A
:10A7D000482083F8491083F84A2083F84EE083F834
:10A7E0004F20A3F8507083F84B4083F84C4083F817
:10A7F0004D400C33B342E6D1002380F84430F0BD25
:10A800002DE9F74F04464FF4AF6200210EF03EFBF6
:10A8100040F2031340F6C4124FF49670A4F8E0011E
:10A82000C820A4F8E2016420A4F8E4014FF42F70DA
:10A83000A4F82A02202084F8EC016E20A36084F89A
:10A84000160292230A202370A4F8E621032308228B
:10A850005A2184F817022B20637184F8DA2100232F
:10A86000012284F8DC1184F819024FF4C871212008
:10A8700084F8EA21A4F8DE1184F8D42184F8ED21CB
:10A8800084F8EE2184F8182284F8AC34A4F8E83176
:10A89000A4F8D83184F8DB3184F8EB31A4F82E32F7
:10A8A000A4F82C32A4F8303284F8C53184F8C631CB
:10A8B00084F8C73184F8D53184F81A0284F81C2250
:10A8C00084F8222284F8D12284F8412284F8432299
:10A8D00040F2DC52A4F8482240F24C42A4F84A224A
:10A8E00040F26C72A4F84C2240F27532A4F8542263
:10A8F00040F64302A046A4F8562222462320A4F89C
:10A900001E12052184F81B02A4F82032A4F8243278
:10A9100084F8D03284F8DC3284F8DD3284F8DE3218
:10A9200084F8DF3284F8E01284F8403284F842324E
:10A930004FF0000A032BCCBF0121002103F10103DA
:10A9400082F858120CBF05211E21122B82F85912D1
:10A9500002F10202EED1002384F8443284F8463238
:10A9600084F85032062384F8513240F246531E22B6
:10A9700084F84522022284F84E22132284F84F22C2
:10A98000A4F8523204F5247204F520734FF47A705F
:10A990004FF4FA6123F8040C23F8021C04339A42A2
:10A9A0004FF47A774FF4FA6BF4D1052384F88F32A1
:10A9B000192384F8903240F22E43A4F8CC3040F2B0
:10A9C0007E53A4F8D63040F2EA53A4F8D83040F2CF
:10A9D000B45340F2DC52002501264FF4C871A4F8AC
:10A9E000DA303223A4F8D220A4F89412A4F8DC3090
:10A9F000A4F8DE10A4F8E03084F88C5284F88D526C
:10AA000084F88E6284F8926284F8936284F8965295
:10AA100084F89862A4F8D45084F8E26004F52970B0
:10AA2000A4F8CEB0A4F8D07004F575790192FFF7C0
:10AA30006CFC4846FFF764FE454BA4F8F251C4F89D
:10AA4000F8312823A4F8F451A4F8F05184F8FC312B
:10AA500084F8FD3184F8106204F50E713D480093CE
:10AA6000FDF774FF009B642184F828324FF448738B
:10AA7000A4F812320A2384F89A3284F89B322346CF
:10AA8000019A84F8265284F8275284F8296284F8BF
:10AA9000145284F89E5284F8A262A4F89C72A4F81E
:10AAA000A01204F170055A20FF26A3F85471A3F8F0
:10AAB00056B1A3F8582183F85A1183F85B0183F843
:10AAC0005C0183F85D610E339D42EED1002384F872
:10AAD000C43104F1C003C8F80CA008F110084345C4
:10AAE000F9D104F559753822002128460EF0CEF927
:10AAF000194A002352F8230045F8230001330E2B96
:10AB0000F8D18022002104F539700EF0BFF924221B
:10AB1000124904F569700BF027FD0B22104904F56A
:10AB200072700BF021FD49460122002384F857255D
:10AB300084F8582504F588606C2284F8D33384F8AF
:10AB4000593584F85A3503B0BDE8F04F0BF00CBD11
:10AB500000002041C3C30108A6A00108DEA001082F
:10AB600002A1010810B50B4C2046FFF749FE0A4B25
:10AB700004F575721A6094F81834084A13700C22A0
:10AB800002FB0343BDE81040054A03F21A43136079
:10AB900007F012BC303B002008140020CF37002003
:10ABA000C83500202DE9F04102780346202A00F143
:10ABB0000100F9D0092AF7D02D2A02D103463F4DD2
:10ABC00004E02B2A08BF03464FF07E551C460026A2
:10ABD000234614F8012BA2F13007F9B209290CD849
:10ABE0003749304609F018F80646384608F0C0FFE5
:10ABF000314608F009FF0646EAE72E2A17D1304F02
:10AC0000234614F8010B3038C2B2092A0FD808F0D5
:10AC1000AFFF394609F0B4F80146304608F0F4FEBB
:10AC200027490646384608F0F7FF0746E8E71A784E
:10AC300002F0DF02452A35D15A782D2A02D102339B
:10AC4000012704E02B2A14BF013302330027013B04
:10AC500000240A2013F8012F303AD1B2092902D872
:10AC600000FB0424F6E7B4F59A7F28BF4FF49A74EA
:10AC7000A0464FF07E50B8F1070F05D9114908F0F2
:10AC8000CBFFA8F10808F6E704F0070424B10C494B
:10AC900008F0C2FF013CF9E737B10146304609F040
:10ACA0006FF805E04FF07E500146304608F0B4FFE3
:10ACB0000146284608F0B0FFBDE8F081000080BFE3
:10ACC0000000204120BCBE4C30B5002387B00C46AC
:10ACD0000021054600930193029309F059F929498F
:10ACE00018B1284608F090FE02E0284608F08AFED7
:10ACF000254908F091FF09F06BF9054680EAE070FC
:10AD000003A9A0EBE57001F0FBFE002DACBF2023F2
:10AD10002D2303A88DF8003008F0C6F9012807D1CB
:10AD200030238DF801308DF802308DF803300CE0BF
:10AD3000022805D130238DF801308DF8023004E06F
:10AD4000032804BF30238DF8013003A968460EF0B4
:10AD5000C5F8684608F0A8F90338C5B22A4669461E
:10AD600020460EF016F900236355084920460EF0E0
:10AD7000B5F80DEB050120460EF0B0F8204607B0FF
:10AD800030BD00BF6F12033A00007A4441D301087E
:10AD900070B50646B6FBF2F40846154614B12046D7
:10ADA000FFF7F6FF05FB1464024B1B5D00F8013B47
:10ADB00070BD00BFCCC301082DE9F04F81468A4623
:10ADC00016461C4689B000253178002900F0D9804C
:10ADD000252901D001368EE072784FF00008302A24
:10ADE0000CBFB278B71CA2F1300312BF4FF0000BBA
:10ADF000F71C4FF0010B092B19D8A2F13003D9B27F
:10AE0000092905D80A2202FB083817F8012BF4E7B4
:10AE1000A2F16103052B02D8A2F1570305E0A2F1CC
:10AE20004103052B03D8A2F137030A2BEADD6C2A74
:10AE30004BD13A787E1C642A00F094800BD8252AE6
:10AE400058D003D8002A00F09C80BDE7582A0CD0C7
:10AE5000632A34D0B8E7732A3DD002D86E2A52D084
:10AE6000B2E7752A5CD0782AAED1A2F158004242EE
:10AE700004F1040705AB424110212068FFF71AFADC
:10AE80003C460FE043D9582A16D1A2F158014A4254
:10AE900004F104064A41206805AB10213446FFF74F
:10AEA00009FA3E4605AB009342465B46514648468A
:10AEB00007F026FE054487E7632A2AD13E4621781B
:10AEC0004846271DD04701350FE0642A38D00ED9F7
:10AED000732A14D13E46236842460093514600230C
:10AEE000484607F00DFE271D05443C466CE7252A21
:10AEF000C8D13E4625214846D047013564E70AD8E7
:10AF00006E2A06D13E46236804341D605CE7002AA1
:10AF100037D03E4658E7752A07D0782AB5D0F8E7EB
:10AF2000271D05AB00220A21A7E7231D039300225A
:10AF300005AB0A212068FFF7BDF93E46039CB1E747
:10AF40002068231D002803930ADA2D238DF814307E
:10AF500040420DF1150300220A21FFF7ABF9ECE79F
:10AF600005ABF8E72068271D002808DA2D238DF8A7
:10AF7000143040420DF1150300220A217EE705AB93
:10AF8000FAE7284609B0BDE8F08F0FB437B50A4C90
:10AF900006AB53F8042BA16FE06F0193FFF70CFF92
:10AFA0000546206800F0FCFA0028FAD0284603B0D5
:10AFB000BDE8304004B0704718180020026B03460B
:10AFC000C16810B5406942B11A6C8C1A013A08BFC9
:10AFD0000A46005D1A64C0B210BD1A6A805C013274
:10AFE0008A4228BF0022C0B21A6210BD436B13B15F
:10AFF00090F844007047836A406A1B1A58425841CF
:10B000007047426A816A03698A4238BFD218521A6D
:10B01000416B21B149680A44591E8A4203D2013B5F
:10B02000981AC0B2704700207047036B13B159687B
:10B03000036C01E0C169036A994237BFC268C81A4C
:10B040008818C01A7047F0B5056D8279AB8912F087
:10B05000020F23F400534FEA03434FEA1343AB813B
:10B060002B8A08BF00219BB218BF4FF4005123F474
:10B0700040530B43876846792B82A98912F0040F4D
:10B0800014BF4FF4806E4FF0000E89B216F0010F1E
:10B09000044621F4B05114BF04200020B60748BF75
:10B0A00040F0080221F00C0148BF90B24EEA0101C5
:10B0B00040EA0102AA81AB8A87B023F440731B04E3
:10B0C0001B0CAB8201A801F057FE264A039B049E8D
:10B0D000954218BF1E4619227243AB8913F4004FE4
:10B0E00014BF7E00BE00B2FBF6F66427B6FBF7F095
:10B0F000AA8900010109120407FB116307D5D900D1
:10B100003231B1FBF7F202F00702104306E01A01F8
:10B110003232B2FBF7F303F00F031843A37980B286
:10B12000DB07288108D5226D0F4B9A4204D10F4BC3
:10B130000121186802F032FAA379226D13F0080F8A
:10B14000938A0BBF23F008039BB21B0443F0080350
:10B1500008BF1B0C938293899BB243F400539381E5
:10B1600007B0F0BD003801400044004098180020AE
:10B17000417168E7816066E7044B014658681B7AB5
:10B180000BB981F0010102F009BA00BF9818002044
:10B19000836A8169426B1944D160416A8B4229BF3D
:10B1A0000169CB1ACB1A53602ABF00235360836214
:10B1B0004FF0000380F84430136838BF816243F0D9
:10B1C000010313607047436A8269D154436A02697C
:10B1D0000133934228BF00234362436B1BB11B68BA
:10B1E000DB0705D4D4E7026DD36843F08003D36056
:10B1F00070472DE9F0431D46B04B8DB0984288460C
:10B2000017469DF850605FD1AD4BAE4AAE49DA604B
:10B2100003F584721A6203F502725A624FF4807267
:10B220009A61DA61A94AD865DA63A2F54842543ACC
:10B230004E205F619A6519645A6505F019FC20205B
:10B2400005F016FC330709D5192001F099FF0722F4
:10B250008271C271012202721E2119E0AC070BD566
:10B26000192001F08DFF072282710522C27101228F
:10B2700002721A2101F0AAFFE8070BD51A2001F08B
:10B280007FFF072282710622C271012202724A21C7
:10B2900001F09CFF8E4B8F499A6D48698E4C02439A
:10B2A0004A618E4ADC651A6593F8553000228DF8A4
:10B2B000043001A801238DF805308DF806208DF8A3
:10B2C000073005F0F3FBAEE0854B984252D17C4B42
:10B2D0007C4AC3F8B0001A664FF48072DA661A67C7
:10B2E00003F542725A6703F581629A677D4A7120BD
:10B2F0009F66C3F8A820C3F8AC2005F0B9FB202056
:10B3000005F0B6FB310709D5122001F039FF0722FD
:10B310008271C271022202721E2119E0AA070BD5A6
:10B32000122001F02DFF072282710522C271022234
:10B3300002721A2101F04AFFEB070BD5132001F02E
:10B340001FFF072282710622C271022202724A2165
:10B3500001F03CFF26238DF804300022012301A8D0
:10B360008DF805308DF806208DF807305E4C05F01D
:10B370009DFB58E05D4B984240F00181504B514A93
:10B38000C3F80401C3F8B42003F5A162C3F8C820D0
:10B3900003F5C162C3F8CC204FF48072C3F8C0201B
:10B3A000C3F8C420524A7220C3F8BC70C3F8FC2012
:10B3B000C3F8002105F05CFB340709D52A2001F011
:10B3C000DFFE07228271C271032202721E2119E080
:10B3D000A8070BD52A2001F0D3FE0722827105228F
:10B3E000C271032202721A2101F0F0FEE9070BD5A7
:10B3F0002B2001F0C5FE072282710622C2710322B2
:10B4000002724A2101F0E2FE27238DF80430002267
:10B41000012301A88DF805308DF806208DF807303E
:10B4200005F044FB334C4FF00009012384F844300D
:10B43000C4F82090C4F81C90C4F82890C4F8249054
:10B44000C4F82C806571A760A6712046FFF7FBFD4C
:10B45000EA0759D5236B002B4ED001A801F0E8FB79
:10B46000E36C206B01934FF480530A93802306937F
:10B47000E368CDF82C900493202309936369CDF8F9
:10B4800014900293CDF81C90CDF82090CDF80C903C
:10B4900001F0F9FB01A9206B01F0D7FB226B216DB4
:10B4A000136843F0010313608B8A9BB243F040039F
:10B4B0008B8253689BB2236426E000BF00380140B2
:10B4C0009818002010A101084400024058000240D2
:10B4D000A802002000100240A418002095FA0008DD
:10B4E0000044004004440040F81800200048004098
:10B4F000044800404C1900204FF6DF72236D1A807B
:10B50000DA6842F02002DA60AB0730D5636B002BBB
:10B5100028D001A801F08CFBA36C002501934FF407
:10B5200080530A93802306932369606B049310234E
:10B5300003930B95059507950895099501F0A3FBD5
:10B5400001A9606B01F081FB636B1A6842F0020293
:10B550001A60226D5D605D60938A9BB243F0800348
:10B56000938204E0226DD36843F08003D360226DA0
:10B57000204693899BB243F40053938100E000205E
:10B580000DB0BDE8F08303685B6A03B118477047EC
:10B5900003681B6A03B11847704703689B69184723
:10B5A00003685B6918470368DB68184703685B68D2
:10B5B000184703681B68184703682DE9F041DB69E9
:10B5C00004460E46174693B90D467B1B3344002BA9
:10B5D0000BDD236820469B6898470028F9D015F8B2
:10B5E000011B2046FFF7E5FFEFE7BDE8F081BDE86E
:10B5F000F04118471FB50123ADF808300023ADF81E
:10B600000C30ADF80A30094BADF8041093F8083748
:10B6100001A9012B08BF0323ADF8062008BFADF830
:10B620000C30FCF7A5FE05B05DF804FB981800206F
:10B6300070472DE9F04F87B01C46074602910392F0
:10B6400004F07AFEAC4B1B889E0709D53B7F97F828
:10B65000412097F84010208A04F0F1FD019001E0AC
:10B6600064230193BA460024A44B4FEA840853F89C
:10B67000240008F0ADFCA04B19888D0724D0022CC3
:10B6800022D09F4B650033F91420029B52005B428D
:10B690009A4203DB029B9342A8BF1346994AAA5ED3
:10B6A0009A1A039B33F914301344CA0703D5387A26
:10B6B0005843001108E0BA7C5343019A5343642273
:10B6C00093FBF2F300EB23108F4B042258F8031086
:10B6D0009AF8015091FBF2F2811A4D430C3313F8A2
:10B6E00004C064230CFB05F595FBF3F5834BED11CA
:10B6F00093F82BB0BBF1030F0CD9FE8D56B1022C81
:10B700000CD173429D42C0F2F480B5422B46A8BFD3
:10B710003346EEE0022C01D1BB8D00E07B8D00288A
:10B72000B8BF4042800190FBF3F0B0F5807FA8BF26
:10B730004FF4807020EAE0709AF80B30C0F580700A
:10B7400080B2584303126D48B0F82CE000F1300984
:10B7500001FB0EF658F80900F61206FB03066B4BC8
:10B76000B6F5001FA8BF4FF400169E42B8BF1E4694
:10B77000022C48F809604FEA663665D097F8283001
:10B7800009F10C0959F808001BB9081A49F8081002
:10B7900002E0801A49F808204FF6FF734FEA1E1E98
:10B7A000B3FBFEFE5A4B00FB0EF01B7840110B2B37
:10B7B0000CD19AF8153043430CFB03FC64239CFB2B
:10B7C000F3FC544B4FEA2C2C23F814C0B7F820B0EC
:10B7D000BBF1000F27D008F0CBF9FB7F8146012B8E
:10B7E00007D14D4B01461C2000FB043007F086FAC0
:10B7F00016E06BB904F004FE034648484FF00C0E07
:10B800005FFA8BF249460EFB040007F063FB07E08A
:10B81000434B01464FF4F87000FB043007F018FA70
:10B8200048460BF085F89AF815303E4A5843135DA8
:10B8300002F5CD625843642390FBF3F0AB1900127C
:10B84000034422F8143039E07A8C9AB1049204F05F
:10B85000D7FD049A0590D2B22846049208F088F9E0
:10B86000059B0146049A09F5CD6007F033FB08F00B
:10B87000AFFB0546A919214B09B2BBF1030FA3F891
:10B8800094161AD9FB7D1D4ADB00C3F5C873B2F9C3
:10B890001020502BB8BF502382EAE27EAEEBE27E4E
:10B8A0005842CEEB0002914204DB03EB0E028A42C7
:10B8B000A8BF0A46114BA3F8942600200F4B93F81B
:10B8C000A43613B9184A22F81430184B013448F83A
:10B8D000035003F10C02032C03F1180348F8026033
:10B8E00048F803000AF1010A7FF4BEAE07B0BDE8D4
:10B8F000F08F1D4610E700BFF0350020A41F002088
:10B90000B01F0020B81F0020C01F00200000E0FF73
:10B91000EA160020EC160020EC1F0020402000203A
:10B9200064200020CC1F0020342600204C2600205C
:10B930002DE9F04FB24C89B0054694F828001E4618
:10B940000692059108F014F9AE4908F019FA029030
:10B95000284604F0F1FCAC4B1B8899070ED52B7FD1
:10B9600095F8412095F84010308A04F068FC08F002
:10B97000FFF8A44908F004FA039002E04FF07E5368
:10B98000039395F83560002E3AD044F62061E06AC2
:10B99000B4F8CC36B1FBF0F19942994A2DD8B2F9FE
:10B9A0001270B2F9CE36F81A0028D8BFD81B08F0AA
:10B9B000DFF88046304608F0D7F8944908F02CF9B3
:10B9C000414608F029F90021064608F0C3FA30B9CB
:10B9D0008F49304608F0DCFA10B18D4E00E00026A9
:10B9E0004FF07E51304608F00FF88A4BA4F8CE761F
:10B9F00018600023A4F8CC3602E00133A2F8CC365C
:10BA0000A8467F4B00240093834F98F80100E35D24
:10BA1000A7F5DA6783420DD107F2D36398F80B20BC
:10BA2000E35C9A4206D107F2D66398F81520E35CEE
:10BA30009A4264D008F09CF8784908F0EDF8784E06
:10BA400046F8240098F80B0008F092F8754908F0C1
:10BA5000E3F806F10C0949F8240098F8150008F0FD
:10BA600087F8714908F0D8F806F1180949F8240058
:10BA700095F8370008F07CF8624908F081F906F182
:10BA8000240949F8240095F8360008F071F85D495A
:10BA900008F076F901464FF07E5007F0B3FF06F14B
:10BAA000300949F82400288F4FF47A7909FB00F017
:10BAB00008F05EF8824604F0A3FC0146504608F008
:10BAC000ABF8C7F81807688F09FB00F008F050F8CA
:10BAD000814604F095FC0146484608F09DF898F828
:10BAE0000120A6F10C031A5598F80B20A6F10903C2
:10BAF0001A5598F81530063EC7F81C073355404BC9
:10BB0000022C0CBFD3F81867D3F81C67002130460D
:10BB100008F016FA58BB454B4FEA840953F82470D5
:10BB2000009B3946186807F06DFF0021824608F037
:10BB30002FFA002840F03B820AF10041304608F01D
:10BB400009FA78B10021504608F022FA20B13946AE
:10BB5000304607F059FF03E03146384607F052FF00
:10BB6000009B1860009B1A68304B49F80320264B55
:10BB70001F88BA0775D0022C73D02D4B4FEA4409A9
:10BB800033F9140007F0F4FFE96B08F045F8059B62
:10BB90000646584207F0ECFF82460146304608F060
:10BBA000D9F948B9059807F0E3FF824601463046C7
:10BBB00008F0EEF900B9B2461E4B33F9090007F060
:10BBC000D7FF0146504607F01DFF069B064633F996
:10BBD000140007F0CDFF0146304607F015FF164967
:10BBE00008F0CEF8FB07064628D5287A07F0C0FFF4
:10BBF000314608F011F8104908F0C2F82FE000BFF4
:10BC0000A41F00200000C842F03500206F12833AC4
:10BC10000000A0405003002074260020D730033DD0
:10BC200080260020033F7A3E97AC0A3AC4260020C3
:10BC3000B01F0020B81F002000002041A87C07F0A2
:10BC400097FF314607F0E8FF039907F0E5FFA649A3
:10BC500008F096F8009B0146186807F0D5FE009B97
:10BC60001860DFF8C0A2A1495AF8240008F088F84B
:10BC7000009B0146D3F800900490484607F0C2FEAE
:10BC8000AAF1500A5AF82410074607F0C5FF029996
:10BC900007F0C2FF022C01900CBFA88D688D07F041
:10BCA00067FF002182464846A60008F071F910B9E6
:10BCB00009F1004000E04846514608F061F80146AD
:10BCC0004FF07E5007F09EFE0021824608F042F9B8
:10BCD00040B94FF07E51504608F05AF920B14FF06C
:10BCE0007E5A01E04FF0000A814B5046196807F078
:10BCF00093FF804B834656F803A0503BF1583846DB
:10BD000007F08AFF074604F07BFB0146384607F040
:10BD100083FF594607F080FF514607F075FE7649CC
:10BD2000824608F017F938B97449504608F030F9DE
:10BD300020B1DFF8C8A101E0DFF8BCA16D4F022CF3
:10BD400046F807A000F0F080A7F1380356F803B0DA
:10BD500095F83630632B42D80021484608F018F990
:10BD600007F10C0358B19B5948461946079307F051
:10BD700049FE079B0146184608F00AF911E0002128
:10BD80004846079308F0E6F8079B40B39B5948469E
:10BD90001946079307F036FE079B0146184608F040
:10BDA000D9F8E0B107F11803F1582C3FF7590846CC
:10BDB00007F032FF594607F02FFF394607F02CFFF6
:10BDC000394607904FF07E5007F01CFE594607F0A9
:10BDD00023FF079B0146184607F016FE8346484B93
:10BDE000494646F803905846079307F015FF049913
:10BDF00007F008FE079B834603F11807F1590493E7
:10BE000007F000FE46F807B0814604F0F9FA014653
:10BE10004FF07E5007F0B4FF494607F0FDFE394A67
:10BE200007461278049B0B2A0BD1503BF15807F0C0
:10BE3000F3FE029907F0F0FE08F0CAF8324B23F83F
:10BE40001400324890F8643743B11C2300F5ED60CC
:10BE5000394603FB040006F051FF0746B5F8209071
:10BE6000B9F1000F21D0EB7F012B07D1284B1C200B
:10BE7000394600FB043006F041FF15E063B904F0D9
:10BE8000BFFA0346234839460C275FFA89F207FBBD
:10BE9000040007F01FF807E01F4B4FF4F870394615
:10BEA00000FB043006F0D4FE07461C4B3846F15820
:10BEB00007F0B2FE029907F0AFFE0746514601981F
:10BEC00007F0A2FD394607F09FFD0AF031FD2A8EEA
:10BED0005342984203DB90420346A8BF1346104AE0
:10BEE00022F814303AE000BF000020413333834190
:10BEF00050030020DC26002000007AC300007A43B3
:10BF0000E8260020EA160020EC160020A41F0020DE
:10BF1000EC1F0020402000206420002098260020F4
:10BF200034260020D0260020B5F82290B9F1000F69
:10BF30000AD004F065FA5FFA89F203460199A7F185
:10BF4000A00006F0C7FF01905146019807F05CFD84
:10BF50000AF0EEFC1A4B0027A3F89406184B93F84E
:10BF6000A4261AB903F5D26323F81420019808F027
:10BF70002FF8DFF85090013449F80600504608F0D9
:10BF800027F809F10C0B4BF80600384608F020F8AA
:10BF9000009B09F118090433032C49F8060008F145
:10BFA000010800937FF430AD09B0BDE8F08F514631
:10BFB000304607F0CFFF00287FF4C9ADD2E500BFBF
:10BFC000A41F00204C26002010B504460B4B014650
:10BFD0001868FFF7EEFA0A4B0822188880EA042056
:10BFE00010F4004F4FEA40001CBF80F4815080F0F5
:10BFF0000100013A80B2F3D1188010BDD435002081
:10C00000DC35002010B5064C2068FFF7CFFA002879
:10C01000FAD0034BBDE810401868FFF7C4BA00BF60
:10C02000D435002008B5FFF7EDFF0A4A0821138830
:10C0300083EA00239BB213F4004F4FEA43031CBF73
:10C0400083F4815383F0010301399BB2F3D1138050
:10C0500008BD00BFD835002010B504462046FFF7C4
:10C060009FFA18B90A2004F097FCF7E710BD0023E7
:10C07000F0B51C460A490B4D91F8BC27FF265F57C7
:10C08000874204BF5E5502F1FF3203F10C0304BF87
:10C09000D2B201243C2BF2D10CB181F8BC27F0BD07
:10C0A000A41F0020B040002030B5084C00230C2114
:10C0B00001FB03425568A84203D00133052BF7D199
:10C0C00030BD0023C3621381536030BDB0400020F7
:10C0D0002DE9F341054688469DF820701146234816
:10C0E0001A469DF8243000264FF00C0C0CFB06F489
:10C0F00004EB000E2456AC4203D00136052EF5D1D8
:10C1000002E0BEF8080008B100202BE0022D11D09B
:10C1100006DC5DB1012DF7D1009315483B460CE0DC
:10C120001E2D0ED01F2DEFD101200AE000931148E3
:10C130003B4602E000933B460F48FFF75AF804469F
:10C1400005E0F9F715F839460446FFF726FA002C02
:10C15000DAD02046054A0C2303FB06262571A6F8F3
:10C160000880746002B0BDE8F08100BFB0400020DC
:10C1700000440040003801400048004010B5084B22
:10C180000022196801EBC20393F90240844201D1F5
:10C19000981C10BD0132052AF4D1002010BD00BF4B
:10C1A000AC40002038B1438813EA010003D08B4231
:10C1B0000CBF01200220704770B50D4B0D491D6862
:10C1C00091F8BD270024042A0DD8134605EBC303BC
:10C1D0009E88541C3042E2B24FF00104F3D081F843
:10C1E000BD27981C70BD0CB181F8BD27002070BD23
:10C1F000AC400020A41F0020024B002283F8BD2782
:10C20000DAE700BFA41F00202DE9F74F264B274A8D
:10C210001B68126890F803E0C3F3007313421FFA1F
:10C220008EF303EB8307C3F1000290F80480C3F19F
:10C230007803CEF1640C9BB208BF0E881C4D18BF6A
:10C240004FF47A765FFA8CFC7F00C8F1640B92B2EF
:10C2500001934FF00A0A4FF47A7913B2002B02DCF3
:10C2600003D1012402E0644600E0744603FB03F0BE
:10C27000644308FB00F090FBF4F45C44634393FBDD
:10C28000FAF33B441BB225F8023F48880A32801B70
:10C29000434393FBF9F333442B80019B92B29342C7
:10C2A000DBD103B0BDE8F08FF43500205417002037
:10C2B000602700200A7849788A421CD20F4B04304C
:10C2C00033F91000B0F5617F05DB40F63303984287
:10C2D000A8BF184601E04FF4617019235A4302F2D7
:10C2E0008332904207DD4B4303F283339842CCBF45
:10C2F0000020012070470020704700BF5817002021
:10C300000C4B1B6813F4805F0B4BB3F9063009D05C
:10C310000A4A1268D20005D4008A421A934207DD05
:10C32000084400E0408A8342B4BF002001207047E7
:10C33000012070475417002058170020F4350020C2
:10C3400038B50D4B05461B680C461B0313D50B4B2C
:10C3500093F8D637093B012B0DD8452006F06AF932
:10C360000D2006F067F9284606F064F92046BDE87E
:10C37000384006F029BA38BD54170020A41F002009
:10C38000044B1B681B015DBF034B1868C0F3805052
:10C3900001207047F43500205417002010B500200C
:10C3A000FEF7EAFE074B00241C70FCF789FB064BE6
:10C3B00083F8D747C3F8D847A3F8DC47C3F8E0476A
:10C3C00010BD00BFAC170020A41F002030B470B116
:10C3D000194BD3F85C3513F400330BD0174B1B68A3
:10C3E00013F0020306D0164B1B78012B01D830BC8A
:10C3F000D4E70023134A0C2505FB03F18C18895C54
:10C40000814203D00133142BF6D112E00E4AD2F848
:10C41000E01719B16078497888420AD209490C209E
:10C4200000FB0313C2F8E0370023A2F8DC37C2F8A0
:10C43000D83730BC704700BF303B00205417002075
:10C4400064030020D0950108A41F00204000142898
:10C45000094A30B4A8BF14200023022514249D5497
:10C4600002339918984201F8014CF8DC024AFF2186
:10C47000D1540F2030BCA9E70C14002010B504469D
:10C48000FAF744FD164B174A9A1A237903F00F0363
:10C49000052B22D8DFE803F003060A0D11170378F5
:10C4A000805C0CE090F90030805608E00388805AE8
:10C4B00005E0B0F90030805E01E0036880581B1A87
:10C4C0005842584110BD815800684FF0010407F0F0
:10C4D00037FD00B90446E0B210BD002010BD00BF1A
:10C4E00088270020303B00202DE9F04FB74C4FF05B
:10C4F000000989B0494605469346C4F87895182244
:10C50000C4F87C95C4F8809504F2845098469DF850
:10C5100048600CF0BBFCAE4B94F89C751822012FC0
:10C520008CBF1F465F1E4946A4F89D9504F5B46074
:10C530000CF0ACFC2320C4F8B87504F02DFA0DF112
:10C5400015020121752003F04DF8B8B1A14B0DF192
:10C550001602C4F8A435A04B0121C4F8A8354846FA
:10C56000432384F8A03503F03DF89DF8163003F01E
:10C570007E038DF8163000283FD147E094F8BC7553
:10C580000FBB2C2000F0FCFD142282710E22C27120
:10C5900007721321C4F8C00500F018FE8F4A1388F3
:10C5A00023F040031B041B0C1380138823F0380373
:10C5B0001B041B0C138013889BB243F040031380B1
:10C5C000012384F8BC3506AA01217520FCF7C0FAC6
:10C5D0009DF81830A3F17002012A01D9AF2B5ED16A
:10C5E000052384F89D35432384F8A0357C4BC4F89B
:10C5F000A4357C4BC4F8A83551E0682B06D1012343
:10C6000084F89D351D2384F8A03548E09DF8153049
:10C6100003F07E03682B8DF815303BD102230621F1
:10C6200084F89D3506AAD4F8A435084698479DF8A5
:10C630001D209DF81B3092005B0003F0020302F006
:10C6400004021A439DF8193003F00103134311D07B
:10C65000012B01D1002302E0022B03D1012384F836
:10C660009E351CE003F00303032BF7D0032004F0F6
:10C670009DF914E0554B0DF11702D3F8A4350121B3
:10C680000C2098479DF8173013F00F03EED0042BC1
:10C69000E4D1DFE7702B04BF042384F89D3594F8C0
:10C6A0009D250020022A494B84F8C4050FD14E492C
:10C6B000C3F884154D49C3F888154D49C3F8901542
:10C6C0004C49C3F89415012183F8C41528E0012AC8
:10C6D00012D1494983F8C425C3F88415434904227B
:10C6E000C3F888154549C3F88C154149C3F890151E
:10C6F0004049C3F8941513E0043A012A00F29881E6
:10C700003F4AC3F88425394AC3F88825384AC3F814
:10C710009025384AC3F89425012283F8C4250722BE
:10C72000384BD4F8C8751A7047F001020393C4F867
:10C73000C825002384F8C535082D00F2B880DFE84D
:10C7400005F00BB60B2D6B8B2DA4A400012D40F230
:10C75000B880002583F8C55594F89C35DFF86C90B7
:10C76000012B1BD84FF0000A08AB03F808AD0122DB
:10C770005146532004F004FA80B19DF81830E52B9F
:10C780000CD1214B89F8C6A5C9F878351F4BC9F8DB
:10C790007C35042384F8C53502238CE094F89D256C
:10C7A0000A4B022A38D11A4AC3F87825194AC3F825
:10C7B0007C2593F89E35002B14BF6E236F2384F8DD
:10C7C0008235012384F8C535032374E088270020CF
:10C7D00039A10108E5F5000869F5000800380040B6
:10C7E000518B0008818B000809FA000885F40008C5
:10C7F0006DF4000890C1793D21F5000839F4000876
:10C8000021F900085403002093F5000891F6000870
:10C810006DFA0008CDF4000894F89C35012B1BD864
:10C82000002208AB03F8082D0D2101221C2004F082
:10C83000A7F988B19DF818302A2B01D01A2B0BD1FB
:10C840007D4B0222C4F878357C4BC4F87C357C4B98
:10C8500083F8C52504232EE0002108AB03F8081D4A
:10C860000122182004F08CF978B19DF81830FB2BC8
:10C870000BD1744B0122C4F87835734BC4F87C3566
:10C880006F4B83F8C525052315E094F89D256C4B67
:10C89000043A012A3FF65AAF6C4AC3F878256C4A2D
:10C8A000C3F87C25012283F8C525082303E0012D68
:10C8B00007D900253EE7039A47F003075370C4F8F1
:10C8C000C875D4F8C8355E489A0708D54FF4807308
:10C8D000A0F88035D0F8783500F5AF609847B8F10A
:10C8E000000F07D0B8F1070F16BF4FF47A737D23FE
:10C8F000012600E07D23721E5E4384F8CC25C4F837
:10C900009865D4F884354046984794F8CD754C4DD9
:10C910002FB9B4F8CE85B8F1000F3BD12FE0D5F890
:10C920009835002BF5D0002605F22C6894F8D03508
:10C93000012B0CD1384607F017F9464B01461C2055
:10C94000D5F8982500FB063006F090FA13E04BB9B5
:10C95000D5F8980507F008F93F4907F05DF9C5F8E3
:10C96000280608E04FF4F870B5F89825394600FB22
:10C97000068006F09FF90136032ED7D1C9E7304B68
:10C98000B3F8FC3B33B9354B93F8C5214AB384F86F
:10C99000C42526E0D4F89835002BF4D0304F00257C
:10C9A000012607F15809404607F0DEF800960146D7
:10C9B000D4F8003CD4F89825781906F0CBF9B4F8EF
:10C9C000FC0B07F0D1F800960146D4F8583C09EB6F
:10C9D0000500D4F898251C3506F0BCF9542DE2D199
:10C9E000D1E793F8C6310BB184F8C535D4F8C83512
:10C9F000134D1B0718D564209BFBF0F400FB14B00B
:10CA000000B207F0B5F8174907F006F906462046C8
:10CA100007F0AEF80146304606F0F6FF124907F07F
:10CA2000FBF8C5F8B00C02E00023C5F8B03C0120CB
:10CA300009B0BDE8F08F00BF59F70008F1F5000814
:10CA40008827002073F500084BF60008F9F9000864
:10CA5000CDF400085C2D0020BD378635303B00202A
:10CA60008C3300208988883C00002041002101206F
:10CA700002F0D8B8F8B50F46204C1D25064684F8BC
:10CA8000B45CFDF729FB002001F06AF8082001F0F2
:10CA900067F80E2001F064F8284601F061F80420E0
:10CAA00001F05EF8042001F05BF8002001F058F876
:10CAB000302001F055F8002001F052F8384601F01E
:10CAC0004FF8002001F04CF8FDF7EEFA04F6B540FF
:10CAD000FDF758FA224678B194F8B53C5BB994F862
:10CAE000B63C302B00D033B992F8B73C1BB9034B9E
:10CAF00093F8B83C33700120F8BD00BF88270020B0
:10CB0000031EB8BF2D2210B5B8BF58420C46AEBFA9
:10CB10000A2201F8012B0A22FEF73AF900230370DA
:10CB2000204610BD2DE9F84381460F461D4B1E4E91
:10CB30000025F61ADFF87C8008EB0504237903F062
:10CB400030034B4527D12046FFF798FC55F8088065
:10CB500001464346154A384602F034FC50B120469F
:10CB6000FAF7D4F900228119204602F081FA104820
:10CB7000F9F7BAFC2046FFF781FC434601460B4A11
:10CB8000384602F03FFC30B12046002102F0D2FAD4
:10CB90000748F9F7A9FC1435B5F5436FCAD1BDE8CC
:10CBA000F88300BF303B002088270020F1C3010834
:10CBB000F3BB01083CA10108012810B50C4613D8AD
:10CBC00000F022FE0948F9F78FFC0948F9F776FBD7
:10CBD0000848F9F789FC21461020FFF7A3FFBDE8BC
:10CBE00010400348F9F750BB10BD00BFFBC301085C
:10CBF0003FB20108F3BB0108022810B50C460FD85C
:10CC000000F03AFD0748F9F76FFC0748F9F73CFBDD
:10CC10000648F9F769FC2146BDE81040202081E76D
:10CC200010BD00BF09C401083FB20108F3BB0108F1
:10CC30000023036043608360C360036143618361D9
:10CC4000C36103624362836270470A6A10B58C68ED
:10CC5000036814430A6923F4FF4314434A6923F029
:10CC6000700314438A691443CA6914434A6A14431B
:10CC70008A6A224313430360CB6843600B68836076
:10CC80004B68C36010BD4FF6FE730268134003602B
:10CC90000023036043608360C360294B984201D145
:10CCA000284A27E0284B984201D1264A2AE0274B00
:10CCB000984201D1234A2DE0254B984201D1214AC7
:10CCC00030E0244B984201D11E4A33E0224B984277
:10CCD00004D11C4A536843F470032EE01F4B984262
:10CCE00004D1184A536843F0706326E01C4B984205
:10CCF00004D11C4A536843F00F031EE01A4B9842BC
:10CD000004D1184A536843F0F00316E0174B9842D9
:10CD100004D1144A536843F470630EE0144B9842F4
:10CD200004D1104A536843F4704306E0114B984213
:10CD300004D10C4A536843F470235360704700BF1A
:10CD400008000240000002401C0002403000024087
:10CD500044000240580002406C0002408000024043
:10CD600008040240000402401C0402403004024057
:10CD70004404024058040240224A10B5536803F0AC
:10CD80000C03042B03D0082B04D01F4B14E01F4BC3
:10CD90005B6811E053685168C3F38343C90303F12F
:10CDA000020301D41A4906E0516811F4003F174903
:10CDB000496818BF49084B4303605368154CC3F3D7
:10CDC0000313234493F8341C0368CB404360516839
:10CDD000C1F30221214491F8341C23FA01F181604E
:10CDE0005168C1F3C221214491F8341CCB40C36087
:10CDF0005268C2F38132224492F8442CB3FBF2F31E
:10CE0000036110BD0010024000127A00540300209C
:10CE100000093D0038A1010810B50446FBF794FA5B
:10CE2000012806D11CB1FBF78FFA013CF8E7052079
:10CE300010BD002C08BF052010BD00BF10F80A3C33
:10CE40000133DBB20A2B00F80A3C07D910F8131C97
:10CE5000034A002322F8113000F80A3C704700BF53
:10CE60002415002070B5524B14241A78DD68013265
:10CE7000B2FBF4F004FB102298681A705A6C8142DD
:10CE80000A4404D293F84C0008B102F580324948B4
:10CE90000078B2FBF0F295420AD293F84C401CB1F4
:10CEA0004FF4803494FBF0F4501B041B1C6106E02B
:10CEB0004FF4803494FBF0F0401B104418619960EB
:10CEC00093F8501000240131DA60142283F84C40AA
:10CED00091FBF2F402FB141183F8501093F85110F7
:10CEE0001C69013191FBF2F502FB151283F8512008
:10CEF00040F68C2294422E483DD9027990F949108F
:10CF000014468A420CD1111F082909D890F84A10FA
:10CF100018299ABF013180F84A1080F8482002E0B1
:10CF2000002183F84A1093F94800214982421AD11E
:10CF300091F84B00B8B1204D10310020904205DA35
:10CF400051F8046F25F810600130F7E71A49002006
:10CF50000C2C03D021F814000134F9E793F8521097
:10CF6000013183F8521083F84920002201211A71FF
:10CF700083F84B1070BD90F84B20C2B140F2DA52EA
:10CF8000A4F2EF21914208D802790B2A05D800EBD0
:10CF90008203013202715C6170BD002283F84B2074
:10CFA000064B03F1300143F8042F8B42FBD170BDD7
:10CFB000503400205C030020241500206034002041
:10CFC00010B50A4B14241A780132B2FBF4F004FBBA
:10CFD00010221A705A6C01320A445A644FF6FF72DA
:10CFE000914204BF012283F84C2010BD5034002030
:10CFF000024B53F820301B681980704754390020C9
:10D00000074BA1F57A7153F820301A681B895943F0
:10D010004FF47A7391FBF3F189B21180704700BF2E
:10D020005439002038B510F80E2C044650F8043C52
:10D030005AB9012200F80E2C20F80C1C59791868F6
:10D040000222BDE83840FEF7D5BA30F80C2C20F8A3
:10D050000A1C891A89B220F8081C084A10F80F0C1B
:10D06000002522F8101004F80E5C2A465979186839
:10D07000FEF7C0FA04F8065C38BD00BF2415002096
:10D08000094B10B553F82030A1F57A701C6806F0F2
:10D090006FFD064906F0C0FD054906F0B5FC09F034
:10D0A00047FC80B2208010BD54390020EC51B83FBD
:10D0B0000000B443084B10B553F820301820484303
:10D0C0001C6806F055FD054906F05AFE09F030FCD3
:10D0D00080B2208010BD00BF543900200000C04144
:10D0E000084B10B553F82030C8001C6806F040FD0E
:10D0F0004FF0785106F090FD09F01AFC80B22080C4
:10D1000010BD00BF543900200D4A2DE9F0411546ED
:10D1100014685369DFF82C801C40012774B1B4FAFD
:10D1200084F3C3F11F0307FA03F608EB8303586D7A
:10D1300024EA0604036898476E61EFE7BDE8F081D2
:10D140000004014050340020054B03EB8003D3F86A
:10D1500094301BB107289CBF1B681980704700BF23
:10D1600050340020054B53F8202032B193881268C8
:10D17000D1680B4218BF1B041361704780AD0108D2
:10D1800038B50409013C022C00F00F0217DC0D4DEC
:10D1900005EB4403998941FA02F313F001000FD023
:10D1A000012303FA02F00138084006F0A7FF2C44DF
:10D1B000A37C054A03440C2000FB032038BD00205B
:10D1C00038BD00BF80AD0108283600202DE9F041B0
:10D1D0000C46074600285AD003682E4A03F1404304
:10D1E000A3F5843302EB9323587D03F041FCE20660
:10D1F000BD8804F00C0104F07C0644BF04F0030475
:10D20000214315F0FF0F3B681ED01A6800204FF035
:10D21000010E4FF00F0C0EFA00F737EA05040FD19C
:10D2200084000CFA04F822EA080201FA04F4282E19
:10D2300042EA040201D15F6102E0482E08BF1F618B
:10D2400001300828E7D11A60FF2D20D95A68002044
:10D250004FF0010E4FF00F0C00F108040EFA04F429
:10D2600034EA05070FD187000CFA07F822EA080212
:10D2700001FA07F7282E42EA070201D15C6102E0B9
:10D28000482E08BF1C6101300828E5D15A60BDE86E
:10D29000F08100BF80AD01082DE9F0471746054633
:10D2A000DFF8E0920A4699F8B440394604F1010AE1
:10D2B0005FFA8AFA006889F8B4A01E4603F0B0FA53
:10D2C0002879FFF75DFF03228271022280F808A00F
:10D2D000C2711A21FFF77AFF95F807E06B790EF01B
:10D2E0000401002909F1B80848464FEA04140BBFAD
:10D2F0004FF000094FF00409012100211EF0020F38
:10D30000A0442A6814BF4FF0000A4FF0020A0C2B09
:10D3100000F2FB80DFE813F00D00F900F900F900DE
:10D320005100F900F900F9008A00F900F900F9004C
:10D33000C300138C23F001031B041B0C1384138CF8
:10D34000B2F804C09BB2B2F818E023F0020319430C
:10D350002EF0730E8A4B4FEA0E4E4FEA1E4E9A4243
:10D360001FFA8CFC4EF0700E4AEA01010FD003F553
:10D3700000639A420BD003F540639A4207D003F54D
:10D3800080639A4203D003F580639A4207D121F06B
:10D390000C012CF4407C41EA09014CF4807CA2F899
:10D3A00004C0A2F818E096861184138B23F00803BA
:10D3B0001B041B0C43F0080336E0138C23F010030E
:10D3C0001B041B0C1384B2F820C0B2F804E01FFA4F
:10D3D0008CFC138B2CF0200C4CEA011123F4E64357
:10D3E000DFF89CC11B041B0C62451FFA8EFE43F440
:10D3F000E04341EA0A1103D00CF5006C624507D105
:10D4000021F0C0012EF4406E41EA09114EF4806E05
:10D41000A2F804E0138316871184138B23F40063AE
:10D420001B041B0C43F4006313836EE0138C23F482
:10D4300080731B041B0C1384138CB2F804C09BB2C2
:10D44000B2F81CE023F4007343EA01212EF0730EBE
:10D450004B4B4FEA0E4E4FEA1E4E9A421FFA8CFC7F
:10D460004EF0700E41EA0A2103D003F500639A42A0
:10D4700007D121F440612CF4405C41EA09214CF4CD
:10D48000805CA2F804C0A2F81CE096871184938BFC
:10D4900023F008031B041B0C43F0080334E0138C37
:10D4A00023F480531B041B0C1384138CB2F804C0A8
:10D4B0009BB2B2F81CE023F4005343EA01312EF48E
:10D4C000E64E2F4B4FEA0E4E4FEA1E4E9A421FFA7F
:10D4D0008CFC4EF4E04E41EA0A3103D003F50063C0
:10D4E0009A4203D12CF4804C4CF4804CA2F804C036
:10D4F000A2F81CE0A2F840601184938B23F400632F
:10D500001B041B0C43F400639383EB79DB0708D502
:10D51000B2F844306FEA43436FEA53439BB2A2F838
:10D52000443013889BB243F0010313806B790C2BBA
:10D5300019D8DFE803F0071818180B1818180F1877
:10D5400018181300031902F134010AE0031902F15B
:10D55000380106E0031902F13C0102E0031902F16F
:10D560004001C3F8B8100444D4F8B830C4F8BC2063
:10D570000022A4F8C07040461A80BDE8F08700BFC2
:10D58000002C01405034002010B1036882885A6199
:10D59000704710B1036882881A61704738B1838878
:10D5A0000029026814BF002110218B4013617047CD
:10D5B000024B81F0010153F82000EFE780AD010834
:10D5C00030B1036882889B681A4214BF0120002092
:10D5D000704728B18088B0FA80F0C0F11F00704712
:10D5E0004FF0FF3070478FE58EE58DE58CE58BE5DC
:10D5F0008AE589E510B5427A044632B1036800F144
:10D600000A01406898470023637210BD10B4447A41
:10D61000631CDBB204444372A172027A9A4201D8BD
:10D6200010BCE7E710BC7047064B10B51A881C46C3
:10D6300022EA00008242188002D00120FEF706FF95
:10D64000208810BDF0350020064B10B51A881C4606
:10D6500010438242188002D00120FEF7F7FE208896
:10D6600010BD00BFF0350020024A936823EA000095
:10D6700090607047303B0020032888BF02200B4990
:10D680000B4B91F8AC2418706C235343CA1882F8E2
:10D6900018040C2202FB0030064B084400F21A402A
:10D6A000CC31C3F87801FEF7AFBD00BF303B00209E
:10D6B000CF370020503400202DE9F347FBF7B6F9AF
:10D6C0004C4A922313704FF4AF635380BE231371FF
:10D6D000EF2382F8643500231946164682F8653533
:10D6E000F25C0133B3F5AF6F81EA0201F8D1414B2F
:10D6F000414C83F86515414BDFF80891636003F1F5
:10D700008833636004270020013F17F0FF075ED0D5
:10D7100034233B4DE36005F17848A8F5FC38C8F3A5
:10D72000090353B100234FF4005056F808800193C9
:10D73000FFF772FB0428E7D11BE04FF43020FFF71E
:10D740006BFB0428E0D123694FF4302043F002033F
:10D7500023616561236943F040032361FFF75CFBAC
:10D7600041F6FD732269042803EA02032361D9D03C
:10D77000CAE723694FF4005043F0010323611FFA05
:10D7800088F32B80FFF748FB0428DFF86CA013D147
:10D79000AB1C0193019B4FEA1848A3F800804FF49B
:10D7A0000050FFF739FB41F6FE732269042803EAB3
:10D7B0000203236108D0A7E741F6FE73DAF81020D0
:10D7C0001340CAF810309FE704354D45A3D10A4AEB
:10D7D0000428136943F08003136102D1FCF7BAFDFA
:10D7E00010B9052003F0E2F8FBF70CF902B0BDE830
:10D7F000F08700BF303B0020002002402301674536
:10D8000000F8010878FD010810B50446064B83F8BE
:10D81000AC04FFF751FFFCF7BFFD601CC0B2BDE8D0
:10D820001040FEF713BE00BF303B002008B5FFF7E5
:10D8300043FFFCF7B1FDBDE808400120FEF706BE3E
:10D8400010B50C4908220B8880EA030414F0010F7C
:10D850004FEA530318BF83F4204302F1FF3214BF91
:10D8600083F001039BB212F0FF024FEA5000EBD1AC
:10D870000B8010BDCC350020F8B5800040F48064EA
:10D8800003F04CF805460C4E0C4F44F001043B7875
:10D8900056F82300E30702D5FFF77BFE01E0FFF710
:10D8A00073FE640805F1340504D003F037F88542AF
:10D8B000FBD8ECE7F8BD00BFDC170020D81700202C
:10D8C0002DE9F041164F174D3B780C4606461221C4
:10D8D00055F82300FFF77AFC134BA8461D46013C80
:10D8E000E4B2002201341A705A7034443078FFF7E1
:10D8F000C3FF16F8010BFFF7A3FFA642F6D1AB78E2
:10D90000094C2BB12078FFF7B7FF6078FFF7B4FF21
:10D910003B784A2158F82300BDE8F041FFF756BC98
:10D92000D8170020DC170020CC350020234B2DE930
:10D93000F04707461C461D68214EDFF888A00235D7
:10D940009AF80030DFF8788056F82300FFF738FEA9
:10D95000DFF8709028B123689D42F1D80020BDE81F
:10D96000F08702F0DBFF00F11B0602F0D7FF8642D2
:10D97000FBD800252C464FF0010A99F8003058F8E2
:10D980002300FFF71DFE18B10AFA05F31C43A4B2E9
:10D99000092D06F1340605D002F0C0FF8642FBD8FF
:10D9A0000135EAE740F201232340B3F5007FD5D1EA
:10D9B00064083C700120BDE8F08700BF8417002098
:10D9C000DC170020D817002037B5044602ADFF232E
:10D9D00005F8013D2846FFF7A9FF10B90CB1013C3D
:10D9E000F8E79DF8070003B030BD73B5FE238DF84E
:10D9F000043000238DF805308DF806300B7806468C
:10DA00000C4615468DF8073013B901238DF8063002
:10DA100004210DEB0100FFF753FF0220FFF7D4FFB5
:10DA2000FF281CD121786068FFF74AFF2820FFF704
:10DA3000CBFFA0F130025042504188B101230221B6
:10DA400001A88DF805308DF80460FFF739FF2846EE
:10DA5000FFF7BAFFA0F130035842584100E0002020
:10DA600002B070BD07B50368114A23F07F4323F06D
:10DA7000FF03934218D0FF238DF8043000238DF864
:10DA80000530437804218DF8063083780DEB0100D2
:10DA90008DF80730FFF714FF0220FFF795FFA0F184
:10DAA00030035842584100E0012003B05DF804FB08
:10DAB00000FFFF001E4B73B506461C4601390022CD
:10DAC000CDB21A705A709A71DA710135FF228DF851
:10DAD000072005443046FFF729FF08B316F8010B6D
:10DAE000FFF7AEFEAE42F5D1A378114DA3B1A81D4C
:10DAF000FFF71CFFA0B1E81DFFF718FF80B10DF183
:10DB00000700FFF713FF58B12A88EB889A4207D025
:10DB1000C2238DF8073003E00DF10700FFF706FF81
:10DB20009DF80700A0F130035842584102B070BD83
:10DB3000CC35002037B5054608460C46FFF792FF66
:10DB400060B12378022101A88DF804508DF80530CA
:10DB5000FFF7B6FE21786068FFF7ACFF03B030BD79
:10DB6000F8B507461D4A1E4C13781E4D43401370EE
:10DB700008262B7854F82300FB070BD5FFF709FD87
:10DB8000402002F0E7FE2B7854F82300FFF7FCFC5E
:10DB900040201AE0FFF7FDFC202002F0DBFE2B788E
:10DBA00054F82300FFF7F0FC202002F0D3FE2B787E
:10DBB00054F82300FFF7EDFC202002F0CBFE2B7879
:10DBC00054F82300FFF7E0FC2020013E02F0C2FEE3
:10DBD00016F0FF064FEA5707CBD1F8BD1618002004
:10DBE000DC170020D81700202DE9F04FC24DD1B02E
:10DBF000A860FEF7D3FB4FF000090DF1400A85F84D
:10DC00000C9085F80D90FEF70DFA2F284FF00004C8
:10DC1000F5D101212046FFF7CBFCADF80840FEF717
:10DC200001FA8346FEF7FEF98DF81500FEF7FAF9C2
:10DC30008DF81600FEF7F6F90646FEF7F3F90AF836
:10DC400004000134E3B29E42F7D1FEF7DBF98DF810
:10DC50000D00FEF7D7F98DF80C00BDF80C80AB89EC
:10DC60000121984514BF4FF003084FF00008084603
:10DC7000FFF79EFCB8F1000F40F09181ABF130034B
:10DC8000CDF818A00F2B00F28281DFE813F012000C
:10DC9000360076013A0010004C0080016D008E00C5
:10DCA000BE00E0001F018001FE004B014400012680
:10DCB00076E1AB78002B00F072818F4B9B7B002BC1
:10DCC00000F0C281022B02D9032B10D0BCE1FD234E
:10DCD00002210AA88DF828308DF82990FFF7F0FD71
:10DCE0000120FFF771FEC12800F05981ACE1FCF77B
:10DCF00017FA002800F0A88151E16A238DF8083056
:10DD00004DE190238DF8083004238DF8093000266A
:10DD100002AC022746E19AF800305A1E022A00F2AD
:10DD20003081AB733BE19AF80030E97B724A99424B
:10DD300005D8002602AC01274FF0080832E16F49F0
:10DD40000B70937B013B012B09D8012302210AA808
:10DD50008DF828908DF829909370FFF7B1FD85F824
:10DD6000029085F803901AE19AF80030EA7B85F872
:10DD700002909A4285F80390DBD9604A5E4C13709A
:10DD80000326FCF7CDF9002800F0758101215C48DD
:10DD9000FEF770FE002800F06E8102215948FEF760
:10DDA00069FE002800F0678156E1AB7B032B40F051
:10DDB000EE80554B12241C70FCF78EF90020FFF703
:10DDC000CFFE0720FFF7CCFE0E20FFF7C9FE20464E
:10DDD000FFF7C6FE1420FFF7C3FE0020FFF7C0FECA
:10DDE000AC20FFF7BDFE8820FFF7BAFE1320FFF737
:10DDF000B7FE7620FFF7B4FEFCF756F94348FCF770
:10DE0000C1F8002840F0CB8022E1AB7B012B40F031
:10DE1000BE809AF8003005A88DF808305B008DF8B8
:10DE200015308DF81690FFF71DFE002800F01081C8
:10DE3000374B02211B880AA8ADF82830FFF740FDB8
:10DE40001420FFF7C1FD302800F0A98000E19AF806
:10DE500000308DF81430AB7B002B00F09E80022B3D
:10DE600002D9032B05D098E005A90CBF0720032099
:10DE700017E005A8FCF7E8F9002800F0E980224B3C
:10DE800014221A700DEB02001DE09AF800308DF894
:10DE90001430AB7B022B02D0032B0AD07DE005A906
:10DEA0000420FFF747FE002840F058814FF00F088C
:10DEB00075E005A8FCF7C8F9002800F0C980124BEE
:10DEC00016221A7005A8FCF799F9ECE7AB7B8DF8E0
:10DED0001460002B63D0022B02D9032B1AD05EE012
:10DEE00005A8FFF7BFFD002800F0B28014220DEB5B
:10DEF0000201012032E000BFCC350020D8170020FD
:10DF0000CF350020CE3500203C3400203D340020A9
:10DF10009DAD010805A8FCF797F9002800F098804E
:10DF2000132224E0AB7B8DF81460022B0DD0032B61
:10DF300017D0012B4FF0000602AC4FF001070CBFC9
:10DF40004FF002084FF00F082CE005A8FFF78AFDFC
:10DF500000287DD040F2DC5205A90520FFF745FDE1
:10DF60004FE705A8FCF770F9002871D015227E4B09
:10DF700005A81A70FCF7F0F843E700267B4C092748
:10DF800010E0002602AC01274FF009080AE0002645
:10DF900002AC01274FF0020804E04FF0020800260F
:10DFA00002AC01270021084685F8109085F81190F1
:10DFB000FFF7FEFAA868FDF7EBFA2E20FEF704F84B
:10DFC0005846FEF701F89DF81500FDF7FDFF9DF896
:10DFD0001600FDF7F9FF3846FDF7F6FF013FFFB2E7
:10DFE0000137274414F8010BFDF7EEFFBC42F9D1CD
:10DFF0004046FDF7E9FF697CA868FDF7DAFA297C5D
:10E00000A868FDF7D6FAA868FDF7BDFA002101203F
:10E01000FFF7CEFA002E3FF4F2AD554F554EEC7B94
:10E0200064B1013CE4B256F824001A21FC73FFF7F6
:10E03000CDF856F82400FFF7A7FAF0E74E4B01227F
:10E040001A7051B0BDE8F08F85F8029085F8039002
:10E05000002602AC01277EE049F20732638823F0F4
:10E060000801914275D049F20A32934271D049F2C7
:10E070000B4293426DD0414A04AF93781188BB7034
:10E080003980131D0DF1280E1432F44618685968B2
:10E090000833ACE803009342E646F6D118681B79D2
:10E0A000CCF8000015210AA88CF80430FFF708FC12
:10E0B00007AA082110460192FFF7FCFC48B9013E6F
:10E0C00016F0FF067FF45DAEAE70EE702C4C0427A8
:10E0D00041E0019A0023D05CF95C8842EFD1013322
:10E0E000032BF8D1D3782B711379EB7053794FF25E
:10E0F0001032AB70638823F02001914211D04FF2AF
:10E10000104293420DD04FF29032934209D04FF615
:10E110005002934205D003F5BA520F3292B2012A4F
:10E1200001D801230EE049F2073123F008028A42A8
:10E1300007D049F20A32934203D049F20B4293428C
:10E14000BDD10223AB73AB7B00266B710C4C042753
:10E1500028E70323F6E74FF00F0823E79DF8147034
:10E16000002654461EE700BF3C3400206ECD010857
:10E17000CC350020DC1700205D0300209FAD010896
:10E18000CE350020022803D0431E58425841704724
:10E19000064B1B681B7823B1054B1868C0F3C040C1
:10E1A0007047044B1878C0F380007047581800205F
:10E1B000F4350020F8350020F0B51A4A58B113881C
:10E1C0005B08012B98BF48F2050313800B6803F529
:10E1D000C333A0330B60138813F0010320D1124C1A
:10E1E000124D134E1349144F2278934218DA2A68BD
:10E1F0004FEA830E52F82320C2F30732500705D4AA
:10E2000012070BD53A680B3A2B2A07D891F8CC2382
:10E2100001EB8202D2F864034EF806000133E3E713
:10E22000F0BD00BFE0350020D04300208006002074
:10E230002E430020303B0020CC4300202DE9F0434A
:10E24000264B274CC8B11A78F02A0FDD7F221A70AE
:10E25000A07893F90120824201DA002A02DA987844
:10E2600040429870987802445A7001E00F321A7058
:10E270000A6802F582421A320A601A4A187815684A
:10E2800000221146247893F9016093F90270DFF8B7
:10E290005880A0F17F0EC0F1FF0CA2421CD255F8AD
:10E2A00022309B0416D5CBB29B1B83EAE379A9EB02
:10E2B000E379B9F1010F05DC33B1BB4214BF63460A
:10E2C000734602E0082300E0034608EB820989F860
:10E2D000033001310132E0E7BDE8F0835E03002046
:10E2E000D0430020800600202E4300202DE9F04777
:10E2F000244E70B1244A937803B9F378013BDBB222
:10E300009370224B1A68224B93FBF2F30A68134472
:10E310000B6000210C461F4D1A4FDFF87CE0DFF840
:10E320007CC0DFF86490A5F538783378994227DA15
:10E3300055F8040FC0F30323062B1FD19EF80030BD
:10E340005B070DD599F8023097F803A0234493FB9F
:10E35000FAF20AFB1233012BCCBF0023012303E0A6
:10E3600004F0010383F001033BB1C0F3834008EBE9
:10E370008000D0F864034CF8210001340131D4E767
:10E38000BDE8F087D0430020E0350020CC430020DA
:10E3900080841E00103E0020F83500202E4300200F
:10E3A000A0F17D03012B70B504460D460A4E05D839
:10E3B0007D213068FDF7FDF884F0200421463068A7
:10E3C000FDF7F7F835B12B881C4404EB142404F056
:10E3D000FF042C8070BD00BF801300205E2810B5A4
:10E3E0000146094C05D15D216068FDF7E2F83E2148
:10E3F00005E05D29606803D1FDF7DBF83D21606829
:10E40000BDE81040FDF7D5B8E03500202DE9F84310
:10E410002C4C20B32C4B08681B78DBB12B4AB2F98B
:10E420000230B2F90020002BB8BF5B42002AB8BF0F
:10E4300052429342B8BF13461933322B244AB8BF15
:10E44000322392FBF3F303440B60237A83F001033E
:10E45000237204E000F5433303F5A0730B60237AC5
:10E4600073B31A4BB3F90020192A04DC1A32CCBF5B
:10E470000024C02400E03024B3F90230192B02DD5F
:10E4800044F0500403E01933B8BF44F0A004114E27
:10E49000114FDFF84880DFF8489000253B789D4217
:10E4A0000EDA56F8043FDB0308D5284603F044FF94
:10E4B00020421CBFD9F8003048F825300135EDE77F
:10E4C000BDE8F883E0350020640D0020B01F002077
:10E4D00080969800103E0020D04300202E4300205C
:10E4E000B2A00108154AA8B1154B1888642343430C
:10E4F00040F2FF3093FBF0F3322B03DD0023537225
:10E50000012003E0142BCCBF02200820537A83F0B3
:10E51000010353720B4B93FBF0F00B681844537AD2
:10E52000086053B9084B4FF4806093F8CB1303EBAA
:10E53000810101F5597103F0E5BE7047E035002017
:10E54000D443002040420F00303B0020124A70B1FB
:10E55000124B1B7823B1012B0CBF0220082001E0D5
:10E5600093720120937A83F00103937200E00120FB
:10E570000B4B93FBF0F3086803440B60937A53B999
:10E58000084B4FF4407093F8CB1303EB810101F576
:10E59000597103F0B7BE7047E0350020CE37002038
:10E5A00040420F00303B0020274B30B3DA7A013273
:10E5B00002F00F02DA72DAB91A73244A126890076D
:10E5C00004D52348007808B102201873D20506D577
:10E5D000204AD2781AB11A7B42F004021A731E4AFA
:10E5E000127812F0050F02BF1A7B42F001021A7373
:10E5F0000A6802F5C332A0320A601B7B13B3124AC9
:10E60000D17A8A081341DB071CD5012A01F00103E6
:10E6100007D002D3022A0BD07047104AA2F118018A
:10E6200009E00F4A02F10801002B18BF114605E06E
:10E630000C4A02F11801002B08BF11464FF40030BC
:10E6400003F060BE704700BFE03500205417002083
:10E65000CE37002088170020F8350020BEA0010822
:10E66000A6A00108B6A00108024B597B024B18680E
:10E67000FCF79FBFE03500209813002010B504463A
:10E68000044B01461868FCF794FF034B587B60402D
:10E69000587310BD98130020E035002010B50446D3
:10E6A000C0B2FFF7EBFF200ABDE81040E6E738B53F
:10E6B0000546094C094B0022206824215A73FCF7B7
:10E6C00078FF20685421FCF774FF29462068BDE8D4
:10E6D0003840FCF76EBF00BF98130020E0350020E3
:10E6E00030B585B004AC002524F8025D0091ADF88A
:10E6F000060021461020FFF753FE21469DF8060034
:10E70000FFF74EFE21469DF80700FFF749FE214620
:10E710009DF80000FFF744FE21469DF80100FFF739
:10E720003FFE21469DF80200FFF73AFE21469DF884
:10E730000300FFF735FE9DF80E002946C043C0B226
:10E74000FFF72EFE05B030BD73B50D460646084CEA
:10E750002068FDF7A9FC002296F9000001920095BF
:10E760004FF496430821FDF7B3FC206002B070BD62
:10E770006813002010B5054C2068FCF717FF18B18E
:10E780002068FCF710FFF7E710BD00BF68130020FA
:10E790000028114AB8BF404290FBF2F330B50F4C4D
:10E7A0003C2504FB030068430D4D90FBF2F22D68FD
:10E7B0002D7B25B903EB830303EB830301E0C3EB5C
:10E7C000031302EB830304FB02020B804FF47A7302
:10E7D00092FBF3F24A8030BD80969800806967FF13
:10E7E0001C13002010B50446C0B2FFF7F7FDC4F3B8
:10E7F0000720BDE81040F1E5024B5E215868FCF7A8
:10E80000D8BE00BFE035002038B50546054C5E2176
:10E810006068FCF7CEFE29466068BDE83840FCF72A
:10E82000C8BE00BFE0350020438803F0400080B23E
:10E8300020B113F0140F14BF0120002000F00100DC
:10E840007047654B73B51A68644972B11046FFF79B
:10E85000EBFF50B10B78002B2FD1614B1B6863B3DA
:10E86000604A536001230B7027E05F4B5B4D1878C3
:10E87000FFF788FC0B78044683421ED0B8B1E2B1A2
:10E880005A4B92F900001B6800225B780421003388
:10E8900018BF01230193022300934FF41653FDF791
:10E8A00017FC504B586040B101232B7005E04D4ED2
:10E8B0007068FDF7F9FB74602C704D4B4D4D187866
:10E8C000FFF760FC2B780446834218D088B14A4B8E
:10E8D0001B68A3B10022012493F9000008214FF422
:10E8E000964301920094FDF7F3FB444B186028B95E
:10E8F00005E0424E3068FDF7D7FB34602C70404B8A
:10E90000404D1878FFF73EFC2B780446834229D00F
:10E9100000B33D4B1B682BB33C4A93F900001268CF
:10E92000032352782021002A0CBF082209220192D9
:10E93000009300224FF46143FDF7CAFB344B18608B
:10E9400080B1344A012313702B70334B1A68334B58
:10E950001A6007E02E4E3068FDF7A6FB2D4B3460A1
:10E960001C702C702E4B2F4D1A685AB11046FFF7B1
:10E970005BFF38B12B7863BB194B1B684BB32A4A3A
:10E9800013601CE0294B1878FFF7FCFB2B7804463A
:10E9900083421ED0B0B1E2B1D37992F900000221D6
:10E9A0000022002B8DE80600214908BF022351F800
:10E9B00023301021FDF78CFB1B4B186048B101235D
:10E9C0002B7006E0184D2868FDF76EFB154B2C6088
:10E9D0001C7002B070BD00BFB809002000130020F9
:10E9E000B8410020E0350020BC0900201C130020A5
:10E9F000BD09002024130020781300206813002094
:10EA0000C40900207E130020C009002090130020BC
:10EA10008013002084130020841700208813002016
:10EA2000C80900209513002098130020CC0900206D
:10EA300080B10108FEF7EABD08B50448F7F754FDB8
:10EA4000BDE808400120F7F747BF00BF78CD0108B7
:10EA500046492DE9F04F0A884B6802F0080003F49C
:10EA60004754044303F4804012F0010F44EA0004C9
:10EA700003F4004014BF4FF0020A4FF0000A0443B1
:10EA800012F0020F03F4803014BF4FF004094FF06E
:10EA90000009044312F0040F03F4003003F480254E
:10EAA00014BF4FF010084FF00008044312F0400F5D
:10EAB00044EA050414BF4FF0200C4FF0000C03F49F
:10EAC000002012F0100F40EA040014BF4FF4007E43
:10EAD0004FF0000E03F4801412F0200F14BF4FF417
:10EAE00080670027044312F4807F087A14BF4FF434
:10EAF0000066002603F0285312F4007F14BF4FF481
:10EB000000150025C0F3800012F4806F43EA040270
:10EB100042EA00024FF00000034642EA0A0242EADB
:10EB2000090242EA080242EA0C0242EA0E0242EA02
:10EB3000070242EA060242EA050214BF4FF0806B68
:10EB40004FF0000B4E7A42EA0B020A310125B34224
:10EB500009D25C5C05FA04F414421CBF05FA03F404
:10EB600020430133F3E7BDE8F08F00BFF03500200C
:10EB700038B50D4C05462368984206D1FDF794FA46
:10EB80004C22002120460AF081F9E36CAB4209D106
:10EB90002846FDF789FABDE838404C220021034899
:10EBA0000AF074B938BD00BFEC40002038410020A5
:10EBB000034B9A6AD379591CD1711344187A704760
:10EBC000F035002010B5FFF7F3FF84B2FFF7F0FF38
:10EBD00004EB002080B210BD10B5FFF7F3FF044630
:10EBE000FFF7F0FF04EB004010BD38B50446054DBB
:10EBF0000146E86AFEF70AFDAB6A987960409871B1
:10EC000038BD00BFF035002010B5054CA36A9879D7
:10EC1000FFF7EBFF206BBDE81040FCF7B4BC00BF72
:10EC2000F035002070B506460D460E4C206BFCF703
:10EC3000AFFC2420FFF7D9FF4D20FFF7D6FF002EB1
:10EC400014BF21203E20FFF7D0FFA36A00222846F0
:10EC50009A71FFF7CAFFA36ABDE8704093F84900B4
:10EC6000C3E700BFF035002001460020DAE710B509
:10EC70000446C0B2FFF7B9FF200ABDE81040B4E770
:10EC800010B5044680B2FFF7F2FF200CBDE810403B
:10EC9000EDE7024B0146586BFEF7B8BCF03500209B
:10ECA0000FB407B5064804AB53F8042B0549406B75
:10ECB0000193FCF781F803B05DF804EB04B07047F2
:10ECC000F035002035EA00082DE9F3471E48FFF72C
:10ECD000E7FF1E4D1E4E05F5D279AB7995F808A0D9
:10ECE00056F82370EB792C6806EB8303D3F8688021
:10ECF0002846BAF1000F11D0FEF76BFC04F1404139
:10ED0000A1F58431890A0246CDF80480CDF800A02F
:10ED10003B4641310F48FFF7C3FF0EE0FEF759FCB9
:10ED200004F14041A1F58431890A0246CDF8008002
:10ED30003B4641310848FFF7B3FF0C35A945CCD11C
:10ED400002B0BDE8F08700BF91CD01082836002051
:10ED5000B8AD0108AFCD0108C1CD010807B5064B1C
:10ED6000064A0193064B074900930748074BFFF7F4
:10ED700097FF03B05DF804FB97B20108CFB3010819
:10ED80008EB20108CAB30108D1CD010882B20108D0
:10ED90002DE9F04F4C4800258BB0FFF781FF2E4640
:10EDA000A8464A4C4A4B1A68002393425BDA494909
:10EDB00051F823108C4201D00133F6E76368012D2E
:10EDC0000793E36AD4F800A00893236BD4F824B027
:10EDD00009935ED1404BB3F8DC0104F0C5FE014657
:10EDE0003E4804F0CDFF05F0F3F83D4B814693F823
:10EDF000EA31012B90FBF3F755D85346079A294681
:10EE00003848FFF74DFF4F46089B099803FB07F270
:10EE10000BFB07F302F59C5203F59C534FF47A71F8
:10EE200008320833B2FBF1F2B3FBF1F3B0FBF1F1BE
:10EE300004910A2193FBF1F0052D18BFF61801FB90
:10EE40001033039392FBF1F318BF904401FB13229C
:10EE5000029001920093089A5B4639462248FFF7D8
:10EE60001FFF012D25D0214B3434A34205F10105AC
:10EE700098D10A2296FBF2F398FBF2F102FB13669B
:10EE80001B48009602FB1182FFF70AFF0BB0BDE89A
:10EE9000F08FA06A04F068FE0146104804F070FF8D
:10EEA00005F096F80746524629461248FFF7F8FE45
:10EEB000AAE70B4B93F8EA31012BD4D94A460799BC
:10EEC0000D48FFF7EDFECEE7F3CD010898000020D6
:10EED000181700201C170020F0350020002474496A
:10EEE000303B00204CCE01085ECE0108A00200207D
:10EEF00096CE01083DCE010884CE01082DE9F743E6
:10EF00002C492D4C08882D4B64282D4A2D4EA8BF26
:10EF100064201D68128823782B4F019096F8DE013B
:10EF2000DFF8D49007EB8000D0F8B41027480091A8
:10EF30004FF47A71B5FBF1F1FFF7B2FE6168244B33
:10EF40002448B1FBF3F1FFF7ABFE234B0024D3F8C9
:10EF50000080224B53F82410E1B10125A54015EAA9
:10EF6000080F15D02B0713D014F809200C2303FB2E
:10EF7000042307EB8303D3F8E4201948FFF790FE3E
:10EF8000022D05D1174B997A11B11748FFF788FE6A
:10EF90000134DEE71548F7F7A7FA154BB6F8DC1190
:10EFA0001A8814484FF4AF6392B203B0BDE8F0433F
:10EFB00076E600BF28140020640300208417002098
:10EFC00014170020F0350020B8AD0108C6CE0108A6
:10EFD00040420F0013CF0108502D00207CAE0108E5
:10EFE00023CF0108002D00202BCF0108F3BB01081F
:10EFF0002C3B00202FCF01085403002070B503796B
:10F0000013F0C00302D0402B06D070BD0269C16866
:10F01000BDE87040104843E6057B1048F7F764FAF6
:10F020000F4BED002B4493F8A8610024B4420ED29C
:10F0300014B10C48F7F758FA094B0B482B44D3F896
:10F04000A43153F82410FFF72BFE0134EEE70748F4
:10F05000BDE87040F7F748BA61CF01087ACF0108E0
:10F06000B8AD01088ACF0108ADBA0108F3BB0108A9
:10F0700037B5154602790B4602F00F010446052903
:10F0800032D8DFE801F00305080A0D0F19782CE0EB
:10F0900093F9001029E0198827E0B3F9001024E063
:10F0A000196822E069461868FBF70EFE01461C4805
:10F0B000FFF7F6FD95B3237913F0C00F2ED1E0686A
:10F0C00004F056FD6946FBF7FFFD01461548FFF7C2
:10F0D000E7FD206904F04CFD6946FBF7F5FD0146AC
:10F0E0001048FFF7DDFD19E0002112F0C0020CD03E
:10F0F000402A13D1227B0C4B03EBC203D3F8A4317B
:10F1000053F82100FFF7CCFD08E00848FFF7C8FDE1
:10F1100025B12269E1680648FFF7C2FD03B030BDA2
:10F12000AEBA0108ADBA0108B8AD010890CF010828
:10F130008CCF010838B50D460446F7F7E7FE2A469E
:10F1400001462046BDE8384092E72DE9F843002407
:10F1500081462546134E54F8068049464046A71975
:10F1600009F02AFF88B141460F48FFF799FD0021B9
:10F170003846FFF7DFFF0D48F7F7B6F93846FFF7D7
:10F180003DFF0A48F7F7B0F901351434B4F5436F81
:10F19000E1D125B9BDE8F8430548F7F7A5B9BDE8C1
:10F1A000F88300BF3CA10108F5C30108F3BB0108C7
:10F1B00086BA01082DE9F74F064603F075FF0546AC
:10F1C00020B1012818D133782A2B15D17348F7F7CD
:10F1D0008BF9734E0024A159A7197248FFF760FDFF
:10F1E00029463846FFF7A6FF14346F48F7F77CF935
:10F1F000B4F5436FEFD1CEE03D21304609F07DFEFE
:10F20000002800F0C380034613F8012C591E202A61
:10F2100001D10B46F8E79B1B013082469AF800208B
:10F220000130202AF9D05E4C4FF000094FF0140B4A
:10F23000DDB20BFB09F353F804801F19404603F0BD
:10F2400033FF414602460090304609F064FE002834
:10F2500040F09080009BAB4240F08C803D7915F0EF
:10F26000C0030CD0402B7DD1504A3B7B002602EBE3
:10F27000C30393F8A82104460146834633E0504671
:10F2800007F042F904465046FBF78CFC0646F86846
:10F2900004F06EFC0146304604F070FE002861D098
:10F2A000386904F065FC0146304604F05DFE002834
:10F2B00058D005F00F03052B1AD0264618E0A1B947
:10F2C000D3F8A401514650F824000192009309F0AC
:10F2D000E5FD009B0028019A05BF2646012100217B
:10F2E0004FF0010B01349442E9D3BBF1000F39D048
:10F2F0002B4A142303FB092905F03002102A31465A
:10F30000D9F8083006D12A4A6C2092F8AC2400FBC8
:10F3100002330DE0202A0BD1254A92F8AC04254A8D
:10F3200092F8DF410C2262436C2404FB0022134458
:10F3300005F00F02052A0BD8DFE802F003030505EC
:10F340000709197004E0198002E0196000E01E60EE
:10F3500041461948FFF7A4FC3846002103B0BDE838
:10F36000F04FE7E61548F7F7BFF8384603B0BDE8B9
:10F37000F04F43E609F10109B9F19C0F7FF459AF51
:10F380000F4803B0BDE8F04FF7F7AEB8304603B012
:10F39000BDE8F04FD9E603B0BDE8F08F93CF010888
:10F3A0003CA10108F5C30108F3BB0108B8AD010891
:10F3B000303B0020F0350020A8CF0108B3CF010872
:10F3C00086BA01080CB400F0200307B503F0FF0073
:10F3D00073B161B92320FFF75CFC084805AB049AC0
:10F3E0000749406B0193FBF7E7FC012000E0002098
:10F3F00003B05DF804EB02B0704700BFF0350020A9
:10F4000035EA00080CB4C30607B500D549B9084869
:10F4100005AB049A0749406B0193FBF7CDFC012033
:10F4200000E0002003B05DF804EB02B0704700BFBD
:10F43000F035002035EA000813B50B4B04465B6835
:10F4400001AA02211B20984760B1BDF804304FF497
:10F450008C725BBA9BB203F54E53103393FBF2F3FD
:10F460002333238002B010BD282D0020044B1A78CE
:10F4700002F0FF0012B100221A700120704700BF95
:10F48000D037002037B5104B04465D686A46062128
:10F490001878A847A8B19DF800209DF801300120F8
:10F4A00043EA022323809DF802209DF8033043EABB
:10F4B000022363809DF804209DF8053043EA02236F
:10F4C000A38003B030BD00BF282D002013B5104B22
:10F4D00004465B686A4606213B209847A8B19DF820
:10F4E00000209DF80130012043EA022323809DF88B
:10F4F00002209DF8033043EA022363809DF8042034
:10F500009DF8053043EA0223A38002B010BD00BF7E
:10F51000282D0020014B01221A707047D03700209F
:10F5200070B5104C0546192001F036FAA368002189
:10F530001520984710B9022001F038FAA36845F069
:10F54000180116209847A368002117209847A36840
:10F5500001213D209847A36801213E20BDE870406D
:10F56000184700BF282D00200A460146682001F0F8
:10F57000BDBA10B5044608220F21182001F0B6FAD2
:10F580000E221021182001F0B1FA4FF4805323818C
:10F5900010BD134B10B51B78044608222D215320B3
:10F5A00073B101F0A3FA0A223121532001F09EFA2F
:10F5B0000C222C21532001F099FA9022382108E0E6
:10F5C00001F094FA0A223121532001F08FFA0A2225
:10F5D0002C21532001F08AFA4FF48073238110BD4F
:10F5E0004E2D002013460A460146682001F0C8BA95
:10F5F00013B5062204466B4601211C2001F0C0FA17
:10F6000008B39DF801309DF80020042143EA02224E
:10F6100042F38D0292FBF1F29DF8023022809DF8B8
:10F62000032042EA032242F38D0292FBF1F29DF89D
:10F63000043062809DF8052042EA032343F38D03E2
:10F6400093FBF1F3A38002B010BD13B5062204466C
:10F650006B460221182001F093FAB8B19DF80130F1
:10F660009DF800201B0203EB920323809DF80330DA
:10F670009DF802201B0203EB920363809DF8053086
:10F680009DF804201B0203EB9203A38002B010BD7F
:10F69000304B2DE9F3411B780546002B39D000246F
:10F6A00026462746A04601346B46082232215320C5
:10F6B000E4B201F065FA08B9002047E09DF80120A6
:10F6C0009DF80030202C03EB02231BB29DF8032091
:10F6D00098449DF8023003EB02231BB21F449DF8AF
:10F6E00005209DF8043003EB02231BB21E449DF855
:10F6F000073003F07F0301D0002BD4D198FBF4F83E
:10F7000097FBF4F796FBF4F4A5F800806F80AC80CB
:10F710001CE06B4606223221532001F031FA00280A
:10F72000CAD09DF801209DF8003003EB02232B8006
:10F730009DF803209DF8023003EB02236B809DF8B7
:10F7400005209DF8043003EB0223AB8002B0BDE836
:10F75000F08100BF4E2D002038B5002205462A2139
:10F760001C2001F0C3F902220E211C2001F0BEF979
:10F7700003220F211C2001F0B9F912222B211C2099
:10F7800001F0B4F91520FDF7FBFC1422827100246E
:10F790000822C27104720621FDF718FD02222C21F5
:10F7A0001C2001F0A3F901222D211C2001F09EF95B
:10F7B00022462E211C2001F099F905222A211C2025
:10F7C00001F094F94FF480732B8138BD2DE9F74394
:10F7D0004B4C6578002D40F08F804A4B1B68002B06
:10F7E00000F08A801878FDF7CBFC0646142383715D
:10F7F0000823C37105720621FDF7E8FC424B304631
:10F800006360FDF7E6FE002867DB404B221D43F8EE
:10F8100020203268DFF8048102F14042A2F58432F0
:10F8200018F8007030464FEA9229FDF7D2FEC0B2B8
:10F8300000F0030200F0FC0000F1804000F5803091
:10F84000816892000F23934021EA03038360836859
:10F850005FFA89F101FA02F21A4382603046FDF73D
:10F86000B8FE012101FA00F0C243294B5861D3F8D8
:10F8700000E00EEA020EC3F800E0D3F804E002EA6A
:10F880000E0EC3F804E0D3F800E040EA0E0EC3F811
:10F8900000E0D3F808E002EA0E0EC3F808E0D3F85F
:10F8A0000CE002EA0E02DA601A4A136818431A4B97
:10F8B0001060DA5DF02A10DDF022DA5508EB07035C
:10F8C0001B7C01A88DF8043003238DF805308DF8DA
:10F8D00006508DF8071001F0E9F83046FDF779FE83
:10F8E000012313FA00F01EBF094A136818434FF0B2
:10F8F000010318BF1060637003B0BDE8F08300BF60
:10F90000D0370020402D002015F50008A434002039
:10F9100000040140080401408C05002050B101089A
:10F9200037B50546FFF752FF2E4B1A682E4B9A4209
:10F930000ED14FF40053ADF8043002238DF8073098
:10F9400004230DEB030129488DF80630F5F7D8FCA8
:10F95000274CFFF73BFFA36880216B20984764206A
:10F9600001F01AF8A368072168209847642001F085
:10F9700013F8A36800216B209847642001F00CF86D
:10F98000A36801216B2098470F2001F005F8A368B8
:10F9900018211B2098470F2000F0FEFFA3681821B4
:10F9A0001C2098470F2000F0F7FFA36829461A2073
:10F9B00098470F2000F0F0FF0E4AA3681178192035
:10F9C0009847642000F0E8FFA3681021372098478B
:10F9D0000F2000F0E1FFA36801213820984703B011
:10F9E00030BD00BF58030020001BB70000100140CD
:10F9F000282D0020542D002010B50446FFF7E6FE08
:10FA00004FF40063238110BD70B50546154CFFF718
:10FA1000DDFEA36880216B209847642000F0BCFFC6
:10FA2000A36803216B2098470F4AA3681178192017
:10FA300098470F2000F0B0FFA36829461A20984786
:10FA4000A36818211B209847A36818211C209847F9
:10FA5000A368022137209847A36801213820BDE818
:10FA600070401847282D0020542D002010B5044662
:10FA7000FFF7ACFE064B5B7813B1012B03D010BD32
:10FA80004FF4806301E04FF40063238110BD00BF99
:10FA9000252D002010B4047B01680222A240436996
:10FAA0004A604FF6FE724168086802400A60596A6F
:10FAB0009A6A914203D0184610BCFBF769BB012239
:10FAC00083F8442010BC70470148F5F71FBB00BF06
:10FAD0004C1900200148F5F719BB00BFF8180020A9
:10FAE0000148F5F713BB00BFA41800202DE9F04F23
:10FAF000D04D8BB02888D04FD04C002840F09A8051
:10FB000097F85735012B05D197F85805A0F1200536
:10FB10006842684100F00100F9F730FAF9F744F85B
:10FB2000256849202E4602F085FDC54BDFF814B349
:10FB3000186802F03AFE56F8040B02F036FE304622
:10FB400001F0CAF805F1100001F0C6F805F11C0932
:10FB50004FF010084FF0010ADBF800200AFA08F312
:10FB60001342B84E03D0D9F8000002F02DFE08F180
:10FB70000108B8F1130F09F10409EDD1032105F1D2
:10FB8000280002F025FEB7F8CC30B5F92E00C01AD7
:10FB900002F00BFE3368D90408D5AB4BB5F86C0006
:10FBA0001B88181AC0F30D0002F0FFFD33689A0499
:10FBB00003D5B5F86E0002F0F8FD33681B0403D5D9
:10FBC000B5F8700002F0F1FDA846032105F1300000
:10FBD00002F0FEFD032105F1360002F0F9FD0421DB
:10FBE00005F13C0002F0F4FD38F9440FB7F8CC30D1
:10FBF000DFF864A2C01A02F0D8FD4FF001099AF8AC
:10FC00000030994509DA38F9020FB5F9443009F1A5
:10FC10000109C01A02F0D8FDF1E73368980505D54F
:10FC2000B5F96600A0F2DC5002F0CEFD22686260F9
:10FC3000A260A3E1854B1E68D4F868319E420FD0C4
:10FC4000834BC4F868611B78093B012B08D8452019
:10FC500002F0F0FC002002F0EDFC304602F0A5FDC1
:10FC60007C4BD4F86C811E68464513D0734BC3F8A7
:10FC70006C61774B1B78093B012B0BD8452002F0B8
:10FC8000D9FC1E2002F0D6FC304602F08EFD404624
:10FC900002F08BFD97F857152B8897F858050B4401
:10FCA000013BB3FBF0F200FB1233994240F2798141
:10FCB0000120F9F763F9F8F777FF502026686568A7
:10FCC00002F0B8FC2268A36810681B6862680344ED
:10FCD0001068A3EB400002F077FD06F1040E281D2A
:10FCE000002350F823105EF82320521A02A941F88D
:10FCF00023200133032BF4D1084600F0EDFF06F179
:10FD0000100E05F11000002350F823105EF8232098
:10FD1000521A02A941F823200133032BF4D10846DB
:10FD200002F0B4FC474A06F11C0B05F11C094FF028
:10FD300010084FF0010A13680AFA08F0184208D0B8
:10FD4000DBF80000D9F800300192C01A02F03CFD47
:10FD5000019A08F10108B8F1130F0BF1040B09F136
:10FD60000409E8D106F1260005F12601002331F946
:10FD700002EF30F9022FCEEB02020DF1080E4EF821
:10FD800023200133042BF2D103214FF0000A4FEA64
:10FD90008A035FFA83FA02AB53F821206AB102F1B9
:10FDA00008000F2802D84AF0010A06E08032FF2A34
:10FDB00094BF4AF0020A4AF0030A11F1FF31E6D279
:10FDC00050464FF0000802F035FCC1460DF1080B1B
:10FDD0000AF00301022916D003291ED0012950D1AF
:10FDE000DBF80000B9F1000F04D100015FFA80F8E0
:10FDF000894646E000F00F0040EA080002F01AFCD5
:10FE00004FF000093DE0B9F1000F0DD0DBF8000024
:10FE1000C0F3031040EA08002CE0B9F1000F1DD137
:10FE20009BF8010002F006FC9BF8000002F002FCC7
:10FE300027E000BFBC0A0020303B0020D83700205C
:10FE4000C00A0020B40A0020B80A0020E8410020BF
:10FE50007A270020F4350020CF1F0020DBF80000B7
:10FE6000C0F3033040EA080002F0E4FBDBF80000D6
:10FE7000C0F3071002F0DEFBDBF8001009015FFAA7
:10FE800081F80BF1040B06AB9B454FEA9A0A9FD110
:10FE9000B9F1010F02D1404602F0CCFB454B1B6883
:10FEA00013F4805807D0B6F86C20B5F86C104FF0FA
:10FEB0000108521A029299040BD50AAA02EB880192
:10FEC000B5F86E00B6F86E2008F10108121A41F874
:10FED000202C1A040CD50AAB03EB8802B5F870107D
:10FEE000B6F8703008F101085B1A42F8203C02E0D5
:10FEF000B8F1000F22D0B8F1010F03D1029802F03F
:10FF000063FC1BE008F1FF33002002AA52F8232013
:10FF10004000C0B20AB140F0010013F1FF33F4D247
:10FF200002F088FB4FF0000902AB53F8290008B13A
:10FF300002F04AFC09F10109C145F5DB032130203B
:10FF4000F9F778F803213620F9F774F804213C20FA
:10FF5000F9F770F8184B44201978F9F76BF8154B3E
:10FF60001B689B0506D5B6F96600B5F96630C01A60
:10FF700002F02AFC63682268A36062600F48121ACC
:10FF800091100F4A4A43531C032293FBF2F202EBF7
:10FF900042029A1A742303FB02032360094B0122D5
:10FFA0001A7097F85935012B01D1F9F7ADF90BB05B
:10FFB000BDE8F08FB40A0020CF1F0020E4370020F6
:10FFC00035C2724F350D00200C4A1388013313805F
:10FFD0000B4A1368013313600A4A138801339BB23A
:10FFE000202B03BF00231380074A138002BFB2F8FF
:10FFF00070310133A2F87031704700BFBA0A002097
:020000040801F1
:10000000C00A0020BC0A0020D83700202DE9F74F95
:10001000C2EB030817460E9B0D9A4C4C9B1A00939B
:100020006368002914BF06260426013305468A4664
:1000300024D123689E4240F28580DFF82CB15BF822
:10004000230003F031F80B3002F01AFA814608B1B0
:10005000012078E021683E485BF82120032994BF05
:100060002946514602F0D4FA3A4A1368181A6368CE
:10007000106001336360384B83F87291DFF8D490DD
:10008000DFF8D4A063680C9A304D934242DA0D9A9F
:100090004AB1009A0D995A43895C01228A402F493E
:1000A00009680A4232D003FB08F5236807EB050B09
:1000B00023B9785902F0F8FF431D00E003231846E6
:1000C000019302F0DDF90028C2D1D9F80000019BAC
:1000D000C01A9AF87231C9F800001BB12C2002F046
:1000E000A9FA02E001238AF87231236843B97859EA
:1000F00002F01EFA9BF904104B1C07D0184803E0CD
:100100009B449BF80410174802F082FA636801339D
:100110006360B7E710D1012002F0B2F960B90D4A6F
:100120000A201368013B136002F084FA2B68013344
:100130002B604FF0FF336B602068864294BF002035
:10014000012000E0002003B0BDE8F08FAC0A0020E1
:10015000FED20108A40A0020D8370020B40A0020EB
:100160000DD3010890CF010868B101080C4B800A3B
:1001700098420CD004D8B0F5801F0CD101207047F4
:10018000084B984205D04933984206D003E002203C
:10019000704703207047FE2070470020704700BF63
:1001A00001001000020010002DE9F04705468946C5
:1001B000068A83894FF000479BB21E404FF000082B
:1001C000002E3AD0B6FA86F327FA03F2D2431B3B4D
:1001D00091B229821640042BF2D8DFE803F02622E0
:1001E0001E1A0300D9F8244024B1013CA4B2C9F876
:1001F000248001E0AC8DA4B2D9F820A0BAF1000FA0
:10020000DED0DAF80030504621469847DAF804A0EC
:10021000F4E7D9F80000A98E0BE0D9F80400298F83
:1002200007E0D9F80800A98F03E0D9F80C00B5F869
:100230004010036889B29847C2E7BDE8F087F0B57F
:1002400040F2E6363A4DB5F90040241A04F2F317AD
:10025000B74203D8002CB8BF644201E04FF4FA74EF
:10026000B5F902502F1A40F2E63007F2F315854235
:1002700003D8002FB8BF7F4201E04FF4FA77BC42A9
:10028000B8BF3C462B48C4F5FA74052794FBF7F732
:10029000B0F90240B0F90060002CB8BF6442002EF3
:1002A000B8BF7642B442B8BF3446012A21D1AE2944
:1002B00039DC1220C1F1AF0141430A220C1B91FB32
:1002C000F2F1544394FBF1F2642AA8BF6422002B9C
:1002D000C1BFA7F164006421484390FBF3F0D4BF91
:1002E0000020401822EAE2724243642092FBF0F0C0
:1002F0001BE000290DDDC4F5E164122594FBF5F542
:100300004D43642295FBF2F5501A2844584390FB64
:10031000F2F3002B07DDA7F164006424444394FB4F
:10032000F3F0643001E00020F0BD20EAE070F0BDA1
:1003300058170020B81F00202DE9F3470446808C91
:10034000E8B1294B1D781E46CDB9E18C02F09AFD2B
:100350008146DFF8A880254F4FF0010AA08C03F0FA
:1003600003FCCDF800A001464B467819D8F80020D0
:100370001C3502F0EFFC542DF0D1012333701C4AE0
:10038000E37F1178164699422AD0228C42B3012B82
:1003900003D0E37F022B21D110E0DFF86080154FFE
:1003A0000025208C03F0E0FBD8F8002001467819E6
:1003B0001C3502F05BFD542DF3D1EAE7DFF83C80F9
:1003C0000D4F00257819B8F8002094F8201005F595
:1003D000F87502F06FFCB5F5BA6FF3D1E37F3370B7
:1003E00002B0BDE8F08700BF082700200C270020DE
:1003F0004C390020EC1F002064200020D01F00207A
:1004000010B5084C0021606803F09AFD38B1064B26
:10041000186803F0A9FB054903F0FEFB6060606803
:1004200010BD00BF4C390020D01F0020BD378635DD
:100430002DE9F0472D4F2E4EDFF8B88000243D788F
:10044000E0B2A8422A490FD206EB80039B684BB169
:100450000B2807D898F8002022B106EB4002DB6891
:10046000118F98470134EAE791F85030002B3BD0C8
:10047000002291460C1D01F1080850272826AA42A7
:1004800032DA4FF0000E964509D058F82E00636816
:1004900040685B68984220D00EF1010EF3E7636874
:1004A000D3F804A05046FFF761FEEFF3128387F301
:1004B0001288BAF824E006FB001C1FFA8EFE0EF12B
:1004C0000100CCF87800BAF81400DBB280B240F03A
:1004D0000100AAF8140083F3118854F8043F013294
:1004E0001B68A3F80090CAE7BDE8F087CF1F002083
:1004F0004C3900205D0300200B4B0C481A680C4B54
:1005000030B502F48052D3F8F440D3F8F850002309
:1005100012B1B4F9041001E0B5F9041020F8131079
:1005200001330C2BF4D130BD54170020AC13002044
:100530004C39002070B5124D00242146702205F17F
:10054000FD0085F8FC4008F0A1FC2A46214605F193
:10055000FD04D5F870310B4493F9020078B11E68A0
:1005600008190E519E88073186809B797029837106
:1005700092F8FC3003F1010382F8FC30E9D170BD40
:100580004C390020094BD3F874210E2303FB0020C3
:10059000437AFF2B07D0064A12789A4203D9054ABC
:1005A00032F913007047B0F9040070474C3900204D
:1005B000B0410020581700202DE9F74F494B4A4C15
:1005C000D3F80090D4F878514946284603F024FB2C
:1005D000D4F87C7180464946384603F01DFBD4F8B8
:1005E000806100904946304603F016FB394682464A
:1005F000284603F011FB31468346284603F00CFBE6
:1006000031468146384603F007FB394601903846AB
:1006100003F002FB014603F0F7F931460746304686
:1006200003F0FAFA014603F0EFF9064639464FF0B7
:100630007E5003F0E7F9314603F0E4F95146C4F87F
:100640008401584603F0DEF9014603F0DDF949461E
:10065000C4F88801009803F0D7F9014603F0D4F9F3
:100660005946C4F88C01504603F0CEF9014603F018
:10067000CBF92946C4F89001284603F0CDFA01468B
:1006800003F0C2F901464FF07E5003F0BBF931464A
:10069000054603F0B7F94146C4F89401019803F008
:1006A000B1F9014603F0B0F90099C4F89801484641
:1006B00003F0A8F9014603F0A7F90199C4F89C01D9
:1006C000404603F0A1F9014603F09EF93946C4F80B
:1006D000A001284603F096F9C4F8A40103B0BDE8D0
:1006E000F08F00BF6C0300204C39002010B50C4C7B
:1006F0000123E3704FF48060022384F82030FCF77C
:10070000A3FF084A084BD2F8A8211B68527864213D
:1007100001FB0233636123880133238010BD00BFD6
:10072000881700204C390020841700200149024816
:100730003AE500BF183A002000080040014902488D
:1007400032E500BFF03900200004004001494FF0BD
:10075000804029E5C83900200149024824E500BF4E
:10076000A0390020002C0140FFF7F6BFF8B504685F
:1007700006462046FFF7FAFC03284CD896F805E019
:100780004FEA9E0C39B9A589AFB2022505FA0CFED5
:1007900027EA0E05A5810A2303FB00C31E4D05EBC6
:1007A000830779657A6641B17379A2899B08022132
:1007B00001FA03F313439BB2A381282202FB00F347
:1007C000164F03F120023A44EFF31286502181F3D1
:1007D000128803F10C011C3339443B4451F8047F67
:1007E00017B117600A6804329942F7D100231360E9
:1007F000F3B283F31188282303FB0050436F23B126
:10080000A3899BB243F0010304E0A38923F0010311
:100810001B041B0CA381F8BD4C390020A03900201B
:10082000254B10B55A43254B254C1B680139B3FBAA
:10083000F2F20388013AA04289B292B29BB212D07E
:1008400004F50064A0420ED0B0F1804F0BD0A4F5A7
:100850009834A04207D004F58064A04203D004F588
:100860008064A04202D123F070039BB2154CA042D9
:1008700006D004F58064A0421CBF23F440739BB2F1
:1008800003800F4B8185984202850FD003F50063EA
:1008900098420BD003F54063984207D003F580637C
:1008A000984203D003F58063984201D10023038668
:1008B0000123838210BD00BF40420F006803002067
:1008C000002C01400010004073B505460068FFF79A
:1008D000A7FF2A680124138800269BB243F0010376
:1008E0001380AB7901A88DF804308DF805408DF8A0
:1008F00006608DF8074000F0D9F8AB791B2B0BD1BF
:10090000192301A88DF804308DF805408DF8066094
:100910008DF8074000F0CAF802B070BD10B50A4A61
:100920000A4C1168A36800BF10688142F9D1084AD7
:100930004FF47A70D2F8AC4100FB04F2D31AB3FB47
:10094000F4F300FB013010BD8417002010E000E03C
:100950004C39002038B50446FFF7E0FF0546FFF7A5
:10096000DDFF401BA042FAD338BD10B4084B094943
:100970001A7800231846934205DA51F823400133D0
:1009800024682080F7E740F2DC5010BCE2E700BFAB
:10099000CF1F00205439002010B504462CB14FF46D
:1009A0007A70FFF7D7FF013CF8E710BD2DE9F04161
:1009B00080460B25013D33D001210846FCF7F8FDA8
:1009C00000210846FCF7F4FD08F101063227052452
:1009D0000120FCF7C7FB0020FCF7C4FB0120FAF75D
:1009E000CBFB3846FFF7D8FF0120FCF7BBFB00200C
:1009F000FCF7B8FB0020FAF7BFFB3846FFF7CCFF47
:100A00003CB1013CE4D14FF4FA70FFF7C5FFFA277F
:100A1000DEE7013EDCD14FF47A70FFF7BDFFC9E796
:100A2000024A034BDA60BDE8F08100BF0400FA051A
:100A300000ED00E0024A136801331360704700BF05
:100A4000841700200EB40FB5074A06AB0190074982
:100A500001A80393FAF7B0F9019B00221A7004B0C1
:100A60005DF804EB03B070472CD3010801A3000824
:100A700000F01F0240090123022803FA02F308D004
:100A800003280BD001280DD107494A6913434B6154
:100A9000704705498A6913438B6170470249CA69E7
:100AA0001343CB61704700BF001002400D4B4278EA
:100AB000DB680D49DB43C3F30223C3F1040302FAED
:100AC00003F302781B01DBB20A4482F80033037897
:100AD0000122580903F01F0302FA03F341F8203002
:100AE000704700BF00ED00E000E100E013B5224BCD
:100AF000400002ACC0B2987404F8012DD9740122F0
:100B000000215A7599751A755A741C4A9C61DC61EA
:100B10001974918889051AD41188CC0511D44FF421
:100B2000805410881549800506D5013CF9D11A8EEC
:100B3000013292B21A8615E00A8892B242F48072AB
:100B40000A800E498A8892B242F440728A804FF439
:100B50008054597C084A51B1013CFAD1138E0133BB
:100B60009BB213860120F4F741FC204602E0147C7E
:100B700084F0010002B010BDFC3A00200058004093
:100B800010B54000204CC0B2A074E17401200021D7
:100B90006175A07522751D4A6074E361A3612174BB
:100BA000938813F4007F23461AD11188CC0511D401
:100BB0004FF4805410881549800506D5013CF9D1C1
:100BC0001A8E013292B21A8615E00A8892B242F465
:100BD00080720A800D498A8892B242F440728A80FB
:100BE0004FF48054597C084A51B1013CFAD1138E1C
:100BF00001339BB213860120F4F7F8FB204610BDA9
:100C0000147C84F0010010BDFC3A00200058004024
:100C1000F0B51B4C4FF6FF762746A3894FF47A7345
:100C20008AB111B10D78013100E0FF25B4F808E078
:100C30001EF0020F09D0ADB2BD814FF47A73258941
:100C4000ED0718D510E00120F0BD013B9BB2B34287
:100C5000ECD10C4A538B01339BB25383508B80B23F
:100C6000003018BF0120F0BDBD89ADB208B10570DC
:100C70000130013AD4E7013B9BB2B342DFD1E8E750
:100C8000003800407003002040F2E93310B51049ED
:100C90000C890F4AA40709D540F2E93380B290814C
:100CA0001189C9070ED50A4B988909E0013B9BB20F
:100CB000002BEDD1074A538B01339BB25383508BEA
:100CC000C0B210BD013B9BB2002BE9D1F2E700BFDF
:100CD000003800407003002010B50446006801F0A1
:100CE00073FD606801F070FDA068BDE8104001F080
:100CF0006BBD10B5094B03F1500293F8AD1481425E
:100D000005D193F8AF4493F8B0148C4204D3043364
:100D10009342F2D1002010BD012010BD303B0020D5
:100D20001949F0B50D4691F8AC35D1F8B0750022EF
:100D30004FF00C0E042B1CD8591C07EBC3039E1C50
:100D4000C9B213D09A88D40710D510420ED093F9A7
:100D5000026000230EFB03F20B4C04F2B45C12F9A8
:100D60000CC0B4450AD00133052BF3D101220B4648
:100D7000E0E70AB185F8AC350020F0BD224484F8E4
:100D8000AC15D2F8B805F0BDFC3A0020024B0022A9
:100D900083F8AC25C4E700BFFC3A00202DE9F04FF2
:100DA000012085B0FBF728FA1A4EDFF86CA000246A
:100DB00006F5BE6B50B3012C28D84FF04C0909FB47
:100DC00004F806EB0807D7F8F05515B10134E4B282
:100DD000F0E70379032290F900005AF823300092DB
:100DE00001952A460121FBF773F9039050B14A4659
:100DF00029460BEB080008F049F8039B0134C7F8BB
:100E0000F035E4B20120FBF7D7F9D3E705B0BDE830
:100E1000F08F00BFFC3A002080B10108F0B50C460D
:100E2000054689B014220021204608F02FF804A9B5
:100E30002A680D461E4EC2F38550002340FA03F780
:100E4000FF0748BF9F5D03F1010344BF0F700131ED
:100E5000062BF3D1174800230B70C2F30321014482
:100E600091F82610C2F305368DF818102D300DF1CB
:100E7000190146FA03F7FF0748BF1F5C03F101039E
:100E800044BF0F700131062BF3D100230B70C2F366
:100E90008343029306AB0193009502F00F030649CA
:100EA000C2F303122046FFF7CDFD09B0F0BD00BF2D
:100EB000A0B1010880B101082CD3010838B50E4C4F
:100EC00094F88F1684F88B0601F03F018B1C01F11A
:100ED0000A0584F88D3684F88A5604F5D160083105
:100EE000F7F7D6FD254485F8860694F88A36000A79
:100EF0001C4484F8870638BDFC3A002008B5002061
:100F0000FDF7BCFB0020FDF7B9FB0020FDF7B6FBA9
:100F1000BDE808400020FDF7B1BB73B5214C04F2D9
:100F2000B463C4F8B03694F874325BB1012B14D1B9
:100F3000032284F8B626072284F8B83684F8B72648
:100F40000C2308E0022284F8B626032284F8B8367F
:100F500084F8B726072384F8B436134A134B40208D
:100F60001A62FBF749F90546C8B1FDF75DFC002898
:100F700014BF0323012395F9006005460022019266
:100F800000930B4A4FF4E13340213046FBF7A0F8C1
:100F90000DB1C4F8BC06003018BF0120FFE702B055
:100FA00070BD00BFFC3A0020B17E00087003002035
:100FB000218100082DE9F843AC4BAD4C1D68237826
:100FC00043B1AC4B1B68EB1A002BA1BFAA4A00230C
:100FD00023701370A94B1E6842F2010333400BB912
:100FE000A44A1371300740F10882A54B1B681B7A95
:100FF000082B00F2EA81DFE813F009000900340051
:10100000CE000801310131016F01B4019D4B1A7806
:10101000002A00F0DA8100221A709B4B9B4993F85A
:1010200000E09B4BDFF8A4921B68022293F800C0FB
:10103000984B93F800808B5C571C43FA0EF303F037
:101040000F03634509D20B2B07D8885CCF5D00EAFC
:10105000080007EB002049F823000232102AEAD1E9
:10106000ADE18D4B1A78002A00F0AF8100221A7092
:101070008A4B8B4A93F802E0DF7859780EF007002C
:1010800041EA002107F03F00400140EADE00116024
:10109000197950605879890093F806E041EA971170
:1010A00000F0010741EA87219160DF790EF00F011E
:1010B000C90141EA500107F07F00D1600001197AAF
:1010C00040EA1E1093F809E04900106141EAD71187
:1010D0000EF003009F7A41EA40215161D97A07F06E
:1010E0001F008001C90040EA9E0041EA571193F8B1
:1010F0000DE09F7BD161197B90610EF0070041EA02
:10110000002107F03F00400140EADE001162D97B78
:101110005062187C890093F811E041EA971100F0C1
:10112000010741EA872191629F7C0EF00F01C901FE
:1011300041EA500107F07F00000140EA1E101063F1
:10114000D162D97C93F814E0490041EAD7110EF03E
:10115000030041EA40215163997D5F7DC900DB7D39
:1011600041EA5711D163D9074CBF40F21471AD2148
:1011700007F01F009F07116448BF40F214714FEA47
:10118000801040EA9E0058BFAD219063180751645B
:1011900000F11D8113E1434A1378002B00F0158103
:1011A00000231370404A414F1078414907EB400E2D
:1011B000B1F800C09EF803809EF8041041EA0821AF
:1011C0008C4540F002817978012904D0812940F0D2
:1011D000FF80032300E00B46102884BF102111700C
:1011E000DFF8ECE0334917780022D0B2874201F1F2
:1011F000020140F2ED8011F802CC11F8010C40EA36
:101200000C202EF812000132EFE72B4B1A78002A3F
:1012100000F0DB8000221A70284B1A789846A82A22
:1012200040F0D380DF7C002F40F0CF80DFF8A49027
:1012300008EB4703D8781B7903EB002002F094FCFD
:101240001F4902F09DFD1F4902F0DCFB02F0E6FEA3
:1012500049F827000137082FEAD1B0E01A4B1A7875
:10126000002A00F0B28000221A70A8E0380D002099
:10127000640D0020C0410020650D0020541700209F
:1012800050170020FD150020B2410020ED15002070
:10129000AC410020B34100201E160020051600209E
:1012A000DC140020BD150020C0150020C115002051
:1012B000BE150020C4150020B6150020A115002081
:1012C000CDCCCC400080BB436A140020AC1400207D
:1012D0008C1400206C140020634B1A78002A74D000
:1012E00000221A70614B1988614B1878614B1844C1
:1012F00010F8017C10F8020C00EB07275E48BFB223
:101300000078012812D15D4A127802F11C0E5FFAB2
:101310008EFE981890F801C0985C023200EB0C2009
:10132000D2B20144964589B2F3D105E0985C01320E
:10133000091A1E2A89B2F9D18F4246D14F4A504824
:1013400092F800E000220EEB4201C9B25F187F78EC
:10135000595C01EB072140F8221001320E2AF2D12C
:101360002DE0DFF8408198F800304746022B2CD161
:10137000DFF8349199F802104846F7F789FB00BB73
:1013800099F8002099F8013043EA022343F60162FC
:10139000934203D043F6036293420ED139480023AF
:1013A00009EB030191F807E08A7902EB0E22C2F300
:1013B000CC021A520233202BF2D100233B700123BE
:1013C00006E0002388F8003002E0002300E0032359
:1013D000D90712D52C4A03F00203002B4FF001016C
:1013E0002A4B117108BF002119700CBF0123002383
:1013F000237005F5C333A0331360F20710D5244BD7
:101400001978214B5A798A420AD0224A0120107059
:10141000214A0020107005F5C332A0321A605971BC
:10142000B30407D51D4A002332F8131079B90133EC
:101430000C2BF9D1144B1B7933B9194B1868281AA6
:10144000C043C00FBDE8F8830120BDE8F883114B0D
:1014500001221A70104B00221A7005F5C3330A4A94
:10146000A0331360E6E700BF8F1600206C16002043
:101470006B1600206F1600206A1600206E160020E2
:101480005C1500203C150020C04100200400002015
:10149000A2340020650D0020050000202415002046
:1014A0003C0D0020261600202C1600202DE9F047C8
:1014B000734E33689A0768D545F20721714B724C19
:1014C0001A68A368D31A8B425FDD704DA260F7F7EC
:1014D00093F92B786E4F032B3B881FD10A2B26D90B
:1014E000002328202B70FFF757FAF7F785F9694B8F
:1014F0001888F7F76BF9684B1A68D37890FBF3F00C
:1015000001300828654BA8BF08201870537980B2B5
:101510004343A38113795843E08108E00A2B06D89E
:1015200003235E4A2B7000231370A381E3812B7881
:10153000564A012B0ED002D3022B1FD025E056496C
:10154000A38909683A8889795B1A9A421DDC0123CC
:101550002B7011E05048E3890068398880791B1AA4
:10156000994202DC022313700CE0474B9B898B42AB
:1015700002D20023137008E0082004E03A88E389CF
:101580009A42E4D80720FAF721FFD6F800A01AF40F
:10159000006F73D03B4B3C4C1B682269C2EB0308C5
:1015A00045F20722904569DD23613D4B3D4EB3F97D
:1015B0000650394BA5F57A751F683B7B012B03D08C
:1015C00045D3022B1FD044E0374B61695A7C374B1F
:1015D000082033F8122091FBF0F392B2C91A8B184D
:1015E000636193FBF0F3228340F6E4429BB25343E2
:1015F0007A89C2EB13334FF47A725343B7F9082058
:1016000093FBF2F324E02A4B2A481B78B7F80A90A0
:101610005B07B0F8DC10C6F800901AD500F50E7024
:10162000FAF76EFE18B91AF0100F18BF002505FB67
:1016300005F3322293FBF2F31D44B7F908305D4302
:101640004FF47A7395FBF3F54D44356001E00023C8
:1016500033603368D4E9080103FB08F84FF47A7368
:1016600098FBF3F810EB080041EBE8710023C4E9A4
:101670000801114A02F0F2FC104B1860BDE8F08737
:1016800054170020380D0020C0410020CE37002024
:1016900014170020E8160020C41600206403002060
:1016A000B01F002020130020CC160020E0160020E0
:1016B000F8350020303B0020407E0500C816002091
:1016C000344B2DE9F0411B68DB0402D50A20FAF700
:1016D0007DFE314C2268002A59D0304F304E396897
:1016E0003368994253D32F4B2F4D1878516808BB5C
:1016F000012018702B88CB5C002B3BD013782B4A31
:10170000013BD2F85C2500FA03F3134201D1F9F74B
:1017100033FD274B01221A70F7F7D2F92B88C3B992
:1017200023681B78053B012B13D8FFF7F7F8214BF3
:1017300098620EE04FF0000883F800802B88CB5CA5
:10174000C3B14046F9F718FD194B83F80080F7F74D
:10175000B7F923682A885B689B5CFE2B04D1124B87
:1017600000221A80BDE8F081FF2B07D1BDE8F041CF
:10177000FAF714BE23682A885B689B5C39680A20E4
:1017800000FB0313013233602A80BDE8F081BDE81D
:10179000F08100BFF435002084270020841700204A
:1017A0007C2700207B27002080270020303B002062
:1017B000AC170020C04100202DE9F04F8E4E8BB0B9
:1017C00033688E4D13F0020F00F020848C4C237888
:1017D000002B00F01B84FFF7A1F8D5F80090D5F896
:1017E000048009FB09FB08FB08BBAF68636807FBC3
:1017F00007BBC31A834A0493642303FB0BF3B2F8B9
:1018000008B060600BFB0BFB93FBFBFBABF15203DF
:101810000893336813F008030BD07B4A13682BB18D
:1018200053681BB19368003318BF012303F001050F
:1018300000E01D46049802F097F9744902F0ECF9B3
:10184000734EA4680090306802F092F9214602F0CD
:10185000E3F90190706802F08BF9214602F0DCF99F
:101860000290B06802F084F9214602F0D5F9664B87
:1018700001991A68039005925A689B680846069277
:10188000079302F0C9F902990446084602F0C4F928
:101890000146204602F0B8F803990446084602F0D3
:1018A000BBF90146204602F0AFF805F001FB0990B4
:1018B000002D00F0B380059802F05AF9064606980C
:1018C00002F056F90546079802F052F931460446EF
:1018D000304602F0A1F929468246284602F09CF9DA
:1018E0000146504602F090F821468246204602F01A
:1018F00093F90146504602F087F84649824602F0C5
:1019000047FB002800F08A80504605F0D1FA0146D6
:101910004FF07E5002F034FA83460146304602F022
:101920007BF959468246284602F076F95946064622
:10193000204602F071F9384C05462168504602F005
:101940006BF961680590304602F066F9059B014627
:10195000184602F059F8A1680590284602F05CF993
:10196000059B0146184602F04FF8E1680590504685
:1019700002F052F921698246304602F04DF90146E3
:10198000504602F041F861690646284602F044F9E3
:101990000146304602F038F8059B054619461846C0
:1019A00002F03AF929460646284602F035F9014682
:1019B000304602F029F805F07BFA0146284602F08D
:1019C0002BF900F1004AA169504602F025F90021E7
:1019D00002F01AF8E1690646504602F01DF90021AE
:1019E00002F012F8216A0546504602F015F900216E
:1019F00002F00AF8044614E0502D00200C130020D9
:101A0000EC410020002D0020740A0020BD378635EF
:101A1000C01F00200AD7233CD03A002000242546CE
:101A20002646089B262B7DD8484602F0A1F8814621
:101A3000404602F09DF88046384602F099F8494643
:101A40000746484602F0E8F841468246404602F022
:101A5000E3F80146504601F0D7FF39468246384642
:101A600002F0DAF80146504601F0CEFF51498246B5
:101A700002F08EFA002855D0504605F019FA0146BA
:101A80004FF07E5002F07CF982460146484602F053
:101A9000C3F851468146404602F0BEF851468046A2
:101AA000384602F0B9F8444F83463B6A404619462F
:101AB000069302F0B1F8D7F81CA00590514658469D
:101AC00002F0AAF8059A0146104601F09BFF014674
:101AD000304601F099FFBF6906463946584602F084
:101AE0009BF8069B83461946484602F095F8014646
:101AF000584601F087FF0146284601F085FF514610
:101B00000546484602F088F839468146404602F0CC
:101B100083F80146484601F075FF0146204601F072
:101B200073FF0446254B4FF0000AD3F8009051464E
:101B3000D9F80480224F404602F02AFA30B32149F6
:101B4000099802F007FA38B33146404602F064F8CB
:101B5000009902F061F8F96801F056FF2946F86033
:101B6000404602F059F8009902F056F8396901F040
:101B70004BFF21463861404602F04EF8009902F0D2
:101B80004BF8796901F040FF786105E0C7F80CA0D7
:101B9000C7F810A0C7F814A00B4BD9F808001B78A1
:101BA0005A0717D4094B1A6844F61F639A4211D892
:101BB000074911E00AD7233CD03A002080180020C2
:101BC000EC410020C2B8B23EF83500208417002056
:101BD000000020414FF07E5102F01EF88046014681
:101BE000304602F019F8F96801F00EFF019901F092
:101BF0000BFF41460646284602F00EF8396901F00F
